:100000000C9479190D9434030D9465030D949603A3
:100010000D94C7030D94F8030D9429040D945A040C
:100020000D948B040C9436760C94AA190C94AA198E
:100030000C94AA190C94AA190C94AA190C94AA1934
:100040000C94AA190C94AA190C94AA190C94AA1924
:100050000C94AA190C94AA190C94AA190D94BC0416
:100060000C94AA190D9425090D945B090C94AA19F6
:100070000C94AA190C94AA190C94AA190C94AA19F4
:100080000C94AA190C94AA190C94AA190C946CB685
:100090000D94D2090D94080A0C94AA190C94FF1B14
:1000A0000C94AA190C94AA190C94AA190C94AA19C4
:1000B0000C94AA190C94AA190C94AA190C94AA19B4
:1000C0000C94AA190C94AA190C94AA190C94AA19A4
:1000D0000C94AA190C94AA190C94AA190C94AA1994
:1000E0000C94AA190C94AA190C94AA190C94AA1984
:1000F0000C94AA190C94AA190C94AA190C94AA1974
:100100000C94AA190C94AA190C94AA190C94D375DE
:100110000C94E2750C94AA190C94AA190C94AA19BF
:100120000C94AA190C94AA190C94AA190C94AA1943
:100130000C94AA19CBA8CBA867A87CA89AA8CBA88E
:10014000D7A8E2A81DA91DA9A7A949A95FA91DA90A
:10015000B1A9A7A986C583C583C583C589C59CC523
:1001600083C599C599C599C599C599C583C599C5CB
:1001700099C599C5A7C6AEC6EEC6EEC6EEC6EEC612
:10018000D1C8EEC6EEC6BD03F70397035D02A30414
:100190009103930181048304070285024D03AD049A
:1001A0009F0383031D0237022903C504E5010704E9
:1001B000AD048D0397019B03FB038D02B902550427
:1001C0005F015B03DB03B9042D030D022102E10390
:1001D000E70231025B037F016F01D50207634236FC
:1001E000B79BD8A71A39685618AEBAAB558C1D3CC8
:1001F000B7CC5763BD6DEDFD753EF6177231BF008C
:100200000000803F08000000BE922449123EABAAC5
:10021000AA2ABECDCCCC4C3E00000080BEABAAAA20
:10022000AA3E00000000BF000000803F0000000068
:1002300000084178D3BB4387D1133D190E3CC3BDA1
:100240004282AD2B3E68EC8276BED98FE1A93E4C4E
:1002500080EFFFBE01C4FF7F3F00000000000C9450
:10026000DE360C9464C10C9469AE0C9449890C94EC
:10027000F19C0C9436B20C942EA50C94384F0C942F
:1002800018370C948C500C94733D0D940E020C9402
:10029000EB660C94098D0C94CB520C9400F80C94E2
:1002A0002F520C946D650C94E44E0C94FD360C9416
:1002B00068AD0C943F4A0C94715E0C94539A0D9463
:1002C000CA060C9430A80C949A500C94E1930C94A8
:1002D0005F8B0C9410560C942A370C9423390D9490
:1002E000FF060C94A2DD0C94F1360C9470460C942D
:1002F000B9B40C94C0940C9497B60C94C19C0D9412
:10030000FB060C944F1A0D9465020C94F6390C946C
:10031000969F0C94B4B60C9451960C9479310C942D
:10032000EC940C942B3A0D9427030C9414370D94F1
:1003300098060C946F810C9499AD0C94C94A0C9456
:10034000385F0C942DE70C949CC50C946E840C942F
:10035000B78A0C94AA360D94320A0C940F370D9478
:10036000A6020C94EEF70C94EDA10C9463520C943D
:10037000443C0C94B5490C94C18D0C94956B0D9430
:100380005E080C94096B0D943C080C9439680C942D
:10039000844A0C9440540C94D49A0C94805A0C9433
:1003A000DC360C9423960C94E12E0C94804D0C9426
:1003B00012840C945E370C94353A0C9434370C94B8
:1003C000E2A80C9459DD0C941D370D947A060C9418
:1003D0006DDD0C9452440C9449A90C9406370C948E
:1003E000E5930C949D740C943F3F0C94A7510C948E
:1003F000E6480C946CC10C9448950C94CC570C9422
:10040000DBDC0C9426840C9436840C9467A80D9441
:100410001F060C94F88A0C94D59F0D94E3060D9456
:100420003C0A0C944E530C9459BE0C94398B0C948A
:100430003E530C947D890C9455900D944D060C946C
:10044000A4DE0D94E7060C9480D80C94529A0C9478
:100450009C330C94963D0C94CBA80C9455B40C94FE
:10046000B8400D94F5060C9449520C94A9F50D94DE
:1004700057060D94E8070C94479B0C945FA90C94C5
:10048000392A0D9498020C944EAD0C94AB9F0C94A9
:1004900087940C944B2A0C94F59A0C94E4930C9446
:1004A000E0870C940ADF0C940BD60C942B490D9426
:1004B00051020C94061A0C949E600D94EC020C945C
:1004C000708C0C94473E0C942BA50C940E660C94E7
:1004D000024F0D94AD020C944DDC0C944F900C9493
:1004E00018950C94DC2B0C9401580C9483C50C9437
:1004F00056E30C9461B40C9483DD0C94343E0C945C
:1005000050B60C94AAE20C94711A0D9429060C941E
:1005100051390C9448D60C94E93D0D94D1060C94B5
:10052000EEE60C94524F0C94B49F0C9412D60C949B
:1005300053DE0C94F9A50C9419500C94203E0C94A5
:10054000E09F0C9470490C9468B40C9459840C94FA
:100550001D1B0C94B79B0C94BFAD0C940E4B0C94CC
:10056000AFD60C94E19C0C9459440C944FE90C9434
:10057000EEC60D94C0060C947E9C0C94F99C0C94D1
:10058000193A0C94721A0C9466FC0C9440DE0C948C
:10059000DFB60C9445B40C9460400C9428A20D94E2
:1005A0006A020C94CAAE0C9473530D9403070C9416
:1005B000FA490C94A8420C94223A0C9467B40C9417
:1005C00047AD0C947B5B0C94DB470C9445A20D94D7
:1005D000F1060C949BD60C94D7E70C9449DD0C944F
:1005E000448D0C94E9430C9462740C94313F0C9448
:1005F0006F510C94EA9F0C941FA70C947E500D949D
:10060000DA070C9499C50C94E8360C947CA80C94E9
:10061000D8B00C943AC10C9451E70C94DCDF0C94E4
:100620000B960C9478C10C9402A10C948CDE0C9463
:100630000B900C9486C50C94A29F0D9406050D9406
:10064000FC070C94BB890C9440AD0C94005B0C949B
:10065000D71F0D9461060C941BA20D94DF060C9419
:100660008A950C941DA90C9474AF0C9443610C945E
:10067000FB240C9449AD0C94155C0C949FA10C9434
:10068000E4470C94B0D60C9432960C94E0DD0C94B4
:1006900032B50C944F9A0C9410970D9433060C9429
:1006A00085D60C94428A0C942DAB0C94283F0C9464
:1006B00055510C94D9730D9408070C9415E30C94C0
:1006C000E29C0C94FD560C9418C10C9458C10C94E7
:1006D000AEC60C94C1510C94944F0C9449410C94A7
:1006E000C1DD0D94CD070C9455AE0C94714B0C9458
:1006F000B0540C944AAD0C94955C0C94C2B60C9416
:1007000046390C94E6A00D9445060C94318F0C9458
:1007100040DF0C9464A10C9494C10D948E060C944B
:1007200070500D941A030C94534B0C9423C10D94E8
:10073000E0020C94A7A90D94A2060C9464810D9478
:100740003D060D9421020C9430690C948C210C947C
:1007500065640C943E4E0C945EC10C9401970C940D
:10076000B3700C94DF500C949D3E0D949F020C943A
:10077000056A0C9439C10D94F80A0D940E030C947B
:1007800026BE0C94CC5F0C94621A0C94FB430C9420
:10079000F2430C9413E70C949F1A0C94CE960C948D
:1007A00051B40C941E9B0C94D1A50C94A84F0D949D
:1007B000CF070C94CA9F0D94D5060C940BDE0C94B5
:1007C000DE890D94ED060C94A6380C941CDE0C9476
:1007D000CC950C942A250C9447370C94E9640C941E
:1007E000472A0C9455E70C94DE9C0C94BF9F0D9403
:1007F000D8020C9420840D94CE060C94A1480C943D
:1008000065B30C94D7A80C94D98F0C94A7C60D94FB
:1008100084060C9442C10C94CBDE0D948F090C9489
:1008200072C10C94108A0C942F370C9437FC0C94E2
:10083000C9470D9485090C94B7B60C94D1C80C9493
:10084000E0B10C941F4F0C944C8B0C9490D60D94EB
:100850007F0A0C944AAB0C948D510C94363F0C9447
:100860003B580C948F450C94B8B60C94F8E50C9456
:100870002B8C0D947C020C9474620C94034E0C949B
:1008800090D20C945C480C9466DE0C948FA60C9469
:1008900062500C94FBF10C94471A0C943D840C9418
:1008A00072E90C94864C0D9424020D94C4060C94A9
:1008B000E0610C949D470C94FD3A0C947AD60C940C
:1008C000D6630C94204E0C942F920C94DB510C9414
:1008D000D2470C945D3E0C94EDB50C94DD830C94E2
:1008E00032DC0C94768A0C94999F0C94FDD50C9470
:1008F000684C0C9489C50C94B0B50C947A470C9450
:1009000008D60D9415060D941A060D9416020C9433
:1009100021370C94D68C0C944F840C94972C0D9406
:100920006B020C94EEDE0C9485D20C9425370C945B
:10093000B1A90C94EE8F0C9479870C945B670C949E
:1009400018AF0C942FDE0D94F9020C9454890D9479
:1009500034020C947ADE0C9442B40D94AC060C94E0
:10096000C0A90C94C93E0C9424510C949AA80C94E0
:10097000112B0D94D9060C944DAD0C942D5D0C9457
:1009800038A60C944E500D94D50A0D946B06756ED6
:100990006B6E6F776E0032204D622F730031204DE9
:1009A000622F7300353030206B622F730032353088
:1009B000206B622F7300756E6B6E6F776E002D313A
:1009C000362E352064426D002D31312E35206442A3
:1009D0006D002D382E352064426D002D362E3520C9
:1009E00064426D002D342E352064426D002D332E6F
:1009F000352064426D002D322E352064426D002D6D
:100A0000312E352064426D002D302E352064426D2C
:100A100000302E352064426D00312E322064426D4C
:100A200000312E382064426D00322E332064426D36
:100A300000322E382064426D00332E332064426D24
:100A400000332E352064426D00556E6B6E6F776EED
:100A5000204361757365205265736574004A544183
:100A600047005761746368646F670042726F776E06
:100A70002D6F75740045787465726E616C00506FEF
:100A80007765722D6F6E0029002C002C0052756E58
:100A90006E696E673A20616E616C6F6750696E4572
:100AA00076656E7448616E646C6572280029002C4E
:100AB000002C0052756E6E696E673A206469676932
:100AC00074616C50696E4576656E7448616E646CD5
:100AD0006572280070776D00696E7075745F70754F
:100AE0006C6C7570006F757470757400696E7075DC
:100AF000740064697361626C656400726573657229
:100B000076656400756E73657400646973636F6EF7
:100B10006E65637465640072756E6E696E672065DC
:100B200076616C206F663A2000290052756E6E69FE
:100B30006E673A2074656D70657261747572654593
:100B400076656E7448616E646C6572280029005287
:100B5000756E6E696E673A20626174746572794170
:100B60006C61726D5472696767657265644576651C
:100B70006E7448616E646C65722800290052756E4F
:100B80006E696E673A206261747465727943686158
:100B90007267696E674576656E7448616E646C65F0
:100BA000722800290052756E6E696E673A20626184
:100BB000747465727950657263656E7461676545BA
:100BC00076656E7448616E646C6572280072783068
:100BD00000007478300000643200000064330000CC
:100BE000006434000000643500000064360000003A
:100BF0006437000000643800000073730000006D6B
:100C00006F7369006D69736F0073636B00007278B6
:100C1000310000747831000073636C00007364610C
:100C2000000076636300006261747400626B706B35
:100C30000063686700006C656462006C6564720044
:100C40006C65646700613000000061310000006184
:100C500032000000613300000061340000006135A3
:100C6000000000613600000061370000007365720B
:100C700076657220756E7661696C61626C65004D97
:100C800065736820616E6E6F756E6365206661695D
:100C90006C65643A200020006D65736820616E6E9B
:100CA0006F756E63696E6720746F200052455452F1
:100CB00059006572726F723A2000737563636573D1
:100CC000730020204D65737361676520636F6E66E6
:100CD00069726D6174696F6E202D20002D3E63680E
:100CE000756E6B00206C656E2000636F6D6D616EBC
:100CF000643A200069643A2000746F3A2000696EFB
:100D000076616C696420636F6D6D616E642C207216
:100D10006571756972657320746F2C2069642C206D
:100D2000636F6D6D616E6400636F6D6D616E642ED7
:100D3000616C6C282268712E6F6E6C696E65222C56
:100D400032290048512061636B2764004A534F4E9B
:100D5000207061727365206661696C6564006C6FF8
:100D60006F6B696E6720666F72207061636B65746C
:100D700020696E3A2000207365636F6E6473207380
:100D8000696E6365206C61737420485120616374DF
:100D900069766974792C207265636F6E6E65637411
:100DA000696E67003A005265636569766564206123
:100DB0006E737765722066726F6D2053636F757402
:100DC00020004D554C544943415354206F6E2077B9
:100DD000726F6E6720656E64706F696E7400524545
:100DE000545259006572726F723A200073756363D2
:100DF0006573730020204D65737361676520636FB1
:100E00006E6669726D6174696F6E202D20002D3ED3
:100E10006368756E6B00206C656E2000676F7420D0
:100E2000726573756C74200072756E6E696E6720E2
:100E3000636F6D6D616E64200077616974696E67C0
:100E400020666F72206D6F72650063616E2774207B
:100E50007265636569766520636F6D6D616E642090
:100E60007768696C652073656E64696E6720616E72
:100E70007377657200727373693A20002020006CEA
:100E800071693A2000526563656976656420636F15
:100E90006D6D616E64005369676E616C6C696E673D
:100EA0002048513A20004851206F66666C696E6593
:100EB0002C2063616E2774207369676E616C006D0E
:100EC000756C74696361737420696E200072756E4D
:100ED0006E696E672064656C6179276420636F6D4D
:100EE0006D616E643A2000204669656C642053632E
:100EF0006F757420726561647900204C65616420AF
:100F000053636F757420726561647900206279742F
:100F100065732066726565002000290020536B65AB
:100F200074636820287265762000200020285368AA
:100F3000656C6C206261736564206F6E2042697419
:100F40006C6173682076322E30202863292032307D
:100F500031342042696C6C20526F79290048656CED
:100F60006C6F2066726F6D2050696E6F6363696F7E
:100F700021003E20006C6F6F6B696E6720666F7298
:100F800020636F6D6D616E642000726566726573BB
:100F900068656420637573746F6D20636F6D6D6138
:100FA0006E647320696E64657820746F3A20005017
:100FB000696E206D75737420626520636F6E66695B
:100FC000677572656420617320696E707574004383
:100FD000616E6E6F7420656E61626C652077616B07
:100FE000657570206F6E206120726573657276651D
:100FF000642070696E0057616B657570206E6F7448
:1010000020737570706F7274656420666F722074DF
:101010006869732070696E00496E76616C6964203E
:1010200070696E206E756D626572007573616765BB
:101030003A20706F7765722E77616B6575702E70D0
:10104000696E282270696E4E616D65222C205B6589
:101050006E61626C655D290075736167653A206D2C
:101060006573682E636F6E6669672873636F757446
:1010700049642C2074726F6F704964205B2C20636C
:1010800068616E6E656C3D32302C206B65795D2930
:101090000075736167653A206D6573682E736574BA
:1010A0006368616E6E656C286368616E6E656C293D
:1010B0000075736167653A206D6573682E7365749A
:1010C000706F77657228706F7765724C6576656CA6
:1010D000290075736167653A206D6573682E7365C5
:1010E00074646174617261746528646174615261D1
:1010F0007465290075736167653A206D6573682EA4
:101100007365746B657928226B6579222900757384
:101110006167653A206D6573682E6A6F696E6772E4
:101120006F75702867726F757049642900757361F7
:1011300067653A206D6573682E6C656176656772C8
:101140006F75702867726F757049642900757361D7
:1011500067653A206D6573682E696E67726F75708A
:101160002867726F75704964290075736167653A05
:10117000206D6573682E766572626F736528666C84
:101180006167290020202020207C002020202020B2
:101190007C2020202020002020202020207C2020B7
:1011A000202020002020202020207C202020202003
:1011B00020002020202020207C2020202020200013
:1011C0002020202020207C202020202020002020E3
:1011D000202020207C202020202020007C20202077
:1011E000202020007C202020204669786564202073
:1011F00020207C20204D756C7469636173742020FD
:101200007C2020202053636F7265202020207C20CA
:101210002020204473744164642020207C204E658B
:101220007874486F7041646472207C2020202052C2
:10123000616E6B20202020207C20202020204C511B
:101240004920202020207C00726D206D6573682E5F
:1012500066742E656163683B726D206D6573682EE0
:1012600066742E70696E673B726D206D6573682EB3
:1012700066742E61636B3B6C65642E6F66660072EC
:10128000756E206D6573682E66742E656163682CBB
:101290003530300066756E6374696F6E206D6573EE
:1012A000682E66742E65616368207B206D657368A7
:1012B0002E6561636828226D6573682E66742E70D2
:1012C000696E6722293B7D0066756E6374696F6E77
:1012D000206D6573682E66742E70696E67207B20A2
:1012E000636F6D6D616E642E73636F75742E6163D1
:1012F0006B28226D6573682E66742E61636B222CD9
:101300006172672831292C226C65642E626C7565C8
:10131000222C313030293B207D0066756E63746964
:101320006F6E206D6573682E66742E61636B207B13
:1013300069662861726728312929206C65642E72DC
:1013400065643B20696628617267283229203E2047
:101350003020262620617267283229203C3D203823
:101360003029206C65642E677265656E28313030D7
:10137000293B20696628617267283229203E20387F
:101380003029206C65642E79656C6C6F773B7D002D
:10139000636F6D6D616E642E6F7468657273282261
:1013A000636F6D6D616E642E73636F7574222C6D47
:1013B0006573682E69642C226D696C6C69732229CF
:1013C0000075736167653A206D6573682E6669659F
:1013D0006C6474657374287365636F6E647329003D
:1013E00075736167653A206D6573682E6561636822
:1013F0002822636F6D6D616E64222900636F6D6DCD
:10140000616E6420746F6F206C6F6E672C203130BA
:1014100030206D6178006275737920636F6D6D6146
:101420006E64696E6720616C7265616479007573C2
:101430006167653A20636F6D6D616E642E73636FD3
:1014400075742873636F757449642C2022636F6D03
:101450006D616E6422205B2C617267312C61726752
:10146000325D2900636F6D6D616E6420746F6F2053
:101470006C6F6E672C20313030206D6178006275A2
:10148000737920636F6D6D616E64696E6720616C46
:1014900072656164790075736167653A20636F6D89
:1014A0006D616E642E73636F75742E61636B282299
:1014B00063616C6C6261636B222C2073636F757463
:1014C00049642C2022636F6D6D616E6422205B2C59
:1014D000617267312C617267325D2900636F6D6DD7
:1014E000616E6420746F6F206C6F6E672C203130DA
:1014F00030206D6178006275737920636F6D6D6166
:101500006E64696E6720616C7265616479007573E1
:101510006167653A20636F6D6D616E642E616C6CFE
:101520002822636F6D6D616E6422205B2C6172678F
:10153000312C617267325D2900636F6D6D616E647D
:1015400020746F6F206C6F6E672C20313030206DEF
:101550006178006275737920636F6D6D616E646987
:101560006E6720616C72656164790075736167658F
:101570003A20636F6D6D616E642E6F74686572736F
:101580002822636F6D6D616E6422205B2C6172672F
:10159000312C617267325D290029002800756E6B5D
:1015A0006E6F776E206661696C7572653A200050C7
:1015B0006879736963616C206368616E6E656C2025
:1015C000616363657373206661696C7572653A2047
:1015D000004E6F20726F75746520746F20646573A0
:1015E00074696E6174696F6E3A20004E6F2061639A
:1015F0006B6E6F776C656467656D656E7420726580
:101600006365697665643A20004F7574206F6620C3
:101610006D656D6F72793A20004572726F723A2073
:101620000029002028436F6E6669726D656420771B
:1016300069746820636F6E74726F6C206279746570
:101640003A20002D2020436F6D6D616E642073750C
:10165000636365737366756C6C792073656E742053
:10166000746F2053636F757420002061636B2000DA
:101670003A20003A200053656E7420636F6D6D61EF
:101680006E6420746F2053636F75742000636F6DF8
:101690006D616E6420746F6F206C6F6E672C2031EB
:1016A0003030206D6178006275737920636F6D6DE5
:1016B000616E64696E6720616C7265616479007542
:1016C000736167653A20636F6D6D616E642E67723A
:1016D0006F75702867726F757049642C2022636F74
:1016E0006D6D616E6422205B2C617267312C6172BA
:1016F00067325D29006D73006F6E2E6D65737361C7
:1017000067652E7369676E616C206576656E7420FF
:1017100068616E646C657220746F6F6B20002900C5
:101720002800756E6B6E6F776E206661696C7572DE
:10173000653A2000506879736963616C2063686161
:101740006E6E656C20616363657373206661696C9E
:101750007572653A20004E6F20726F757465207443
:101760006F2064657374696E6174696F6E3A2000EE
:101770004E6F2061636B6E6F776C656467656D6536
:101780006E742072656365697665643A20004F75F2
:1017900074206F66206D656D6F72793A2000457216
:1017A000726F723A200029002028436F6E666972BA
:1017B0006D6564207769746820636F6E74726F6CF6
:1017C00020627974653A20002D20204D6573736185
:1017D0006765207375636365737366756C6C7920D8
:1017E00073656E7420746F2053636F757420003AB4
:1017F000200053656E74206D657373616765207496
:101800006F2053636F7574200075736167653A20AC
:101810006D6573736167652E73636F757428736389
:101820006F757449642C20226D657373616765223E
:10183000290075736167653A206D6573736167652B
:101840002E67726F75702867726F757049642C20EF
:10185000226D657373616765222900757361676521
:101860003A2074656D70657261747572652E73656A
:10187000746F66667365742876616C75652900758A
:10188000736167653A2074656D7065726174757215
:10189000652E63616C6962726174652876616C752E
:1018A00065290072756E6E696E6720616C6C2072BE
:1018B00065706F7274730041736C6565703A2000D7
:1018C0004177616B653A2000546F74616C3A200077
:1018D00075736167653A206C65642E626C696E6B26
:1018E000287265642C20677265656E2C20626C75A9
:1018F000652C206D733D3530302C20636F6E74691C
:101900006E756F75733D30290075736167653A2098
:101910006C65642E736574686578282268657876CE
:10192000616C756522290075736167653A206C6585
:10193000642E736574726762287265642C20677206
:1019400065656E2C20626C7565290075736167652D
:101950003A206C65642E73617665746F72636828D3
:101960007265642C20677265656E2C20626C7565EB
:10197000290075736167653A2070696E2E6D616B21
:1019800065696E707574282270696E4E616D65228E
:101990002C20696E707574547970653D494E5055B0
:1019A000545F50554C4C5550290075736167653A2A
:1019B0002070696E2E6D616B656F7574707574281B
:1019C0002270696E4E616D652229007573616765CD
:1019D0003A2070696E2E6D616B6570776D2822708C
:1019E000696E4E616D6522290075736167653A20E5
:1019F00070696E2E6D616B65646973636F6E6E6581
:101A000063746564282270696E4E616D65222900D9
:101A100075736167653A2070696E2E6469736162DF
:101A20006C65282270696E4E616D652229007573A0
:101A30006167653A2070696E2E7365746D6F6465B9
:101A4000282270696E4E616D65222C2070696E4D82
:101A50006F64652900496E76616C69642070696EF7
:101A6000206E756D6265720075736167653A2070EE
:101A7000696E2E72656164282270696E4E616D65B3
:101A8000222900496E76616C69642070696E207647
:101A9000616C756500496E76616C69642050574DC4
:101AA0002076616C75650050696E206D75737420C9
:101AB00062652073657420617320616E206F757498
:101AC000707574206265666F7265207772697469DB
:101AD0006E6700496E76616C69642070696E206E75
:101AE000756D6265720075736167653A2070696E25
:101AF0002E7772697465282270696E4E616D652259
:101B00002C2070696E56616C756529004661696CA0
:101B1000656420746F206368616E67652070696E0C
:101B2000206D6F646500496E76616C696420706930
:101B30006E206D6F64650050574D206D6F64652099
:101B40006E6F7420737570706F72746564206F6E41
:101B500020746869732070696E0043616E6E6F74E3
:101B6000206368616E6765206D6F6465206F662015
:101B700072657365727665642070696E00496E7671
:101B8000616C69642070696E206E756D62657200AB
:101B900075736167653A2070696E2E73617665288A
:101BA0002270696E4E616D65222C2070696E4D6FDA
:101BB00064652C205B70696E56616C75655D2900EB
:101BC0007D002C007D00300031002C202277616BDD
:101BD000657570223A002C202270776D223A74725B
:101BE000756500222C202276616C223A2200756EE7
:101BF0006B6E6F776E00222C20226D6F6465223A27
:101C00002200223A7B226964223A2200202022000C
:101C10007B0075736167653A2070696E2E6E756D15
:101C2000626572282270696E4E616D6522290075A9
:101C3000736167653A2070696E2E6F7468657273A0
:101C4000646973636F6E6E65637465642829002927
:101C5000002028004572726F722070617273696E85
:101C600067206E616D65003A20004E6F20626163EF
:101C70006B7061636B7320666F756E64004661699B
:101C80006C656420746F20666574636820454550F8
:101C9000524F4D00496E76616C6964206261636BDE
:101CA0007061636B206E756D626572004661696C70
:101CB000656420746F2077726974652045455052C1
:101CC0004F4D004661696C656420746F20757064C7
:101CD00061746520454550524F4D00496E76616CE8
:101CE0006964206261636B7061636B206E756D6205
:101CF00065720020627974657300454550524F4DFE
:101D000020757365643A200020627974657300451C
:101D10004550524F4D2073697A653A20002E780065
:101D2000454550524F4D206C61796F757420766532
:101D30007273696F6E3A20004261636B7061636B0E
:101D400020427573206669726D77617265207665D1
:101D50007273696F6E3A20002E78004261636B7077
:101D600061636B204275732050726F746F636F6C88
:101D70002076657273696F6E3A20005365726961EF
:101D80006C206E756D6265723A203078002E0042CC
:101D90006F617264207265766973696F6E3A2000B4
:101DA0004D6F64656C206E756D6265723A20307897
:101DB000004261636B7061636B206E616D653A20F8
:101DC00000496E76616C6964206261636B70616367
:101DD0006B206E756D626572002C20636F6E74658A
:101DE0006E74203D20003A20646174612C206C6583
:101DF0006E677468203D20006B627073002C206D4C
:101E00006178207370656564203D20003A20693256
:101E1000632C2061646472657373203D2000756ECD
:101E20006B6E6F776E007541002C206D6178696D67
:101E3000756D203D2000756E6B6E6F776E0075417D
:101E4000002C207479706963616C203D2000756EF0
:101E50006B6E6F776E007541002C206D696E696D39
:101E6000756D203D2000706F7765723A2070696E45
:101E7000203D20003A206770696F2C2070696E2029
:101E80003D2000756E6B6E6F776E00627073002C74
:101E9000207370656564203D20002C207278203D01
:101EA00020003A20756172742C207478203D200047
:101EB000756E6B6E6F776E004D687A002C206D61C9
:101EC00078207370656564203D20003A2073706946
:101ED0002C207373203D20004661696C656420747A
:101EE0006F206665746368206F722070617273651D
:101EF000207265736F7572636520646573637269C0
:101F000070746F727300496E76616C6964206261EF
:101F1000636B7061636B206E756D626572004572F4
:101F2000726F723A2057692D466920646972656341
:101F30007420636F6D6D616E64206661696C6564A9
:101F4000004572726F723A2057692D4669206469A4
:101F50007265637420636F6D6D616E642066616984
:101F60006C6564004F6B2C207465726D696E6174D2
:101F7000696E672E20476F6F6462796520446176D1
:101F8000652E00466163746F7279207265736574A3
:101F9000207265717565737465642E2053656E6477
:101FA00020636F6D6D616E6420616761696E20747E
:101FB0006F20636F6E6669726D2E002D2D2D2D2D95
:101FC0002D2D2D2D2D2D2D2D2D00656E61626C6515
:101FD000642020206E616D65004661696C65642037
:101FE000746F20656E61626C65206D6F64756C65E1
:101FF000200075736167653A206D6F64756C652E9E
:10200000656E61626C652822737472696E67220066
:1020100075736167653A2068712E736574746F6BB0
:10202000656E2822746F6B656E220075736167653B
:102030003A2068712E7072696E7428227374726906
:102040006E67220075736167653A2068712E72654C
:10205000706F727428227265706F72746E616D6534
:10206000222C202276616C756522295B2C227661F8
:102070006C7565222E2E2E5D0075736167653A20A2
:1020800068712E7365746164647265737328226865
:102090006F7374225B2C20706F72745D006F6E2EF4
:1020A00068712E6F6E6C696E650075736167653A55
:1020B000206B65792822737472696E6722205B2C0D
:1020C0002074656D705F666C61675D290075736172
:1020D00067653A206B65792E66726565286B657950
:1020E000290075736167653A206B65792E70726996
:1020F0006E74286B6579290075736167653A206B8A
:1021000065792E6E756D626572286B65792900752B
:10211000736167653A206B65792E73617665282255
:10212000737472696E67222C20617429006D7300CC
:102130004469676974616C2070696E206576656EAC
:10214000742068616E646C65727320746F6F6B20AD
:10215000006D7300416E616C6F672070696E206561
:1021600076656E742068616E646C65727320746F3E
:102170006F6B20006D73006F6E2E626174746572F8
:10218000792E6C6576656C206576656E7420686165
:102190006E646C657220746F6F6B20006D73006FDE
:1021A0006E2E626174746572792E636861726769FC
:1021B0006E67206576656E742068616E646C65720A
:1021C00020746F6F6B20006D73006F6E2E74656DE1
:1021D0007065726174757265206576656E742068CD
:1021E000616E646C657220746F6F6B20006D73009C
:1021F0006F6E2E6D6573736167652E73636F757493
:10220000206576656E742068616E646C65722074FA
:102210006F6F6B200020727373692000206C7169EE
:1022200020002066726F6D200052656365697665D7
:1022300064206D657373616765206F66200043617C
:102240006E6E6F74207570646174652045455052E0
:102250004F4D207374617274696E6720706173747E
:102260002074686520656E64206F66207468652040
:10227000454550524F4D0043616E6E6F742077722A
:1022800069746520454550524F4D2066726F6D2030
:10229000736B657463682077697468206E6F6E2D48
:1022A0007A65726F206F6666736574004661696C4B
:1022B000656420746F20616C6C6F63617465206D60
:1022C000656D6F727920666F7220706172736564DC
:1022D0002064657363726970746F7200000000009F
:1022E0002C01000058020000B0040000600900004A
:1022F000C012000080250000004B00000096000086
:1023000000E1000000C2010064009001E803480DF4
:1023100000000000000000000000000101000000BB
:1023200000000000000005000400000000000000A4
:1023300000020104646174610000000002010100F8
:1023400000000000000000040106756172740000C6
:102350000000030103693263000000000003010272
:102360007370690000000000FF4E43000000FF563C
:102370005553420013424B504B00FF525354000040
:102380000C53434B00000B4D49534F000A4D4F5324
:102390004900095353000000005258300000015416
:1023A00058300000024432000000034433000000B3
:1023B00004443400000005443500000006443600A3
:1023C0000000074437000000084438000000FF33D5
:1023D00056330000FF474E440000FF564241540070
:1023E0000D52583100000E54583100000F53434C29
:1023F0000000105344410000FF52454600001841C0
:10240000300000001941310000001A413200000084
:102410001B41330000001C41340000001D41350009
:1024200000001E41360000001F41370000004851E7
:1024300020636F6E6E656374696F6E20646F776E74
:102440002C207365636F6E647320636F6E6E6563BB
:102450007465643A200053534C206E65676F74694D
:102460006174696F6E20746F204851206661696CD9
:1024700065642C2072656173736F63696174696E42
:102480006720746F20726574727900485120636F01
:102490006E6E656374696F6E206661696C65642C2D
:1024A0002072656173736F63696174696E6720740C
:1024B0006F20726574727900436F6E6E6563746924
:1024C0006E6720746F20485120617420002C2072A8
:1024D000656173736F63696174696E6720746F20DF
:1024E0007265747279004661696C656420746F204E
:1024F0007265736F6C7665200054696D6520737921
:102500006E63206661696C65642C2072656173730B
:102510006F63696174696E6720746F20726574728D
:102520007900556E7265636F76657261626C6520C5
:102530006572726F7220696E2074686520776966B3
:1025400069206261636B7061636B2C207265626FDE
:102550006F74696E672073636F75742E2E2E2E0054
:102560004572726F723A205363616E206661696CC6
:102570006564004572726F723A20736176696E67A6
:1025800020576966694D6F64756C653A3A696E7378
:1025900074616E63652E627028292D3E636F6E66CE
:1025A000696775726174696F6E2064617461206619
:1025B00061696C65640075736167653A2077696667
:1025C000692E636F6E666967282277696669415074
:1025D0004E616D65222C20227769666941505061F9
:1025E0007373776F72642229004572726F723A209A
:1025F000736176696E6720576966694D6F64756CA3
:10260000653A3A696E7374616E63652E627028294B
:102610002D3E636F6E66696775726174696F6E20B7
:1026200064617461206661696C6564004572726FF3
:10263000723A20736176696E6720576966694D6FDB
:1026400064756C653A3A696E7374616E63652E6287
:102650007028292D3E636F6E6669677572617469B3
:102660006F6E2064617461206661696C6564004509
:1026700072726F723A20496E76616C696420646E82
:102680007320736572766572004572726F723A20BC
:10269000496E76616C696420676174657761790061
:1026A0004572726F723A20496E76616C6964206E71
:1026B00065746D61736B004572726F723A20496E7A
:1026C00076616C696420495020616464726573733B
:1026D0000075736167653A20776966692E73746166
:1026E00074696328226970222C20226E65746D61E2
:1026F000736B222C202267617465776179222C200C
:1027000022646E732229004572726F723A205769F3
:102710002D46692064697265637420636F6D6D6115
:102720006E64206661696C65640075736167653A03
:1027300020776966692E636F6D6D616E6428226310
:102740006F6D6D616E642229004572726F723A205E
:1027500057692D46692070696E6720636F6D6D61E2
:102760006E64206661696C65640075736167653AC3
:1027700020776966692E70696E672822686F7374A6
:102780006E616D652229004572726F723A20576939
:102790002D466920444E53206C6F6F6B757020631B
:1027A0006F6D6D616E64206661696C656400757340
:1027B0006167653A20776966692E646E736C6F6F26
:1027C0006B75702822686F73746E616D65222900C5
:1027D0004572726F723A2057692D4669204E5450E7
:1027E0002074696D65206C6F6F6B757020636F6D01
:1027F0006D616E64206661696C6564004572726F1C
:10280000723A2057692D466920736C6565702063A4
:102810006F6D6D616E64206661696C656400457200
:10282000726F723A2057692D46692077616B657522
:102830007020636F6D6D616E64206661696C6564A4
:102840000075736167653A20776966692E766572EF
:10285000626F736528666C6167290043616E6E6FF5
:1028600074206163636573732077696669206261B0
:10287000636B7061636B005365636F6E6473206399
:10288000757272656E746C7920636F6E6E656374B9
:10289000656420746F2048513A20004E756D626562
:1028A00072206F6620636F6E6E656374696F6E73FE
:1028B00020746F2048512073696E6365206C6173CA
:1028C00074206173736F63696174696F6E3A20007D
:1028D0004E756D626572206F66206173736F6369F8
:1028E0006174696F6E7320746F2041502073696E3C
:1028F000636520626F6F743A200077696669004EE5
:102900006F2073756368206D6F64756C6500656E0C
:10291000760075736167653A20666C6173682E692D
:102920006E697469616C697A6528637350696E2990
:102930000075736167653A20666C6173682E777203
:1029400069746528616464726573732C20227374E2
:1029500072696E67227C696E74656765722900759D
:10296000736167653A20666C6173682E7265616495
:102970002861646472657373290075736167653AD1
:1029800020666C6173682E65726173652E73756263
:10299000736563746F722861646472657373290070
:1029A00075736167653A20666C6173682E65726144
:1029B00073652E736563746F7228616464726573E6
:1029C00073290075736167653A20666C6173682EC0
:1029D00065726173652E62756C6B282900666C6187
:1029E00073682063686970206E6F7420666F756EFF
:1029F00064006E6F7420696E697469616C697A65D0
:102A00006400666C6173680068656C6C6F00757358
:102A10006167653A206D6F74696F6E2E76657262BC
:102A20006F736528666C616729006D6F74696F6EDE
:102A3000004661696C656420746F2073656E642064
:102A40007265736574004661696C656420746F20FB
:102A500073656E642070696E67004661696C6564B9
:102A600020746F2073656E642073657420616464E4
:102A700072657373004661696C656420746F2073BE
:102A8000656C656374206D656D6F7279004E6F20A3
:102A900070696E67207265706C79004641494C0020
:102AA0004F7461206F7065726174696F6E20696E1A
:102AB0002070726F67726573733F0075736167652D
:102AC0003A206F74612E70696E67286164647229A0
:102AD000004641494C005265747279696E67205412
:102AE00058004661696C656420746F2073656E647C
:102AF0002070696E67004641494C004F7461206F39
:102B00007065726174696F6E20696E2070726F6794
:102B1000726573733F0075736167653A206F746106
:102B20002E737461727428616464722C20647279EB
:102B300072756E29004641494C0054696D656F7588
:102B4000742072656164696E6720646174612066D7
:102B5000726F6D2073657269616C2028004641496F
:102B60004C0044617461206D7573742073746172DC
:102B7000742077697468204E554C20627974650022
:102B80004641494C00496E76616C696420686578FD
:102B9000206469676974004641494C004D656D6F5A
:102BA000727920616C6C6F636174696F6E2066610D
:102BB000696C656400556E6576656E206865782081
:102BC000646967697473004641494C004F74612021
:102BD0006F7065726174696F6E20696E2070726FBC
:102BE00067726573733F0075736167653A206F7430
:102BF000612E64617461286D656D616464722C205E
:102C00006865786461746129206F72206F74612E29
:102C100064617461286D656D616464722C207369F0
:102C20007A652920666F6C6C6F7765642062792005
:102C30005C3020616E642073697A652062696E6120
:102C40007279206461746120627974657300464111
:102C5000494C004F7461206F7065726174696F6ECA
:102C600020696E2070726F67726573733F007573B1
:102C70006167653A206F74612E636C6F6E65004604
:102C800041494C004F7461206F7065726174696FC7
:102C90006E20696E2070726F67726573733F007586
:102CA000736167653A206F74612E656E64006F749E
:102CB00061005265747279696E6720626C6F636B34
:102CC000004641494C00437263206D69736D617425
:102CD0006368004F4B004F4B00504F4E472000752C
:102CE000736167653A20706978656C732E616464FE
:102CF00028706978656C73205B2C322C226E656FAE
:102D0000706978656C222C22726762225D290070DE
:102D10006978656C7300736572766F00207061630B
:102D20006B6574732E004275666665722073697AEE
:102D30006520697320006F6E6C792077617920744B
:102D40006F2073746F7020736E696666696E67209A
:102D5000697320746F2072657365742E00736572D9
:102D600069616C2C20776966692C206574632E2953
:102D700020616E6420646F6573206E6F74207275BD
:102D80006E20616E792053636F757453637269703E
:102D9000742E2054686500736E696666696E672CD0
:102DA000207468652073636F757420646F65732089
:102DB0006E6F7420726573706F6E6420746F206123
:102DC0006E797468696E6720656C736520286D651F
:102DD00073682C00536E696666696E67206D657353
:102DE00068207472616666696320616E64206F7525
:102DF00074707574207061636B65747320746F20D8
:102E000073657269616C2E205768696C6500757313
:102E10006167653A20736E69666665722E737461C8
:102E20007274285B62696E6172795D2900736E69E4
:102E3000666665720029002C002C0052756E6E6962
:102E40006E673A206C65644576656E7448616E64A1
:102E50006C65722800537461727475702062616EC3
:102E60006E65722074696D656F75740086878889D8
:102E70008C8D93858B848AA626267C7C3D3D213DC6
:102E80002B2B2D2D3A3D3E3D3E3E3C3D3C3C2F2FD5
:102E900000A199A2949B8F9C9A9D979F9596989E2E
:102EA00090344444444004404444444444444444EE
:102EB0004408774785777878781111111111878840
:102EC000844222222222222222222222222224443C
:102ED00072422222222222222222222222222787F8
:102EE0007465787065637465642000756E657870CC
:102EF000656374656420006D697373696E67200093
:102F0000737472696E670020756E646572666C6FAB
:102F10007700206F766572666C6F77005E43005EA7
:102F200042005E5500657870006F70003A786279F3
:102F30002B2D2A2F00656F6600766172006E756D0D
:102F40006265720029007361766564006565707260
:102F50006F6D003A3D22003E20006368617200738D
:102F60007461636B007374617274757000696400DE
:102F700070726F6D7074000D0A46756E6374696FC0
:102F80006E733A006F6F7073006172670066756EE2
:102F90006374696F6E000062616E6E6572007072BC
:102FA000696E7420226269746C617368206865724E
:102FB00065212076322E30202863292032303133AB
:102FC0002042696C6C20526F79202D7479706520D5
:102FD00048454C502D222C667265652C226279740E
:102FE0006573206672656522000000006DDD0BDEF2
:102FF0001CDE8CDEA4DE4DDCEEDECBDE0ADFE0DDA7
:103000007ADE2FDE40DEF8E556E39BD64FE972E923
:1030100049DD40DFC1DD1D03A2DD59DD53DEAAE23B
:1030200066DEDBDC83DD15E3687474703A2F2F6293
:1030300069746C6173682E6E65740D0A5365652042
:103040004C4943454E534520666F72206C69636559
:103050006E73650D0A50696E733A2064302D3232FA
:103060002C61302D323220205661726961626C65AC
:10307000733A20612D7A2C20333220626974206CDF
:103080006F6E6720696E7465676572730D0A4F70A5
:10309000657261746F72733A202B202D202A202FC5
:1030A00020282029203C203C3D203E203E3D203D44
:1030B0003D20213D203C3C203E3E2021205E20261C
:1030C000207C202B2B202D2D203A3D0D0A436F6DA7
:1030D0006D616E64733A20000061726700626F6F09
:1030E0007400656C73650066756E6374696F6E005D
:1030F00068656C70006966006C73007065657000CF
:103100007072696E740070730072657475726E000F
:10311000726D0072756E0073746F700073776974EE
:103120006368007768696C650000616273006172B2
:1031300000617700626175640062630062656570BA
:1031400000627200627300627700636F6E73747264
:1031500061696E0064656C61790064720064770077
:1031600065720065770066726565006765746B65FA
:1031700079006765746E756D00696E6200697373BE
:103180007472006D6178006D696C6C6973006D69B3
:103190006E006F7574620070696E6D6F64650070AB
:1031A00072696E74660070756C7365696E00726129
:1031B0006E646F6D007369676E00736E6F6F7A6512
:1031C0000000000001090A0B0000000000000000E0
:1031D00000000000000000070304000000000000E1
:1031E00000000102800810200440200104080204AD
:1031F00008010210804080102040010204081020C5
:1032000040800505020505050505040202020204C9
:103210000404040405040402020206060606060667
:103220000606000000002300000029002C002F00EB
:10323000320000000000000000000000000000005C
:10324000250000002B002E0031003400000000009B
:1032500000000000000000000000240000002A0020
:103260002D003000330000000000000000000000CE
:103270004E414E494E495459494E46CDCCCC3D0A5B
:10328000D7233C17B7D13877CC2B329595E6241F3E
:10329000B14F0A000020410000C84200401C4620F7
:1032A000BCBE4CCA1B0E5AAEC59D7400061A1D1B2F
:1032B000392AAA366274648112844989EE8F4F904C
:1032C0002F921097C19CF99C28A22DAB36B265B302
:1032D00097B6C2B659BE18C194C185D2FDD57AD66B
:1032E00085D690D60D040F02C304472ADC369D74A0
:1032F000559011241FBECFEFD1E8DEBFCDBF00E057
:103300000CBF1AE2A0E0B2E0E0EFF8E402E00BBF8D
:1033100002C007900D92A23BB107D9F727E4A2EBB8
:10332000BAE201C01D92A23CB207E1F712E3CAEE75
:10333000D2E300E006C022970109FE010BBF0F9403
:10334000CC18CC3AD10780E00807A9F70F94E50A1A
:103350000D9466240C940000CF92DF92EF92FF92BE
:103360000F931F93E82FF92F05C001501109210970
:10337000310961F1908196239417B9F305C001508A
:1033800011092109310911F1908196239413F7CF86
:10339000C12CD12CE12CF12C0AC08FEFC81AD80A0D
:1033A000E80AF80A0C151D052E053F0579F0808105
:1033B0008623841791F36C2D7D2D8E2D9F2D1F91CB
:1033C0000F91FF90EF90DF90CF90089560E070E054
:1033D00080E090E01F910F91FF90EF90DF90CF90F1
:1033E00008950F931F9309EA16EE2CE038E741E6A3
:1033F0005CE067E77CE08DE79BE20E942B291F9150
:103400000F9108958DE79BE20C9439270F9300E00C
:1034100020E040E060E082EB9AE20F94C30A0F9153
:103420000895CF93CFB7F8948091BB2A811127C01C
:10343000EBE0F2E38491EBEEF1E39491E82FF0E01E
:10344000EE0FFF1FEA5AFD4CA591B4918C91892390
:1034500021F461E089E00F94420761E089E00F9474
:1034600009078CB580618CBD8CB580648CBD61E032
:103470008CE00F94090761E08AE00F9409078091BE
:10348000BB2A8F5F8093BB2ACFBFCF9108958091D5
:10349000ED2A90E02091EE2A821B91090895209157
:1034A000EE2A8091ED2A281750F4E22FF0E0E15146
:1034B000F54D808190E02F5F2093EE2A08958FEFE5
:1034C0009FEF0895E091EE2A8091ED2AE81730F4FD
:1034D000F0E0E151F54D808190E008958FEF9FEF8E
:1034E00008950895CF92DF92EF92FF920F931F936A
:1034F000CF93DF937C01CB018A012091C92A22233B
:1035000089F0EB016B01C40ED51ECC15DD0569F009
:103510006991D701ED91FC910190F081E02DC701F7
:103520001995F3CF642F0E94D61BC801DF91CF916C
:103530001F910F91FF90EF90DF90CF900895CF9360
:10354000DF931F92CDB7DEB769832091C92A22236A
:10355000D1F02091CA2A203240F021E030E0FC0175
:103560003383228380E090E015C08091CB2AE82F3E
:10357000F0E0E453F54D998190838F5F8093CB2ADF
:103580008093CA2A05C061E0CE0101960E94D61B35
:1035900081E090E00F90DF91CF910895FC011382BC
:1035A000128248EE53E060E070E044835583668306
:1035B000778385E89CE09183808308951092EE2ABA
:1035C0001092ED2A1092CB2A1092CA2A0C94211B39
:1035D000862F413208F040E26FEE7AE20E943F1BF4
:1035E0001092EE2A8093ED2A089521E00C94E81AB7
:1035F00021E00C94E81A81E08093C92A6093EC2AB8
:103600001092CB2A1092CA2A08950C94FB1A0F9399
:10361000062F21E04091CA2A6CEC7AE28091EC2AD4
:103620000E94831B1092CB2A1092CA2A1092C92A98
:103630000F91089561E00C94071B8DEB9AE20C94B6
:10364000CE1A10927C2B81E080937A2B1092792BEA
:1036500061E080E10F94420761E08FE00F94420740
:10366000E9EBF0E080818E7F808380818D7F808395
:1036700088E48093B80085E48093BC0008954132CB
:1036800008F03FC090917C2B9111FCCF91E090937A
:103690007C2B20937A2B2FEF20930F2B1092542BFF
:1036A000240F2093532B90937B2B90917B2B880F8F
:1036B000892B80937B2B8091792B813041F4109260
:1036C000792B80917B2B8093BB0085EC01C085EE2C
:1036D0008093BC0080917C2B8130E1F38091542B4E
:1036E000841710F44091542B25E53BE2FB01D901EE
:1036F0008A2F821B841718F48D918193F9CF842F20
:10370000089580E008950F93413208F046C09091EB
:103710007C2B9111FCCF92E090937C2B00937A2B21
:103720009FEF90930F2B1092542B4093532BFB0140
:1037300065E57BE2DB019A2F961B941718F49191B3
:103740009D93F9CF10927B2B90917B2B880F892B27
:1037500080937B2B8091792B813041F41092792BCF
:1037600080917B2B8093BB0085EC01C085EE80931C
:10377000BC00222321F080917C2B8230E1F38091E8
:103780000F2B8F3F61F080910F2B803251F0809191
:103790000F2B803341F483E007C081E005C080E057
:1037A00003C082E001C084E00F910895613298F473
:1037B00020917C2B243089F46093312BFC0183E32E
:1037C0009BE2DC012A2F281B261718F421912D9348
:1037D000F9CF80E0089581E0089582E0089585EDB5
:1037E0008093BC008091BC0084FDFCCF10927C2BA8
:1037F000089585EC8093BC0010927C2B08951F9255
:103800000F920FB60F9211240BB60F922F933F9386
:103810004F935F936F937F938F939F93AF93BF93D8
:10382000EF93FF938091B900887F803609F49CC0A4
:1038300068F5883209F45BC090F4803109F454C013
:1038400038F4882309F4F5C0883009F44DC0F5C078
:10385000883109F44CC0803209F45DC0EEC0803478
:1038600009F468C048F4803309F455C0883309F07E
:10387000E4C080930F2BA8C0803509F44FC0883571
:1038800009F45DC0883409F0D8C0D5C0883909F47E
:10389000C6C0A8F4883709F467C038F4883609F43C
:1038A00063C0803709F460C0C8C0883809F4B7C065
:1038B000803909F45FC0803809F0BFC05BC0803B2D
:1038C00009F485C038F4803A09F466C0883A09F4EE
:1038D0007EC0B3C0803C09F4A6C0883C09F4A3C0F4
:1038E000883B09F489C0A9C080917B2B10C09091BE
:1038F000542B8091532B981770F5E091542B81E055
:103900008E0F8093542BF0E0EB5AF44D808180931E
:10391000BB0085EC85C080930F2B8DC0E091542BAC
:1039200081E08E0F8093542B8091BB00F0E0EB5A26
:10393000F44D80839091542B8091532B6DC0E09176
:10394000542B81E08E0F8093542B8091BB00F0E0CC
:10395000EB5AF44D808380917A2B81116CC081E009
:103960008093792B84EA60C083E080937C2B109253
:10397000102BCFCF8091102B803208F050C0E091F7
:10398000102B81E08E0F8093102B8091BB00F0E014
:10399000EF5EF44D8083BDCF8091102B803230F4E8
:1039A000E091102BF0E0EF5EF44D10820E94EF1BCF
:1039B0006091102B70E0E091752BF091762B81E1F6
:1039C0009BE219951092102B0E94F91B36C084E0DF
:1039D00080937C2B1092322B1092312BE091772B1D
:1039E000F091782B19958091312B811105C081E0E0
:1039F0008093312B1092332BE091322B81E08E0F8C
:103A00008093322BF0E0ED5CF44D80818093BB001D
:103A10009091322B8091312B981708F47ACF85E85A
:103A20008093BC000AC085EC8093BC0010927C2B74
:103A300004C010920F2B0E94EF1BFF91EF91BF91DA
:103A4000AF919F918F917F916F915F914F913F9136
:103A50002F910F900BBE0F900FBE0F901F901895D7
:103A60002EB3FC012183089508950D940B00DC0111
:103A70001196EC91E150E03140F4F0E0EE0FFF1FC1
:103A8000E754F34F80819181089589E49AE0089585
:103A9000CF93DF93EC018881811105C00E9416B895
:103AA0009985980F01C091E8892FDF91CF910895F2
:103AB000FC01818508951F93CF93DF93EC01162FAE
:103AC0008CEB9FE10F94E9211987DF91CF911F9132
:103AD00008950F931F93CF93DF938B01C2ECDFE127
:103AE000F80161918F01CE010F94E9212196C23E28
:103AF000FFE1DF07A9F7DF91CF911F910F910895A3
:103B00000F931F93CF93DF938B01C2ECDFE1CE01C4
:103B10000F94D521F80181938F012196C23EFFE1D8
:103B2000DF07A9F7DF91CF911F910F910895CF93F0
:103B3000DF93C2ECDFE16FEFCE010F94E921219614
:103B4000C23E8FE1D807B9F7DF91CF91089560E0C9
:103B50008DEB9FE10D94E92188EF9FE10D94DD212C
:103B60008CEF9FE10D94E3218EEF9FE10D94D52121
:103B70008FEF9FE10D94D5210F931F93CF93DF9388
:103B80001F92CDB7DEB78C01862F69830E9489FE14
:103B90006981F801668383EF9FE10F90DF91CF91F8
:103BA0001F910F910D94E9210F931F93CF93DF93F2
:103BB0001F92CDB7DEB78C01862F69830E94B1FEBC
:103BC0006981F801678382EF9FE10F90DF91CF91C8
:103BD0001F910F910D94E921362F3370ECE4F1E041
:103BE00020812C7F232B2083FC0160878EEB9FE1BB
:103BF0000D94E921CF92DF92EF92FF920F931F93E2
:103C0000CF93DF931F92CDB7DEB76C017B018A01A2
:103C1000CB0129830E94D1F1F601F382E282C8012F
:103C20000E94D7F1F601158304832981622FC60112
:103C30000E94BC1D81E00E9485FEF60162817381B5
:103C400086EF9FE10F94FB21F6016481758184EF7B
:103C50009FE10F94FB2182EF9FE10F94D5218F3FCD
:103C600011F0682F01C060E0C6010E94D41D8EEBE8
:103C70009FE10F94D5218F3F11F0682F01C060E0C4
:103C8000C6010F90DF91CF911F910F91FF90EF90A0
:103C9000DF90CF900C94EC1DEF92FF920F931F9347
:103CA000CF93DF931F921F92CDB7DEB7CB0169830D
:103CB0007A830E94F6FA6981E62E7A81F72E02EE67
:103CC0001FE1F70161917F01C8010F94E9210F5FA6
:103CD0001F4F023FFFE11F07A1F70F900F90DF91E9
:103CE000CF911F910F91FF90EF900895AF92BF92E7
:103CF000CF92DF92EF92FF920F931F93CF93DF93B8
:103D0000CDB7DEB7A1970FB6F894DEBF0FBECDBF1B
:103D10007C018E010F5F1F4F580122ECC22E2FE154
:103D2000D22EC6010F94D521F50181935F01FFEFDB
:103D3000CF1ADF0A22EEC2162FE1D20691F7B801A0
:103D4000C7010E94691D80E2F80111928A95E9F786
:103D5000580192EEC92E9FE1D92EC6010F94D521AC
:103D6000F50181935F01FFEFCF1ADF0A22EFC21640
:103D70002FE1D20691F7B801C7010E944C1E80E1E5
:103D8000F80111928A95E9F786EF9FE10F94E321FC
:103D90008C018F3FFFEF9F0761F484EF9FE10F9449
:103DA000E321019631F483EF9FE10F94D5218F3FFA
:103DB00081F083EF9FE10F94D521282F84EF9FE1BD
:103DC00029A30F94E321AC0129A1B801C7010E94E6
:103DD000FA1D82EF9FE10F94D5218F3F21F0682FCC
:103DE000C7010E94D41D8EEB9FE10F94D5218F3F18
:103DF00021F0682FC7010E94EC1D8CEB9FE10F940E
:103E0000D5218F3F11F0F7018187A1960FB6F89465
:103E1000DEBF0FBECDBFDF91CF911F910F91FF90FD
:103E2000EF90DF90CF90BF90AF9008950F931F93C6
:103E3000CF93DF93EC017B876A875D874C870E8782
:103E40001F87288B398B0F9405000E9407FF61E0C4
:103E500089E00F94420761E089E00F94090726E0AA
:103E600040E052EC61E070E083E496E40F94C30814
:103E7000CE01DF91CF911F910F910C94761E0F937D
:103E80001F93CF93DF938B01C2EEDFE1CE010F943E
:103E9000D521F80181938F012196C23FFFE1DF0711
:103EA000A9F7DF91CF911F910F910895CF93DF93E1
:103EB000CDB7DEB760970FB6F894DEBF0FBECDBFAB
:103EC00020E1E1E5FCE0DE01119601900D922A95DA
:103ED000E1F7BE016F5F7F4F0E944C1E60960FB6E8
:103EE000F894DEBF0FBECDBFDF91CF910895862F2E
:103EF000BA010C94DDF1CF93DF93EB01CB010E946B
:103F0000B7F3811105C0CE01DF91CF910C9483F3FB
:103F1000DF91CF910895CF93DF93EB01CB010E9406
:103F2000B7F3882329F0CE01DF91CF910C949CF355
:103F3000DF91CF910895CB010C94B7F3FC018281FE
:103F400093810895FC01848195810895FC01868107
:103F50000895FC01828593850895FC0184859585EB
:103F60000895FC0166857785808991890895DC0133
:103F70001796EC91E03140F4F0E0EE0FFF1FE756AA
:103F8000F34F80819181089586EB99E00895DC01DB
:103F90001896EC91E43040F4F0E0EE0FFF1FEF567E
:103FA000F34F8081918108958EE899E00895A09162
:103FB0005C2CB0915D2C109749F0ED91FC9111971C
:103FC0000190F081E02D682FCD01199408958F9212
:103FD0009F92AF92BF92CF92DF92EF92FF920F9398
:103FE0001F93CF93DF9300D000D0CDB7DEB78C0105
:103FF0004B015A01FC018181882369F067E17BE074
:1040000083E496E40F94360BF5016081718183E4BB
:1040100096E40F949A0B8114910429F090925D2CF0
:1040200080925C2C08C0F8018281882341F01092B4
:104030005D2C10925C2C87ED9FE10E94C2D8F501A7
:10404000808191810E94EEF06B017C01892819F436
:10405000F801828181110E94C7D869ED7CE0CE0110
:1040600001960F94480DBE016F5F7F4FC5010F94FD
:104070007D10B82ECE0101960F94DA0CBB2019F0FA
:10408000C8010E94C558C701B60126960FB6F8941C
:10409000DEBF0FBECDBFDF91CF911F910F91FF907B
:1040A000EF90DF90CF90BF90AF909F908F9008954A
:1040B000CF93DF93EC010E94301DFE01EC57FF4FC0
:1040C00011821082CE0188579F4F0E94827DCE01BF
:1040D0008C569F4F0E94572EFE01EE55FF4F1082C7
:1040E00011821282138234961082319610821182CC
:1040F000128213821B8A1A8A1D8A1C8A1F8A1E8AB0
:10410000198E188E1B8E1A8E1D8E1C8E3D9682E384
:1041100090E0A0E0B0E080839183A283B3833496E3
:1041200081E090E09183808332962AE235E2318308
:104130002083389648EE53E060E070E0408351837E
:104140006283738334969183808332962BEF34E2BB
:1041500031832083389640E65AEE60E070E0408379
:1041600051836283738334969183808332968CE883
:1041700091E291838083E055F1091082B796108215
:10418000BB961082C352DF4F19821882DF91CF9104
:104190000895CF93DF93EC018C569F4F0E945E2EC3
:1041A000CE01DF91CF910C94341D84E10F947807F8
:1041B00021E0892B09F020E0822F08950E94F5BAB2
:1041C00097FD0AC00E94F5BA8536910514F40C9447
:1041D000F5BA84E690E0089580E090E008950C94AC
:1041E000D8BA82E10F94780721E0892B09F020E00A
:1041F000822F08950F931F93CF93DF9384E10F9441
:10420000780701E0892B09F400E0C8E2D0E010E073
:1042100084E10F94780721E0892B09F420E0201332
:1042200003C0112311F00BC011E061E070E080E0E9
:1042300090E00F943505219759F781E001C080E0A7
:10424000DF91CF911F910F9108950C94481DCF934A
:10425000DF93EC010E94481D682F772767FD70955A
:10426000872F972F0F94451426E636E646EE5FE338
:104270000F94A31520E030E040E052E40F943E1389
:1042800020E030E0A9010F949F1587FD1EC0CE01EC
:104290000E94481D682F772767FD7095872F972FFD
:1042A0000F94451426E636E646EE5FE30F94A31519
:1042B00020E030E040E052E40F943E1320E030E094
:1042C00040E05FE30F943E131DC0CE010E94481DE5
:1042D000682F772767FD7095872F972F0F944514C8
:1042E00026E636E646EE5FE30F94A31520E030E0C5
:1042F00040E052E40F943E1320E030E040E05FE302
:104300000F943D130F940E140F9445140F9413142F
:10431000862FDF91CF9108950F931F93CF93DF9353
:104320008091932B9091942B892B59F18DE79BE2EF
:104330000E94DE20182FEC012091FB2B30E02C177F
:104340003D07F9F08091032C882399F065EA7BE022
:1043500083E496E40F94360B4AE050E0BE0183E418
:1043600096E40F94AC0C63EA7BE083E496E40F944C
:10437000760B1093FB2BE091932BF091942B812FD4
:1043800019958091952B9091962B892B61F18DE752
:104390009BE20E94D520182FC82FD0E02091FE2B41
:1043A00030E02C173D07F9F08091032C882399F019
:1043B0006DE77BE083E496E40F94360B4AE050E02F
:1043C000BE0183E496E40F94AC0C6BE77BE083E4DE
:1043D00096E40F94760B1093FE2BE091952BF091C1
:1043E000962B812F19958091972B9091982B892B43
:1043F00071F182E10F94780711E0892B09F010E048
:10440000C12FD0E02091FF2B30E02C173D07F9F0B1
:104410008091032C882399F06FE47BE083E496E499
:104420000F94360B4AE050E0BE0183E496E40F940B
:10443000AC0C6DE47BE083E496E40F94760B109370
:10444000FF2BE091972BF091982B812F199580915C
:10445000992B90919A2B892B09F448C08DE79BE208
:104460000E94481D182FC82FDD27C7FDD095209129
:10447000002C30E02C173D07C9F18093002C8DE70C
:104480009BE20E942721082F8091032C882319F199
:104490006BE27BE083E496E40F94360B4AE050E055
:1044A000BE0183E496E40F944F0C63E071E183E472
:1044B00096E40F94690B4AE050E0602F772767FD80
:1044C000709583E496E40F944F0C69E27BE083E4FB
:1044D00096E40F94760BE091992BF0919A2B602F34
:1044E000812FDF91CF911F910F911994DF91CF917F
:1044F0001F910F91089585559F4FFC01808108956C
:1045000087569F4FFC018081811104C081E090E0BB
:104510000C94798381E00895FC01E355FF4F80817D
:10452000811102C091E090830895F89428E088E119
:1045300090E00FB6F894A895809360000FBE20938A
:104540006000FFCF82559F4F0D94BE0082559F4F54
:104550000D94760084549F4F0D94BE0084549F4F59
:104560000D94760086539F4F0D94BE0086539F4F47
:104570000D9476006F927F928F929F92AF92BF922E
:10458000CF92DF92EF92FF920F931F93CF93DF931F
:1045900000D01F92CDB7DEB73C01480159018C0114
:1045A00002551F4FC80149835A836B837C830F9444
:1045B0007600F301EC54FF4F49815A816B817C8175
:1045C0004083518362837383C8010F94BE00025FEE
:1045D0001F4FC8010F947600F301EE53FF4F808206
:1045E0009182A282B382C8010F94BE0053018AEC6B
:1045F000A80EB11CC5010F947600F301E053FF4FE4
:10460000C082D182E282F382C5010F900F900F9099
:104610000F90DF91CF911F910F91FF90EF90DF905E
:10462000CF90BF90AF909F908F907F906F900D94A0
:10463000BE00603238F4860F911DFC01E25AFF4F34
:10464000808108958DEF08958EEF860F843048F0B5
:104650008BEE860F823028F081E0673119F080E020
:10466000089581E00895603248F4860F911DFC01A1
:10467000E25AFF4F90819D7F81E009F080E008952C
:10468000603250F4860F911DFC01E25AFF4F908179
:104690009D7F81E0913009F080E008959C01862F94
:1046A000603218F5E62FF0E0D901AE0FBF1FA25A15
:1046B000BF4F9C919130B9F01CF4992369F015C05B
:1046C000923051F0933089F43F96EE0FFF1FE20FC6
:1046D000F31F80819181089598EE980F993018F416
:1046E000892F0D94CA050D94780780E090E0089515
:1046F000FF920F931F93CF93DF938B01CDECDBE001
:10470000F12CBE01C8010F94AF1D892B11F48F2D20
:1047100006C0F394259680E2F812F3CF8FEFDF9175
:10472000CF911F910F91FF900895603238F425E0EA
:10473000629FC00111248353944F089580E090E05C
:1047400008956C5F683048F4E62FF0E0EE0FFF1F2D
:10475000ED5FF24F80819181089580E090E00895AF
:10476000262F4091772D5091782D6091792D709161
:104770007A2D2F3F69F081E090E0A0E0B0E0022EBA
:1047800004C0880F991FAA1FBB1F0A94D2F703C049
:1047900080E090E0DC0184239523A623B723892BB6
:1047A0008A2B8B2B39F4223028F02F50293010F02F
:1047B00080E0089581E008959F92AF92BF92CF92DA
:1047C000DF92EF92FF920F931F93CF93DF93EC0151
:1047D0007C018C01B12C9DEFA92E2EEF922ECC24C2
:1047E000CA94DC2C6B2DCE010E94B023F801E25A52
:1047F000FF4F882311F0908201C0A082F701D78E6D
:10480000C68EB394F2E0EF0EF11C0F5F1F4F80E2F3
:10481000B812E8CFCE010E94DE20FE01E258FF4F21
:1048200080830E94D8BAFE01E158FF4F91838083B4
:10483000CE010E94D520FE01EF57FF4F8083CE01AD
:104840000E94F120FE01EE57FF4F8083CE010E94AF
:10485000481DCD57DF4F8883DF91CF911F910F9176
:10486000FF90EF90DF90CF90BF90AF909F90089512
:10487000CF92DF92EF92FF920F931F93CF93DF932C
:10488000EC01C62E8A01D22EE62EF12CF701EE0F96
:10489000FF1FE80FF91F868D978D9E012E0D3F1D7E
:1048A0008017910741F4C901825A9F4FDC018C9116
:1048B0008D1509F456C0178F068FD901A25ABF4F24
:1048C000DC928EEF8C0D873008F040C08A899B897E
:1048D000892BE1F1FE01EA57FF4F8081882381F1A6
:1048E00063EB7AE083E496E40F94360B4AE050E001
:1048F0006C2D83E496E40F948E0C61EB7AE083E4F4
:1049000096E40F94360B4AE050E0B80183E496E455
:104910000F944F0C6FEA7AE083E496E40F94360B21
:104920004AE050E06D2D772767FD709583E496E4AB
:104930000F944F0C6DEA7AE083E496E40F94760BC3
:10494000EA89FB894D2DB8018C2D1995B8EECB0E57
:1049500088E08C1508F445C02C893D89232B19F477
:1049600040C080E03FC0FE01EA57FF4F80818823AE
:1049700091F16DE87AE083E496E40F94360BB70189
:10498000685171094AE050E083E496E40F944F0CBB
:104990006BE87AE083E496E40F94360B4AE050E04B
:1049A000B80183E496E40F944F0C69E87AE083E45D
:1049B00096E40F94360B4AE050E06D2D772767FDA3
:1049C000709583E496E40F944F0C67E87AE083E4F3
:1049D00096E40F94760BEC89FD894D2DB8018C2D52
:1049E000199581E0DF91CF911F910F91FF90EF908A
:1049F000DF90CF900895EF92FF921F93CF93DF93B4
:104A00001F92CDB7DEB78091912B9091922B892B7D
:104A1000D1F053EFE52E5BE2F52E18E1F70121917D
:104A20007F0127FD0DC0612F8DE79BE229830E9446
:104A30004E232981AC01612F8DE79BE20E9438242F
:104A40001F5F103259F70F90DF91CF911F91FF90A8
:104A5000EF900895EF92FF921F93CF93DF931F92F1
:104A6000CDB7DEB780918F2B9091902B892BD1F011
:104A70006DEDE62E6BE2F62E12E0F70121917F013B
:104A800027FD0DC0612F8DE79BE229830E944E23F5
:104A90002981AC01612F8DE79BE20E9438241F5FC2
:104AA000193059F70F90DF91CF911F91FF90EF9040
:104AB0000895CF92DF92FF920F931F93CF93DF93CE
:104AC0001F92CDB7DEB76C01F62E49830E94B0234A
:104AD0002981811133C012162CF02F3F4CF42C3F4A
:104AE00049F02CC0223031F03CF0233029F026C0B0
:104AF00060E003C062E001C061E08F2D29830F9464
:104B00000907298123303CF427FF0AC02F3F79F49D
:104B10000FEF1FEF0CC0233051F400E010E007C08E
:104B20006F2DC60129830E944E238C012981A80183
:104B30006F2DC6010E94382481E001C080E00F90F3
:104B4000DF91CF911F910F91FF90DF90CF9008954B
:104B50000F931F93CF93DF938C01C0E0D0E0F80157
:104B6000EC0FFD1FE25AFF4F80818D3F29F44CEF7F
:104B70006C2FC8010E9459252196C032D10579F7C2
:104B8000DF91CF911F910F910895DF92EF92FF92E5
:104B90000F931F93CF93DF93EC01F62ED42E0E9438
:104BA000B023811108C06F2DCE010E944023E82E52
:104BB000811103C028C0E12C26C00D2D10E08FE12B
:104BC0008F1568F0FE01EF0DF11DE25AFF4F808155
:104BD000833029F4B8018F2D0F94EF0507C06D2D98
:104BE0008F2D0F9442078FE18F1538F0FE01EF0DE6
:104BF000F11DE25AFF4F208101C02DEFA8016F2D5A
:104C0000CE010E9438248E2DDF91CF911F910F91FC
:104C1000FF90EF90DF900895AF92BF92CF92DF9216
:104C2000EF92FF920F931F93CF93DF93EC016A01F2
:104C30007B0159018C0108521F4F41155105610537
:104C4000710541F0CB01BA010E94A87681E0F8011C
:104C5000808302C0F80110828E0103521F4FF801B9
:104C600080819181009711F00F94C719A114B104AC
:104C700021F0C5010F94091E02C080E090E0F80108
:104C800091838083C752DF4FC882D982EA82FB8238
:104C9000DF91CF911F910F91FF90EF90DF90CF9018
:104CA000BF90AF9008952F923F924F925F926F9274
:104CB0007F928F929F92AF92BF92CF92DF92EF92AC
:104CC000FF920F931F93CF93DF93CDB7DEB7629719
:104CD0000FB6F894DEBF0FBECDBF5C011C018DED99
:104CE000280E311CF101E080F180118210826501F3
:104CF000F8EDCF0ED11CF6011082611107C00E94A1
:104D0000EFF181E00E9400770E94F1F1E114F104DB
:104D100009F496C040E150E060E470E08E010F5F5E
:104D20001F4FC8010E9400BF0E94DD76E8EE4E2EA4
:104D3000E3E05E2E612C712CA30192010F94811788
:104D40002F87388B498B5A8BF4E0660F771F881FAB
:104D5000991FFA95D1F7A30192010F9481172901A8
:104D60003A018F859889A989BA8924E0880F991F0B
:104D7000AA1FBB1F2A95D1F7480E591E6A1E7B1E1B
:104D8000B701C8010F94460F61EE74E2C8010F9499
:104D9000460FF501E752FF4F83818F9382818F93F6
:104DA00081818F9380818F9384EE9CE09F938F937A
:104DB0001F930F930E9426BF7F926F925F924F9234
:104DC00083EE9CE09F938F931F930F930E9426BFC7
:104DD00069EE71E1C8010F94460F69817A81CE01B5
:104DE00009960F94480DAE01475F5F4F60E070E099
:104DF0008EE49DE20E94E71F4B015C01CE01099603
:104E00000F94DA0C0FB6F894DEBF0FBECDBF452865
:104E10004628472841F089288A288B2821F0F60166
:104E20008081882321F0C7010F94C71906C081E053
:104E3000F6018083F101F182E082C8010F94DA0C5F
:104E400062960FB6F894DEBF0FBECDBFDF91CF9153
:104E50001F910F91FF90EF90DF90CF90BF90AF9098
:104E60009F908F907F906F905F904F903F902F908A
:104E700008952F923F924F925F926F927F928F92FE
:104E80009F92AF92BF92CF92DF92EF92FF920F93D9
:104E90001F93CF93DF93CDB7DEB729970FB6F89462
:104EA000DEBF0FBECDBF998788878091DF00877FE7
:104EB0008093DF004090692D50906A2D60906B2D9B
:104EC00070906C2D80916D2D90916E2DA0916F2D15
:104ED0008D839E83AF838091DF0088608093DF00A5
:104EE0000E94377620E130E040E050E00F94421815
:104EF000190149835A836B837C834C0130E4A32ED0
:104F0000E2E4BE2EFFE0CF2ED12CE12CF12C00E00C
:104F100010E09101C4010F946F1859016A014A0C05
:104F20005B1C6C1C7D1CA0E4AA2EB2E4BB2E1FE00F
:104F3000C12ED12CE12CF12C00E010E0910149812F
:104F40005A816B817C81C4010F946D184901A42E94
:104F50008D819E81AF81880D991DAA1D8034924458
:104F6000AF4028F0FFEF4F1A5F0A6F0A7F0A0885EB
:104F700019850E551F4FF80140825182628273825B
:104F8000888599850E94351DE885F985EA55FF4F8A
:104F900020812223E9F0F80160817181828193816F
:104FA000E884F984F7EAEF0EF11CF7018080918024
:104FB000A280B38086169706A806B90648F430E0AA
:104FC00040E050E00F948117672B682B692B11F09C
:104FD00010E03EC088EE90E30E94F6BB40E0BC01CA
:104FE00088EE90E30E9447BB88EE90E30E94FABBF4
:104FF00040E0BC0188EE90E30E946CBB88EE90E339
:105000000E94FEBB40E0BC0188EE90E30E9491BB91
:105010000E9442F420E030E060E0FC01E20FF31F68
:10502000418152814F3F5F4F09F061E0295F3F4F5F
:105030002C38310591F7662351F0F8018081918178
:10504000A281B381F70180839183A283B38311E0AE
:105050008EE49DE20E94B574888599858C569F4F99
:105060000E9410340E94B3910E94B1811123F1F08B
:1050700088EE90E30E94B6BB41E0BC0188EE90E36D
:105080000E9447BB88EE90E30E94BABB41E0BC019E
:1050900088EE90E30E946CBB88EE90E30E94BEBB5A
:1050A00041E0BC0188EE90E30E9491BBE885F98560
:1050B000E852FF4F8081882351F10E94E6F1182FBA
:1050C0000E94DD76672B682B692B11F461E003C029
:1050D00011111DC060E08885998529960FB6F89456
:1050E000DEBF0FBECDBFDF91CF911F910F91FF901B
:1050F000EF90DF90CF90BF90AF909F908F907F9078
:105100006F905F904F903F902F900C94532629966C
:105110000FB6F894DEBF0FBECDBFDF91CF911F91C8
:105120000F91FF90EF90DF90CF90BF90AF909F9046
:105130008F907F906F905F904F903F902F90089549
:105140000F931F93CF93DF931F92CDB7DEB7DC0190
:105150000D911C910115110559F0D801ED91FC91AB
:10516000862F69831995F801028113816981F2CF35
:105170000F90DF91CF911F910F910895CF93DF93FF
:10518000EC01FC01E555FF4F81E0808361E081E1A6
:105190000F94420761E0CE018C579F4FDF91CF9172
:1051A0000C94A028FC01E555FF4F108260E08C575D
:1051B0009F4F0E94A02860E081E10D9442070F9369
:1051C0001F93CF93DF93CDB7DEB762970FB6F894F6
:1051D000DEBF0FBECDBF8C01CE010D960F94480DE2
:1051E00068EE7CE0CE0101960F94480D69E173E111
:1051F000CE0107960F94480DAE014F5F5F4FBE0181
:10520000695F7F4FCE010D960F94B811CE010796BE
:105210000F94DA0CCE0101960F94DA0C62E2C80109
:105220000F94560FBE01635F7F4FC8010F943F0F6D
:1052300062E2C8010F94560FCE010D960F94DA0C5E
:1052400062960FB6F894DEBF0FBECDBFDF91CF914F
:105250001F910F910895EF92FF920F931F93CF9399
:10526000DF93CDB7DEB72E970FB6F894DEBF0FBE33
:10527000CDBF7C010E94161F0E94737662E084E11C
:105280000F94090762E082E10F94090761E081E170
:105290000F940907C7010E94D22864E670E080E0FD
:1052A00090E00F943505C7010E94BE2888EE90E378
:1052B0000E9499BC8DEB9AE20E94DE1A84E10E9462
:1052C00093BAC7010E94DC230E94B2910E94EA8334
:1052D000C7018C569F4F0E94612EC70182559F4F78
:1052E0000F94BE00C70184549F4F0F94BE00C701A6
:1052F00086539F4F0F94BE0088EE90E30E9450BEED
:105300008EE49DE20E94256D88EE90E30E94B6BB7C
:105310008C0188EE90E30E94F6BB0817190709F08C
:105320009BC088EE90E30E94BABB8C0188EE90E3AC
:105330000E94FABB0817190709F08EC088EE90E3A7
:105340000E94BEBB8C0188EE90E30E94FEBB081752
:10535000190709F081C040E064E670E088EE90E350
:105360000E940BBEF701EE57FF4F8081882309F49E
:1053700073C0F701EF57FF4F808181116DC06BEE55
:105380007CE0CE0109960F94480D41E050E060E8C2
:1053900070E0CE0101960E9400BFBE01675F7F4FA3
:1053A000CE0101960F943F0F68E2CE0101960F9453
:1053B000560F64EF71E0CE0101960F94960F6CE2E8
:1053C000CE0101960F94560F67EF7CE0CE01019657
:1053D0000E94DF286CE2CE0101960F94560F64E61E
:1053E00070E0CE0101960F94960F6CE2CE0101960B
:1053F0000F94560F67EF7CE0CE0101960E94DF28E4
:105400006CE2CE0101960F94560F64E670E0CE0177
:1054100001960F94960F6CE2CE0101960F94560FF1
:1054200067EF7CE0CE0101960E94DF2869E2CE01A1
:1054300001960F94560FAE014F5F5F4F60E070E032
:105440008EE49DE20E94E71FCE0101960F94DA0CD4
:10545000CE0109960F94DA0C2E960FB6F894DEBFA3
:105460000FBECDBFDF91CF911F910F91FF90EF90B5
:1054700008950F9300E020E040E060E08EE59CE2BC
:105480000F94C30A8DE79BE20F910C9458208DE78F
:105490009BE20C94C920FC01848195810F94560FE6
:1054A0000895CF93DF932091EF2C3091F02C6091F1
:1054B000D62C7091D72C621B730B653671051CF4CA
:1054C000EB01219602C0C4E6D0E08091F12C9091CE
:1054D000F22C9093E02C8093DF2C83E08093E12CDE
:1054E00082E08093E22C8093E32C8091D22C9091E7
:1054F000D32C820F931F9093E72C8093E62CC093BC
:10550000E82C81E19BE29093EA2C8093E92C8AEDD0
:105510009CE20E941CF28091112C8823F9F060918A
:10552000F12C7091F22C4AE050E083E496E40F9461
:105530004F0C66E17EE083E496E40F94360B4AE07C
:1055400050E0BE0183E496E40F944F0C6EE07EE0E1
:1055500083E496E4DF91CF910D94760BDF91CF91A8
:105560000895CF93DF9320918B2C30918C2C6091F8
:10557000912C7091922C621B730B653671051CF493
:10558000EB01219602C0C4E6D0E08091952C909169
:10559000962C90937C2C80937B2C82E080937D2CA6
:1055A00093E090937E2C80937F2C80918D2C909112
:1055B0008E2C820F931F9093832C8093822CC09308
:1055C000842C8CE993E39093862C8093852C86E73A
:1055D0009CE20E941CF28091112C8823F9F06091CA
:1055E000952C7091962C4AE050E083E496E40F9459
:1055F0004F0C64EE7CE083E496E40F94360B4AE0B3
:1056000050E0BE0183E496E40F944F0C6CED7CE017
:1056100083E496E4DF91CF910D94760BDF91CF91E7
:105620000895CF93DF93EC018091112C882331F002
:1056300064EF7DE083E496E40F94360B99898091C2
:10564000112C91111FC0882331F06CEE7DE083E4B2
:1056500096E40F94760B2091EF2C3091F02C8091F2
:10566000D62C9091D72C821B930B85369105A0F1F7
:105670002C593F4F3093F02C2093EF2CDF91CF919A
:105680000C94512A2091ED2C3091EE2C2F5F3F4F3E
:105690003093EE2C2093ED2C2430310584F08823B8
:1056A000D9F064EE7DE083E496E40F94360B4AE093
:1056B00050E0698983E496E40F94950C0DC088232B
:1056C00031F06EED7DE083E496E40F94760BCE012D
:1056D000DF91CF910C941CF21092F22C1092F12CCD
:1056E00060E070E082ED9CE2DF91CF910D94D80DE7
:1056F0001F93CF93DF93EC011091162C112369F0C7
:1057000063E17DE08EE49DE20E94F860688179812A
:105710008EE49DE20E94F8604AC0A0919D2DB09158
:105720009E2D109761F01296ED91FC9113970488CD
:10573000F589E02DCD0102961995811112C0809155
:10574000112C882361F066EA7EE083E496E40F94EE
:10575000760BBE0183E496E40F94880B28C010E01A
:1057600026C08091112C882359F066E97EE083E4FD
:1057700096E40F94760BBE0183E496E40F94880BB5
:1057800080919D2D90919E2DBE0102960F945B0BF2
:1057900080919D2D90919E2DDC011296ED91FC91B2
:1057A00013970284F385E02D0296199511E0812F5D
:1057B000DF91CF911F910895DF92EF92FF920F93A7
:1057C0001F93CF93DF93CDB7DEB728970FB6F8942A
:1057D000DEBF0FBECDBF8C0141E050E060E071E064
:1057E000CE0101967C010E9400BFD80116969C91C3
:1057F0008091112C96FF0AC0882309F472C062ECD4
:105800007DE083E496E40F94760B6BC08823A9F0C7
:1058100066EA7DE083E496E40F94360BF80160813C
:1058200071814AE050E083E496E40F94AC0C64EAA2
:105830007DE083E496E40F94760BD80119968C9161
:1058400019971796ED91FC911897E80FF11D319774
:105850009081911106C0815019968C93DD24D394C8
:1058600001C0D12CF80181818F9380818F93809129
:10587000752C8F938091742C8F938BE29DE09F9376
:105880008F93FF92EF920E9426BFD80119964C91F8
:10589000199750E017966D917C91189721E0C701F8
:1058A0000E94DCBF0FB6F894DEBF0FBECDBFDD2077
:1058B00019F080E29DE002C085E29DE09F938F9306
:1058C00086E59DE09F938F93FF92EF920E9426BF03
:1058D000C7010E94782B0F900F900F900F900F90A0
:1058E0000F90C7010F94DA0C81E028960FB6F89458
:1058F000DEBF0FBECDBFDF91CF911F910F91FF9003
:10590000EF90DF90089584E69CE20F94DA0C8CE629
:105910009CE20F94DA0C8DE89CE20F94DA0C82ED95
:105920009CE20F94DA0C83EF9CE20D94DA0CCF9298
:10593000DF92EF92FF920F931F93CF93DF9300D0EC
:1059400000D0CDB7DEB78C018091112C882359F19E
:1059500065E87EE083E496E40F94360B6FE77EE023
:1059600083E496E40F94360B4AE050E0F801628538
:1059700083E496E40F948E0C6CE77EE083E496E477
:105980000F94360B65E77EE083E496E40F94360BC4
:10599000F8016385772767FD70954AE050E083E45E
:1059A00096E40F94570C8091F12C9091F22C892B56
:1059B00061F01091112C112309F4C0C06AE47EE05B
:1059C00083E496E40F94760BB6C0F801418550E06D
:1059D0006781708583EF9CE20E94DBC0882309F415
:1059E000AAC0F8018385992787FD909597FF03C08A
:1059F0009195819591090E946FF86091F72C7091B3
:105A0000F82C6150710983EF9CE20F949A10FC010D
:105A100090818091112C992359F0182F882309F433
:105A20008CC069E37EE083E496E40F94760B86C035
:105A3000882371F068E27EE083E496E40F94360BED
:105A40006091F32C7091F42C83E496E40F949A0BFC
:105A5000F8018385992787FD909597FF03C091955D
:105A6000819591099093522D8093512DF801828553
:105A700090E09093542D8093532D80819181909349
:105A8000562D8093552D67EA79E182ED9CE20F94C3
:105A9000D80D1C821B828DEA9EE09A83898382ED59
:105AA0009CE29E838D8343EF5CE2BE016F5F7F4F7C
:105AB0008EE49DE20E94E71F6B017C0160E070E0D4
:105AC00083EF9CE20F94D80D8091112C8823B1F0C4
:105AD0006CE17EE083E496E40F94360B2AE030E03C
:105AE000B701A60183E496E40F946F0C6091D22C69
:105AF0007091D32C83E496E40F949A0BF80184817F
:105B0000823039F460E070E082ED9CE20F94D80DB1
:105B100014C0F801808191819093F22C8093F12C34
:105B20001092F02C1092EF2C1092EE2C1092ED2C83
:105B30000E94512A02C010E001C011E0812F269678
:105B40000FB6F894DEBF0FBECDBFDF91CF911F918E
:105B50000F91FF90EF90DF90CF9008952F923F929A
:105B60004F925F926F927F928F929F92AF92BF926D
:105B7000CF92DF92EF92FF920F931F93CF93DF9319
:105B8000CDB7DEB72E970FB6F894DEBF0FBECDBFF0
:105B90008091DF00877F8093DF004090692D5090D7
:105BA0006A2D60906B2D70906C2D80916D2D909171
:105BB0006E2DA0916F2D8C879D87AE878091DF0021
:105BC00088608093DF000E94377620E130E040E07B
:105BD00050E00F9442181901488759876A877B87DC
:105BE0004C0180E4A82E92E4B92E2FE0C22ED12CD5
:105BF000E12CF12C00E010E09101C4010F946F182A
:105C000059016A014A0C5B1C6C1C7D1C30E4A32EFC
:105C100042E4B42E5FE0C52ED12CE12CF12C00E043
:105C200010E09101488559856A857B85C4010F94F0
:105C30006D1849015A018C859D85AE85880D991D89
:105C4000AA1D803422E492072FE0A20740F080547E
:105C50009244AF402FEF421A520A620A720A4982F6
:105C60005A826B827C828D839E83AF83242D3A81FE
:105C70004B815C81682F7E818F8190E02E960FB6DC
:105C8000F894DEBF0FBECDBFDF91CF911F910F9172
:105C9000FF90EF90DF90CF90BF90AF909F908F904C
:105CA0007F906F905F904F903F902F90089541E0CC
:105CB00050E060E070E006960C9400BF06960D94EC
:105CC000DA0CCF93DF93DC0115961C928DE79BE2F3
:105CD0000E948022882399F04CED5BE263E08DE71F
:105CE0009BE20E94771F6FEE7EEB8DE79BE20E94A6
:105CF0007B1F60E070E08DE79BE20E947B1FC1E0AC
:105D0000D0E0BE018DE79BE20E947B1F2196CA3046
:105D1000D105B9F747E95CE262E08DE79BE20E94BA
:105D2000771F49E751E364E08DE79BE20E94771F0C
:105D300084E1EEEBFCE2DF011D928A95E9F7DF9149
:105D4000CF910895FC01608308958091BE2C9091BD
:105D5000BF2C892BA9F16091AA2C7091AB2C8DE7F7
:105D60009BE20E947B1F8091AA2C9091AB2C909378
:105D70009D2C80939C2C84E080939E2C8DE79BE24D
:105D80000E949E1F80939F2C82E18093A02CE09123
:105D9000BE2CF091BF2CF093A42CE093A32CDF0138
:105DA0000D900020E9F7AE1BA093A52C81EE9EE29A
:105DB0009093A72C8093A62C87E99CE20C941CF26C
:105DC0000895CF93DF93EC018989882389F080912E
:105DD000112C882369F06FE77CE083E496E40F944C
:105DE000360B4AE050E0698983E496E40F94950C01
:105DF0008C859D850F94C71942E150E060EC7CE2F0
:105E00008EEB9CE20F942C1E42E150E06CEA7CE2A7
:105E10008AEA9CE20F942C1E1092D12C1092D02C66
:105E2000DF91CF910C94A52E2F923F924F925F92CB
:105E30006F927F928F929F92AF92BF92CF92DF929A
:105E4000EF92FF920F931F93CF93DF93CDB7DEB7FF
:105E5000C05AD1090FB6F894DEBF0FBECDBF2C01DA
:105E60007B0148E050E064E670E00E9400BFD7018B
:105E70001296CD90DC901397C6010F942F198C01C8
:105E8000F70160817181A6010F94231ED70112963C
:105E9000ED91FC911397E00FF11F1082F801019032
:105EA0000020E9F7BF0161507109601B710B20E10F
:105EB00030E0AE014F575F4FC8010F94D501CF5767
:105EC000DF4F88819981C158D040892B19F4C801CE
:105ED0000F94C719AE014F575F4FB80180E090E0B3
:105EE0000F9443010F94131D0E94AA909F938F93C8
:105EF00082E69DE09F938F935F924F920E9426BF10
:105F0000CB57DF4FA880B980C558D040A00EB11E36
:105F1000C957DF4F68817981C758D04020E230E00F
:105F2000AE014F5B5F4FC5010F94D5010F900F90ED
:105F30000F900F900F900F9023968EAD9FAD2397EB
:105F4000892B41F1C757DF4FC880D980C958D0404D
:105F5000C00ED11EC557DF4F68817981CB58D04024
:105F600020E230E0AE014F5F5F4FC6010F94D501D4
:105F700089819A81892B71F0CE018F5B9F4F4C01F3
:105F8000DE0111967D01612C712C6DE6262E69E2F1
:105F9000362E5FC0C8010F94C71960E070E0C201DF
:105FA0000F94D80D89C0AE014F5B5F4FB501C3019F
:105FB0000F9443010F94131D0E94AA909F938F93F7
:105FC000AFE6BDE0BF93AF935F924F920E9426BFB2
:105FD000D7018D919C9111970197F601E80FF91F58
:105FE0000F900F900F900F900F900F902081223202
:105FF00061F411969C938E9312968D919C911397B8
:10600000029613969C938E931297F701808191814B
:106010000280F381E02DEC0DFD1DE80FF91F1082C9
:106020008C0D9D1D9F938F933F922F925F924F9265
:106030000E9426BFF2E06F0E711C84E0880E911C56
:1060400094E0E90EF11C0F900F900F900F900F90BD
:106050000F90D4018D919C91892B09F0A4CFC35747
:10606000DF4F88819981CD58D0400097E9F0C15722
:10607000DF4FE881F981CF58D040E00FF11FE80FE2
:10608000F91F1082800F911F9F938F9386E79DE0E9
:106090009F938F935F924F920E9426BF0F900F9015
:1060A0000F900F900F900F9063E273E1C2010F9475
:1060B000460FC8010F94C719C201C056DF4F0FB673
:1060C000F894DEBF0FBECDBFDF91CF911F910F912E
:1060D000FF90EF90DF90CF90BF90AF909F908F9008
:1060E0007F906F905F904F903F902F900895AF9268
:1060F000BF92CF92DF92EF92FF920F931F93CF93B5
:10610000DF93CDB7DEB760970FB6F894DEBF0FBE52
:10611000CDBF6C01B62EA72E7A018E01075F1F4FEF
:1061200048E050E064E670E0C8010E9400BF8FEED6
:10613000C8168EEBD806E9F4B701CE0101960E948D
:10614000142F8A818F9389818F93AF92BF928FE7AB
:106150009DE09F938F931F930F930E9426BFCE01C4
:1061600001960F94DA0C0FB6F894DEBF0FBECDBFC8
:106170001FC0CD2801F5AF92BF9288EA9DE09F93A2
:106180008F931F930F930E9426BFF7014281538183
:1061900060817181C8010E94DBC06AE17EE0C801B4
:1061A0000F94460F0F900F900F900F900F900F903D
:1061B000C8010E94782BC8010F94DA0C60960FB6C4
:1061C000F894DEBF0FBECDBFDF91CF911F910F912D
:1061D000FF90EF90DF90CF90BF90AF900895EF9237
:1061E000FF920F931F93CF93DF9300D01F92CDB7F1
:1061F000DEB78B017A018DE79BE20E948022882323
:10620000A1F0F701808191819A83898384819581AE
:106210009C838B838DE79BE20E949E1FAE014F5FA4
:106220005F4FBC01C8010E9477308091112C8823F8
:10623000C1F068E97CE083E496E40F94360B4AE011
:1062400050E0B80183E496E40F94AC0C66E97CE07E
:1062500083E496E40F94360BB70183E496E40F943D
:10626000880BF701808191810F94091E0097B1F18D
:106270002091BE2C3091BF2C232BC9F0E0ECFCE226
:1062800021E030E041915191452BE1F02F5F3F4FEC
:106290002A303105B9F70F900F900F900F90DF91D2
:1062A000CF911F910F91FF90EF900D94C71990938C
:1062B000BF2C8093BE2C1093AB2C0093AA2C0E9471
:1062C000A52E0CC0220F331FF901E254F34D918328
:1062D0008083F901E655F34D118300830F900F90F1
:1062E0000F900F90DF91CF911F910F91FF90EF9042
:1062F00008958F929F92AF92BF92CF92DF92EF92CA
:10630000FF920F931F93CF93DF93CDB7DEB7AA977A
:106310000FB6F894DEBF0FBECDBF8C01FC01E78045
:10632000F0848091112C882379F06FEB7EE083E478
:1063300096E40F94360BF801628173814AE050E0D5
:1063400083E496E40F94B20C8DE79BE20E948022D6
:10635000882389F0F801818590E00197FA82E9822B
:106360009C838B8360817181AE014F5F5F4F82811F
:1063700093810E947730F80182819381009709F41C
:10638000ADC08F3E9E4B09F4A9C0F70101900020DB
:10639000E9F73197EE19FF09339708F49FC0F70129
:1063A00080818B3509F09AC00F9406059B01AC01E2
:1063B000BE016F5F7F4FF801878190850E94069133
:1063C0006E01FDE1CF0ED11C41E050E064E170E0D0
:1063D000C6010E9400BFF80183818F9382818F9351
:1063E00081ED9DE09F938F93DF92CF920E9426BF15
:1063F0006D8D7E8D8EE49DE20E94135E0F900F9056
:106400000F900F900F900F90882309F462C07E01C7
:10641000F5E1EF0EF11C40E150E060E470E0C701EF
:106420000E9400BFF80181818F9380818F938381C7
:106430008F9382818F9382EE9DE09F938F93FF9243
:10644000EF920E9426BF8E010B5F1F4F0FB6F8948C
:10645000DEBF0FBECDBFE2E0AE2EB12CF5E28F2E37
:10646000FAE29F2E89819A818A159B05BCF0F8017A
:10647000808191810E5F1F4F9F938F939F928F9288
:10648000FF92EF920E9426BFFFEFAF1ABF0A0F9054
:106490000F900F900F900F900F90E4CF69EE71E185
:1064A000C7010F94460F6D897E89CE0185960F94A2
:1064B000480DAE014B5D5F4F60E070E08EE49DE201
:1064C0000E94E71FCE0185960F94DA0CC7010F9446
:1064D000DA0CC6010F94DA0C81E001C080E0AA96C4
:1064E0000FB6F894DEBF0FBECDBFDF91CF911F91E5
:1064F0000F91FF90EF90DF90CF90BF90AF909F9063
:106500008F900895EF92FF920F931F93CF93DF9395
:1065100000D01F92CDB7DEB77C018A01FA016481F9
:106520007581615071094CE2C8010F948C100F9471
:1065300006059F938F937F936F9389EF9DE09F93C1
:106540008F931F930F930E9426BFA8016FEE7EEBDF
:1065500081E19CE20E94EF30F801808191819A8371
:106560008983848195819C838B83BE016F5F7F4F7C
:10657000C7010E94142F0FB6F894DEBF0FBECDBF27
:10658000C7010F900F900F900F90DF91CF911F9147
:106590000F91FF90EF900895EF92FF920F931F934A
:1065A000CF93DF93CDB7DEB7A9970FB6F894DEBFD0
:1065B0000FBECDBF8091162C811112C0A0919D2DD0
:1065C000B0919E2D1097B1F11296ED91FC91139719
:1065D0000488F589E02DCD0102961995882351F1A3
:1065E0008E010E5D1F4F41E050E060E470E0C80195
:1065F0000E9400BF19A2CE0101967C01BC018DE76B
:106600009BE20E94801DFF92EF928EEF9DE09F9390
:106610008F931F930F930E9426BFC8010E94782B6F
:10662000C8010F94DA0C0F900F900F900F900F90FD
:106630000F900AC08091112C882331F06DE67CE028
:1066400083E496E40F94760BA9960FB6F894DEBF18
:106650000FBECDBFDF91CF911F910F91FF90EF90B3
:106660000895FC0165836623D1F067EA79E1069617
:106670000F94D80D4CED5BE263E08DE79BE20E9446
:10668000771F6FEE7EEB8DE79BE20E947B1F60E041
:1066900070E08DE79BE20E947B1F0C94CC32089542
:1066A000AF92BF92CF92DF92EF92FF920F931F9320
:1066B000CF93DF93CDB7DEB728970FB6F894DEBF40
:1066C0000FBECDBFF82EE92ED62EC72EB42EA52E86
:1066D00041E050E060E870E08E010F5F1F4FC8019D
:1066E0000E9400BFAF92BF92CF92DF92EF92FF92D3
:1066F0008DE19EE09F938F931F930F930E9426BF7F
:10670000C8010E94782BC8010F94DA0C0FB6F894D8
:10671000DEBF0FBECDBF28960FB6F894DEBF0FBE0A
:10672000CDBFDF91CF911F910F91FF90EF90DF9040
:10673000CF90BF90AF900895CF93DF93EC018091FD
:10674000112C882331F062EC7CE083E496E40F9412
:10675000360B99898091112C911120C0882331F03A
:106760006AEB7CE083E496E40F94760B20918B2C0B
:1067700030918C2C8091912C9091922C821B930BB8
:106780008536910508F440C02C593F4F30938C2C2E
:1067900020938B2CDF91CF910C94B12A2091892CDE
:1067A00030918A2C2F5F3F4F30938A2C2093892C75
:1067B00024303105E4F0882369F062EB7CE083E467
:1067C00096E40F94360B4AE050E0698983E496E43E
:1067D0000F94950C6091742C7091752C49E55EE0D6
:1067E0008091952C9091962C0E9450330DC0882357
:1067F00031F06CEA7CE083E496E40F94760BCE01F2
:10680000DF91CF910C941CF21092962C1092952C43
:1068100060E070E08DE89CE2DF91CF910D94D80D9F
:106820002F923F924F925F926F927F928F929F92A0
:10683000AF92BF92CF92DF92EF92FF920F931F938E
:10684000CF93DF93CDB7DEB7C655D1090FB6F89415
:10685000DEBF0FBECDBF1C018DE79BE20E948022F0
:10686000882309F45DC28091162C8823A9F0009139
:106870001B2C10911C2C67E17CE28CE69CE20F94AF
:106880003F0F67EA79E187E19CE20F94D80D10167B
:1068900011060CF44AC039C1A0919D2DB0919E2DD6
:1068A000109709F432C11296ED91FC911397048070
:1068B000F581E02DCD0102961995892B09F425C1AA
:1068C00060919D2D70919E2D6E5F7F4F40E850E04E
:1068D0008CE69CE20E949BBF181619060CF015C1AD
:1068E0000E94AE2D2A962FAF2A972B963FAF2B975B
:1068F0002C964FAF2C972D965FAF2D972E966FAF9E
:106900002E972F967FAF2F9760968FAF60972D961B
:106910008CAD9DADAEADBFAD2D978093122C9093F5
:10692000132CA093142CB093152C8E010F5B1F4FCA
:106930006AE08CE69CE20F9405116C0197FDE5C0BE
:106940008091112CC114D10409F4CDC0882361F0C9
:106950006EE57DE083E496E40F94360B6CE67CE212
:1069600083E496E40F94880B20E230E0AE014F5FA1
:106970005F4FB60180916C2C90916D2C0F94D501D6
:10698000892B09F0A9C0A0906C2CB0906D2CC60189
:106990000F942F197C01A601B5010F94231EAE019F
:1069A0004F5F5F4FB70185E69EE00F94BC015C012D
:1069B0008091112C882329F0B50183E496E40F948B
:1069C0009A0B6FEB72E1C5010F94501E892B79F47D
:1069D00068E27DE0C8010F940A0FA80160E070E052
:1069E0008EE49DE20E94E71FC8010F94DA0C67EA6B
:1069F0007CE1C5010F94501E892B09F069C0AE01DE
:106A00004F5F5F4FB7018AE69EE00F94BC010F9481
:106A1000131D5C01AE014F5F5F4FB70183EF94E13F
:106A20000F94BC014AE050E060E070E00F94F61B68
:106A30002B013C01AE014F5F5F4FB70187EA9CE13C
:106A40000F94BC014C01AE014F5F5F4FB7018AE666
:106A50009EE00F94BC01DC018C91882349F0411425
:106A600051046104710421F08114910409F0CEC035
:106A70008091112C882361F16EEF7CE083E496E431
:106A80000F94760B69EF7CE083E496E40F94360B69
:106A90004AE050E0B50183E496E40F94B20C64EF51
:106AA0007CE083E496E40F94360B2AE030E0B301F7
:106AB000A20183E496E40F94C80C6AEE7CE083E4C0
:106AC00096E40F94360BB40183E496E40F949A0B8A
:106AD000C7010F94C7190FC08091112C882359F05A
:106AE0006CE47DE004C0882331F063E47DE083E45E
:106AF00096E40F94760BA6014F5F5F4F60E070E065
:106B00008CE69CE20F94AB1213CF0E94AE2D6196DF
:106B10002FAF619762963FAF629763964FAF6397CF
:106B200064965FAF649765966FAF659766967FAF23
:106B3000669767968FAF679764968CAD9DADAEAD47
:106B4000BFAD6497F1014181528163817481841BDF
:106B5000950BA60BB70B8D329140A105B10508F43A
:106B6000DFC0D1018C91882391F10E94AE2D229635
:106B70002FAF229723963FAF239724964FAF2497AA
:106B800025965FAF259726966FAF269727967FAFFE
:106B9000279728968FAF289725964CAD5DAD6EADA3
:106BA0007FAD2597F10181819281A381B481481B3A
:106BB000590B6A0B7B0B2AE030E083E496E40F94D8
:106BC000810C66E77DE083E496E40F94760B0E94E7
:106BD000AE2D29833A834B835C836D837E838F83C1
:106BE00089819A81AB81BC81CC97A109B109F1015E
:106BF00081839283A383B48380919D2D90919E2D58
:106C0000009709F48DC00E945E868AC08DE79BE2E2
:106C10000E949E1FA816B90609F05AC0B401C80107
:106C20000F94480D64961FAE1EAE6497EDEAFEE029
:106C30006296FFAFEEAF629784E69CE266969FAFE6
:106C40008EAF6697A801BE01605B7F4F8EE49DE228
:106C50000E94E71FC8010F94DA0C41E050E060E0A9
:106C600070E0C8010E9400BF7F926F925F924F92C6
:106C7000BF92AF92ADE6BEE0BF93AF931F930F9369
:106C80000E9426BF4091682C5091692C6091642C21
:106C90007091652C21E0C8010E94DCBF6AE17EE0B2
:106CA000C8010F94460FC8010E94782B60E070E085
:106CB00084E69CE20F94D80DC7010F94C719C80150
:106CC0000F94DA0C0FB6F894DEBF0FBECDBF13CF12
:106CD0008091952C9091962C892B51F0C7010F949F
:106CE000C71944EA5EE0B201C5010E94503303CFE8
:106CF0005092752C4092742CB092962CA092952CA8
:106D0000B4018DE89CE20F94D80D10928C2C109257
:106D10008B2C10928A2C1092892C0E94B12AD8CEEA
:106D2000CA5ADF4F0FB6F894DEBF0FBECDBFDF915A
:106D3000CF911F910F91FF90EF90DF90CF90BF9078
:106D4000AF909F908F907F906F905F904F903F900B
:106D50002F9008950F9300E020E040E060E08BEF7B
:106D60009CE20F94C30A40E150E060E070E083EFE2
:106D70009CE20E9400BF41E050E060E070E082EDE4
:106D80009CE20E9400BF41E050E060E070E08DE8CE
:106D90009CE20E9400BF41E050E060E070E08CE6C1
:106DA0009CE20E9400BF41E050E060E070E084E6B9
:106DB0009CE20F910C9400BF0C94832C8091662D63
:106DC0009091672DA091682DBC018A2F90E00895C5
:106DD0006091622D7091632D8091642D9091652D4D
:106DE00008956091512D7091522D719561957109A1
:106DF000882777FD8095982F08956091532D709185
:106E0000542D882777FD8095982F08956091552DF2
:106E10007091562D882777FD8095982F089561E011
:106E200070E080E090E0089560E070E0CB010895AC
:106E30006CEF7FEF8FEF9FEF08956FEF7FEFCB0148
:106E4000089560E070E0CB01089561E070E080E0BB
:106E500090E0089562E070E080E090E0089563E0E3
:106E600070E080E090E0089561E070E080E090E004
:106E70000E941EDF21E0672B682B692B09F420E0BC
:106E80002093032C61E070E080E090E0089560E0E2
:106E900070E0CB010E941EDF672B682B692B39F055
:106EA00061E070E080E090E00E941EDF01C065E0DC
:106EB0006093232C70E080E090E0089560E070E043
:106EC000CB010E941EDF672B682B692B79F061E0F4
:106ED00070E080E090E00E941EDF21E061307105EB
:106EE0008105910509F020E0822F01C081E08093A7
:106EF000502D61E070E080E090E008956F927F9205
:106F00008F929F92AF92BF92CF92DF92EF92FF92B9
:106F10000F931F93CF93DF93CDB7DEB727970FB6AD
:106F2000F894DEBF0FBECDBF782E692E09831A8379
:106F30002B833C834D835E836F83C980DA80EB8033
:106F4000FC808D819E81AF81AC016A2F1F926F936F
:106F50005F938F938CE3882E912CA12CB12CC701C9
:106F6000B601A50194010F9481177F936F93CA0115
:106F7000B901A50194010F9481177F936F93C70105
:106F8000B60120E13EE040E050E00F948117CA01D5
:106F9000B90128E130E040E050E00F9481177F9381
:106FA0006F93C701B60120E831E541E050E00F944E
:106FB00081173F932F9381EB9EE09F938F936F9266
:106FC0007F920E9426BF0FB6F894DEBF0FBECDBFE2
:106FD00027960FB6F894DEBF0FBECDBFDF91CF91DD
:106FE0001F910F91FF90EF90DF90CF90BF90AF90E7
:106FF0009F908F907F906F9008952F923F924F9225
:107000005F926F927F928F929F92AF92BF92CF9238
:10701000DF92EF92FF920F931F93CF93DF93CDB741
:10702000DEB72C970FB6F894DEBF0FBECDBF7C0144
:1070300041E050E064E670E08E010F5F1F4FC80131
:107040000E9400BF88EE90E30E94FEBB9C0188EE88
:1070500090E32B873C870E94FABB382E292E88EEBE
:1070600090E30E94F6BB582E492E88EE90E30E94D2
:10707000BEBB782E692E88EE90E30E94BABB982E94
:10708000892E88EE90E30E94B6BBB82EA92E40E070
:1070900050E0BA018DEF96E10E945990D82EC92E8A
:1070A00040E050E0BA0186E091E20E945990898761
:1070B0009A8740E050E0BA0186E091E20E94599040
:1070C0003C853F932B852F932F923F924F925F9257
:1070D0006F927F928F929F92AF92BF92CF92DF92E8
:1070E0002A852F9329852F939F938F9381EE9EE07E
:1070F0009F938F931F930F930E9426BFA80161E176
:107100007CE2C7010E948232C8010F94DA0C0FB6EC
:10711000F894DEBF0FBECDBFC7012C960FB6F89412
:10712000DEBF0FBECDBFDF91CF911F910F91FF90BA
:10713000EF90DF90CF90BF90AF909F908F907F9017
:107140006F905F904F903F902F900895CF93DF9373
:10715000CDB7DEB728970FB6F894DEBF0FBECDBF10
:10716000CE0101960E94FD37CE0101960E940BDAF6
:10717000CE0101960F94DA0C61E070E080E090E0BF
:1071800028960FB6F894DEBF0FBECDBFDF91CF912A
:107190000895CF92DF92EF92FF920F931F93CF93B8
:1071A000DF93CDB7DEB728970FB6F894DEBF0FBEDA
:1071B000CDBF7C0141E050E064E670E08E010F5FDE
:1071C0001F4FC8010E9400BF40E050E0BA0188E5AF
:1071D0009CE10E945990D82EC92E40E050E0BA019F
:1071E00086E09FE00E945990CF92DF929F938F9309
:1071F00080E19FE09F938F931F930F930E9426BF80
:1072000062EA7FE0C8010F94460FA80161E17CE2C9
:10721000C7010E948232C8010F94DA0C0FB6F894AD
:10722000DEBF0FBECDBFC70128960FB6F894DEBFF4
:107230000FBECDBFDF91CF911F910F91FF90EF90C7
:10724000DF90CF900895CF93DF93CDB7DEB7289727
:107250000FB6F894DEBF0FBECDBFCE0101960E94DF
:10726000C938CE0101960E940BDACE0101960F9427
:10727000DA0C61E070E080E090E028960FB6F894B8
:10728000DEBF0FBECDBFDF91CF9108958DE79BE2AA
:107290000E942721682F772767FD7095872F972FEA
:1072A00008958DE79BE20E942521682F772767FDCF
:1072B0007095872F972F08955F926F927F928F928C
:1072C0009F92AF92BF92CF92DF92EF92FF920F9375
:1072D0001F93CF93DF93CDB7DEB728970FB6F894FF
:1072E000DEBF0FBECDBF7C0141E050E064E670E040
:1072F0008E010F5F1F4FC8010E9400BF8DE79BE208
:107300000E94581D582E8DE79BE20E942721C82E0F
:107310008DE79BE20E942521D82E40E050E0BA0183
:1073200086E995E10E945990782E692E40E050E060
:10733000BA0182E795E10E945990982E892E40E08B
:1073400050E0BA0181E793E10E945990B82EA92E2E
:1073500040E050E0BA018CE19FE00E945990252D59
:10736000332727FD30953F935F922C2D332727FD40
:1073700030953F93CF922D2D332727FD30953F93A6
:10738000DF926F927F928F929F92AF92BF929F9364
:107390008F9381E29FE09F938F931F930F930E949F
:1073A00026BFA80161E17CE2C7010E948232C801C8
:1073B0000F94DA0C0FB6F894DEBF0FBECDBFC70135
:1073C00028960FB6F894DEBF0FBECDBFDF91CF91E8
:1073D0001F910F91FF90EF90DF90CF90BF90AF90F3
:1073E0009F908F907F906F905F900895CF93DF93E1
:1073F000CDB7DEB728970FB6F894DEBF0FBECDBF6E
:10740000CE0101960E945C39CE0101960E940BDAF2
:10741000CE0101960F94DA0C61E070E080E090E01C
:1074200028960FB6F894DEBF0FBECDBFDF91CF9187
:1074300008958DE79BE20E947B22682F70E080E038
:1074400090E008958DE79BE20E94D520682F70E0C0
:1074500080E090E008958DE79BE20E94EF20BC0160
:10746000882777FD8095982F08958DE79BE20E94ED
:10747000DE20BC01882777FD8095982F08952F92F4
:107480003F924F925F926F927F928F929F92AF92B4
:10749000BF92CF92DF92EF92FF920F931F93CF9301
:1074A000DF93CDB7DEB72C970FB6F894DEBF0FBED3
:1074B000CDBF6C0141E050E064E670E08E010F5FEB
:1074C0001F4FC8010E9400BF8DE79BE20E947B22F4
:1074D000882329F020E2E22E2DE0F22E04C095E26E
:1074E000E92E9DE0F92E8DE79BE20E94D5208823AE
:1074F00019F020E23DE002C025E23DE08DE79BE28D
:107500002B873C870E94EF2089879A878DE79BE233
:107510000E94DE20382E292E40E050E0BA0189EC8E
:1075200093E10E945990582E492E40E050E0BA0154
:1075300085E392E10E945990782E692E40E050E058
:10754000BA0189EA93E10E945990982E892E40E071
:1075500050E0BA018DE893E10E945990B82EA92E0F
:1075600040E050E0BA018FE394E10E945990FF920D
:10757000EF922B853C853F932F932A852F93298566
:107580002F932F923F924F925F926F927F928F92A2
:107590009F92AF92BF929F938F938CE39FE09F93B4
:1075A0008F931F930F930E9426BFA80161E17CE295
:1075B000C6010E948232C8010F94DA0C0FB6F8940B
:1075C000DEBF0FBECDBFC6012C960FB6F894DEBF4E
:1075D0000FBECDBFDF91CF911F910F91FF90EF9024
:1075E000DF90CF90BF90AF909F908F907F906F90E3
:1075F0005F904F903F902F900895CF93DF93CDB73A
:10760000DEB728970FB6F894DEBF0FBECDBFCE0110
:1076100001960E943F3ACE0101960E940BDACE01FC
:1076200001960F94DA0C61E070E080E090E028961B
:107630000FB6F894DEBF0FBECDBFDF91CF91089596
:107640002F923F924F925F926F927F928F929F9272
:10765000AF92BF92CF92DF92EF92FF920F931F9360
:10766000CF93DF93CDB7DEB768970FB6F894DEBF40
:107670000FBECDBF7C0141E050E064E670E08E01BA
:107680000F5F1F4FC8010E9400BFE9EDFBE22081A0
:1076900029873181E7EDFBE220812A8721812B8731
:1076A000E5EDFBE220812C8721812D87E3EDFBE2D4
:1076B00020812E8721812F87E1EDFBE22081288B1D
:1076C0002181298BEFECFBE220812A8B21812B8BFE
:1076D000EDECFBE220812C8B21812D8BEBECFBE28E
:1076E00020812E8B21816FE18DE79BE2288F3F8BDC
:1076F0000E941923682E6EE18DE79BE20E941923F8
:10770000782E6DE18DE79BE20E941923882E6CE1B3
:107710008DE79BE20E941923982E6BE18DE79BE297
:107720000E941923A82E6AE18DE79BE20E9419238B
:10773000B82E69E18DE79BE20E941923C82E68E10B
:107740008DE79BE20E941923D82E40E050E0BA0159
:107750008DE59FE00E945990382E292E40E050E0A0
:10776000BA0188EB97E10E945990582E492E40E0CB
:1077700050E0BA0184E298E10E9459903F893F931A
:1077800039853F933B853F933A853F933D853F93B2
:107790003C853F933F853F933E853F9339893F9397
:1077A00038893F933B893F933A893F933D893F9383
:1077B0003C893F93288D2F932E892F93262D332795
:1077C00027FD30953F936F92272D332727FD309566
:1077D0003F937F92282D332727FD30953F938F923B
:1077E000292D332727FD30953F939F922A2D33274C
:1077F00027FD30953F93AF922B2D332727FD3095F2
:107800003F93BF922C2D332727FD30953F93CF9286
:107810002D2D332727FD30953F93DF922F923F92F6
:107820004F925F929F938F9383E69FE09F938F93F6
:107830001F930F930E9426BF0FB6F894DEBF0FBEB2
:10784000CDBFA80161E17CE2C7010E948232C8017C
:107850000F94DA0CC70168960FB6F894DEBF0FBE1E
:10786000CDBFDF91CF911F910F91FF90EF90DF90EF
:10787000CF90BF90AF909F908F907F906F905F90D0
:107880004F903F902F900895CF93DF93CDB7DEB701
:1078900028970FB6F894DEBF0FBECDBFCE0101967C
:1078A0000E94203BCE0101960E940BDACE01019688
:1078B0000F94DA0C61E070E080E090E028960FB65B
:1078C000F894DEBF0FBECDBFDF91CF9108952F9208
:1078D0003F924F925F926F927F928F929F92AF9260
:1078E000BF92CF92DF92EF92FF920F931F93CF93AD
:1078F000DF93CDB7DEB765970FB6F894DEBF0FBE46
:10790000CDBF7C0141E050E064E670E08E010F5F86
:107910001F4FC8010E9400BFEBEAFBE220813181CA
:10792000E9EAFBE28081898791819A87E7EAFBE2B5
:1079300080818B8791819C87E5EAFBE280818D873E
:1079400091819E87E3EAFBE280818F879181988B0A
:10795000E1EAFBE28081898B91819A8BEFE9FBE27E
:1079600080818B8B218068E08DE79BE22C8B3D8BA7
:107970000E941923782E67E08DE79BE20E9419236D
:10798000882E66E08DE79BE20E941923982E65E021
:107990008DE79BE20E941923A82E64E08DE79BE20D
:1079A0000E941923B82E63E08DE79BE20E94192301
:1079B000C82E62E08DE79BE20E941923D82E40E09A
:1079C00050E0BA018DE59FE00E945990482E392E73
:1079D00040E050E0BA0188EB97E10E945990682E90
:1079E000592E40E050E0BA0181E198E10E9459909F
:1079F0003D893F932C892F932A852F9329852F9397
:107A00002C852F932B852F932E852F932D852F93A8
:107A100028892F932F852F932A892F9329892F9394
:107A20002F922B892F93272D332727FD30953F93B6
:107A30007F92282D332727FD30953F938F92292D54
:107A4000332727FD30953F939F922A2D332727FD1B
:107A500030953F93AF922B2D332727FD30953F93E1
:107A6000BF922C2D332727FD30953F93CF922D2D9C
:107A7000332727FD30953F93DF923F924F925F92DD
:107A80006F929F938F9386EA9FE09F938F931F93AC
:107A90000F930E9426BF0FB6F894DEBF0FBECDBF76
:107AA000A80161E17CE2C7010E948232C8010F9403
:107AB000DA0CC70165960FB6F894DEBF0FBECDBFD6
:107AC000DF91CF911F910F91FF90EF90DF90CF90BA
:107AD000BF90AF909F908F907F906F905F904F90EE
:107AE0003F902F900895CF93DF93CDB7DEB72897BF
:107AF0000FB6F894DEBF0FBECDBFCE0101960E9437
:107B0000673CCE0101960E940BDACE0101960F94DC
:107B1000DA0C61E070E080E090E028960FB6F8940F
:107B2000DEBF0FBECDBFDF91CF910895EF92FF92E0
:107B30000F931F93CF93DF93CDB7DEB728970FB680
:107B4000F894DEBF0FBECDBF88EE90E30E94BEBBAF
:107B5000F82EE92E88EE90E30E94BABB182F092F69
:107B600088EE90E30E94B6BBEF92FF920F931F93B3
:107B70009F938F9383EE9FE09F938F931F9288E054
:107B80008F938E010F5F1F4F1F930F930F94351F1D
:107B9000C8010E9407DA0F940605AB01BC01C801B9
:107BA0000E945990BC01882777FD8095982F0FB6C9
:107BB000F894DEBF0FBECDBF28960FB6F894DEBF97
:107BC0000FBECDBFDF91CF911F910F91FF90EF902E
:107BD00008958F929F92AF92BF92CF92DF92EF92D1
:107BE000FF920F931F9363E070E080E090E00E94AB
:107BF0001EDF6B017C0162E070E080E090E00E949B
:107C00001EDF4B015C0161E070E080E090E00E94CB
:107C10001EDFAB01BC01950184018DE79BE20E9450
:107C2000BA2261E070E080E090E01F910F91FF9038
:107C3000EF90DF90CF90BF90AF909F908F9008957E
:107C400081E08093042C8DE79BE20E94A6228DE7C1
:107C50009BE20E94AE228DE79BE20E94B62261E089
:107C600070E080E090E008951092042C8DE79BE294
:107C70000E94A2228DE79BE20E94AA228DE79BE24E
:107C80000E94B22261E070E080E090E0089561E03F
:107C900070E080E090E00E941EDF21E0672B682BFF
:107CA000692B09F420E0622F81E19CE20E94A22E60
:107CB00061E070E080E090E0089561E070E080E0D5
:107CC00090E00E941EDF21E0672B682B692B09F4EE
:107CD00020E0622F81E19CE20E94A22E61E070E030
:107CE00080E090E00E941EDF21E0672B682B692B6B
:107CF00009F420E020934D2D61E070E080E090E0F9
:107D00000E941EDF21E0672B682B692B09F420E01D
:107D100020934F2D61E070E080E090E00E941EDF34
:107D200021E0672B682B692B09F420E02093032CBA
:107D300061E070E080E090E00895CF93DF93CDB7ED
:107D4000DEB7A1970FB6F894DEBF0FBECDBFBE0160
:107D50006F5F7F4F8DE79BE20E94801D19A2CE01CD
:107D600001960E9407DA0F940605AB01BC01CE0113
:107D700001960E945990BC01882777FD8095982F25
:107D8000A1960FB6F894DEBF0FBECDBFDF91CF91A5
:107D900008950F931F93CF93DF9300D000D0CDB7FA
:107DA000DEB76AEC7FE1CE0101960F940A0FCE0197
:107DB00001960E940BDACE0101960F94DA0C6BEB60
:107DC0007FE1CE0101960F940A0FCE0101960E9429
:107DD0000BDACE0101960F94DA0C0091702E1091FF
:107DE000712E0115110529F1D80112968C91882365
:107DF00019F080EF9FE002C08BEF9FE00E94CCD88B
:107E0000D801ED91FC910480F581E02DC801199510
:107E1000BC01CE0101960F940A0FCE0101960E947B
:107E20000BDACE0101960F94DA0CF801038114816C
:107E3000D8CF61E070E080E090E026960FB6F8942D
:107E4000DEBF0FBECDBFDF91CF911F910F9108957F
:107E50008DE79BE20E94A71D8DE79BE20E94952281
:107E600008958DE79BE20E94952208958DE79BE29D
:107E70000E94561F61E070E080E090E008958DE779
:107E80009BE20E948022682F70E080E090E00895DD
:107E90002F923F924F925F926F927F928F929F921A
:107EA000AF92BF92CF92DF92EF92FF920F931F9308
:107EB000CF93DF93CDB7DEB76C970FB6F894DEBFE4
:107EC0000FBECDBF7C0141E050E064E670E0CE0122
:107ED00001960E9400BF8DE79BE20E94AD1F182F04
:107EE000092F8DE79BE20E94B11F6B877C878D87EE
:107EF0009E878DE79BE20E94A91F8F87988B8DE755
:107F00009BE20E94AC1D698B7A8B8B8B9C8B8DE7DF
:107F10009BE20E94B01D8D8B9E8B8DE79BE20E94A1
:107F2000B41D89878DE79BE20E94B81D8A878DE783
:107F30009BE20E948022882319F020E23DE002C0EB
:107F400025E23DE040E050E0BA0186E090E12B8F71
:107F50003C8F0E9459908F8B988F40E050E0BA017F
:107F60008FE090E10E945990382E292E40E050E099
:107F7000BA0185E190E10E945990582E492E40E0C7
:107F800050E0BA018CE190E10E945990782E692E60
:107F900040E050E0BA0183E290E10E945990982EAF
:107FA000892E40E050E0BA018AE290E10E945990A7
:107FB000B82EA92E40E050E0BA0183E390E10E9480
:107FC0005990D82EC92E40E050E0BA018BE390E1E1
:107FD0000E945990898F9A8F40E050E0BA0187E162
:107FE00095E10E9459900F931F934E854F934D85B5
:107FF0004F934C854F934B854F9348894F934F85B3
:108000004F934C894F934B894F934A894F9349899A
:108010004F934E894F934D894F931F9249854F93AC
:108020001F924A854F932B8D3C8D3F932F93288D24
:108030002F932F892F932F923F924F925F926F929F
:108040007F928F929F92AF92BF92CF92DF922A8DB2
:108050002F93298D2F939F938F9380E490E19F938B
:108060008F938E010F5F1F4F1F930F930E9426BFA8
:108070000FB6F894DEBF0FBECDBFA80161E17CE270
:10808000C7010E948232C8010F94DA0CC7016C96B6
:108090000FB6F894DEBF0FBECDBFDF91CF911F9119
:1080A0000F91FF90EF90DF90CF90BF90AF909F9097
:1080B0008F907F906F905F904F903F902F9008959A
:1080C000CF93DF93CDB7DEB728970FB6F894DEBF16
:1080D0000FBECDBFCE0101960E94483FCE01019652
:1080E0000E940BDACE0101960F94DA0C61E070E089
:1080F00080E090E028960FB6F894DEBF0FBECDBFAB
:10810000DF91CF910895AF92BF92CF92DF92EF921D
:10811000FF920F931F93CF93DF935C016B01EA01F2
:10812000F12C8F2D90E08C159D05B8F4F501E80F2A
:10813000F91F608170E080E090E030E3E32E02E020
:1081400010E020E030E040E10E941FDA209719F0B3
:10815000CE010E94CCD8F394E4CFDF91CF911F9150
:108160000F91FF90EF90DF90CF90BF90AF90089568
:108170000F931F93CF93DF93CDB7DEB727970FB63B
:10818000F894DEBF0FBECDBF8091892D81110FC045
:108190006AE67CE1CE0101960F940A0FCE010196AA
:1081A0000E940BDACE0101960F94DA0C64C01F8294
:1081B0008F819091892D891708F05DC00091872DDE
:1081C0001091882D92E1899F000D111D112440E02E
:1081D00050E061E070E0CE0107960E94834067E6C0
:1081E0007CE1CE0101960F940A0FCE0101960E9408
:1081F000D8D8CE0101960F94DA0CC8010E94F28102
:10820000009779F464E57CE1CE0101960F940A0FA2
:10821000CE0101960E94D8D8CE0101960F94DA0CB7
:1082200003C005960E94CCD861E57CE1CE010196A1
:108230000F940A0FCE0101960E94D8D8CE01019664
:108240000F94DA0C40E050E068E070E0C8010E9452
:1082500083406FE47CE1CE0101960F940A0FCE01BA
:1082600001960E940BDACE0101960F94DA0C8F81F1
:108270008F5F8F839DCF60E070E0CB0127960FB6B4
:10828000F894DEBF0FBECDBFDF91CF911F910F914C
:108290000895AF92BF92CF92DF92EF920F931F9308
:1082A000CF93DF9300D000D0CDB7DEB761E070E0B0
:1082B00080E090E00E941EDF97FD0AC00091892DAA
:1082C00010E020E030E0601771078207930794F018
:1082D00061EC7DE1CE0101960F940A0FCE0101966B
:1082E0000E940BDACE0101960F94DA0C60E070E088
:1082F000CB011EC122E1269F8001279F100D112472
:108300008091872D9091882D800F911F0E94F2817E
:108310005C01C090872DD090882DC00ED11E61EBDE
:108320007DE1CE0101960F940A0FCE0101960E94C5
:10833000D8D8CE0101960F94DA0CC50105960E949B
:1083400007DA60EA7DE1CE0101960F940A0FCE01B3
:1083500001960E94D8D8CE0101960F94DA0CF6014E
:108360006281718180E090E040E3E42E02E010E061
:1083700020E030E040E10E941FDA0E94B7D96FE8A8
:108380007DE1CE0101960F940A0FCE0101960E9465
:10839000D8D8CE0101960F94DA0CF6011381812F03
:1083A00082958F700E9424D96DE87DE1CE010196FF
:1083B0000F940A0FCE0101960E94D8D8CE010196E3
:1083C0000F94DA0C812F8F700E940FDA6BE77DE13A
:1083D000CE0101960F940A0FCE0101960E94D8D8C3
:1083E000CE0101960F94DA0CF6017581668102E0E8
:1083F00010E020E030E040E1848190E00E941FDA4C
:108400000E94B7D96BE57DE1CE0101960F940A0F6A
:10841000CE0101960E94D8D8CE0101960F94DA0CB5
:10842000F60180810E9424D968E57DE1CE010196A4
:108430000F940A0FCE0101960E940BDACE0101962D
:108440000F94DA0C68E37DE1CE0101960F940A0FD8
:10845000CE0101960E94D8D8CE0101960F94DA0C75
:10846000F50183810E940FDA60E27DE1CE01019681
:108470000F940A0FCE0101960E94D8D8CE01019622
:108480000F94DA0CF50180810E9424D96DE17DE121
:10849000CE0101960F940A0FCE0101960E940BDACD
:1084A000CE0101960F94DA0C6FE07DE1CE010196CA
:1084B0000F940A0FCE0101960E94D8D8CE010196E2
:1084C0000F94DA0CF50181810E9424D968E07DE1E6
:1084D000CE0101960F940A0FCE0101960E940BDA8D
:1084E000CE0101960F94DA0C6AEF7CE1CE01019681
:1084F0000F940A0FCE0101960E94D8D8CE010196A2
:108500000F94DA0CF50182810E9424D963EF7CE19B
:10851000CE0101960F940A0FCE0101960E940BDA4C
:10852000CE0101960F94DA0C61E070E080E090E0FB
:1085300026960FB6F894DEBF0FBECDBFDF91CF9168
:108540001F910F91EF90DF90CF90BF90AF90089563
:108550007F928F929F92AF92BF92CF92DF92EF92D3
:10856000FF920F931F93CF93DF9300D000D0CDB72E
:10857000DEB760E17CE1CE0101960F940A0FCE01D7
:1085800001960E940BDACE0101960F94DA0C00E0FE
:1085900010E0C12CD12C7601C394702E6CE07CE1EC
:1085A000CE0101960F940A0FCE0101960E94D8D8F1
:1085B000CE0101960F94DA0C602F8DE79BE20E94AA
:1085C0009523BC01CE0101960F940A0FCE010196AE
:1085D0000E94D8D8CE0101960F94DA0C62E07CE1BB
:1085E000CE0101960F940A0FCE0101960E94D8D8B1
:1085F000CE0101960F94DA0C802F0E9424D966EFE9
:108600007BE1CE0101960F940A0FCE0101960E94E4
:10861000D8D8CE0101960F94DA0C602F8DE79BE23B
:108620000E941923B82E682F8DE79BE20E94A12398
:10863000009719F46EEE7BE101C0BC01CE010196FA
:108640000F940A0FCE0101960E94D8D8CE01019650
:108650000F94DA0C63EE7BE1CE0101960F940A0FC2
:10866000CE0101960E94D8D8CE0101960F94DA0C63
:10867000B7FE04C08DE20E9408D907C0672D8DE7C0
:108680009BE20E944E230E945ED989E193E10E9401
:10869000CCD8672D8DE79BE20E942423882371F0BC
:1086A00066ED7BE1CE0101960F940A0FCE01019693
:1086B0000E94D8D8CE0101960F94DA0C872D0E9423
:1086C00006798823C9F16AEC7BE1CE0101960F940B
:1086D0000A0FCE0101960E94D8D8CE0101960F94C0
:1086E000DA0CB701A601002E04C0440F551F661F07
:1086F000771F0A94D2F780905E2D90905F2DA09006
:10870000602DB090612D482159216A217B21452B94
:10871000462B472B19F068EC7BE102C066EC7BE14D
:10872000CE0101960F940A0FCE0101960E94D8D86F
:10873000CE0101960F94DA0C64EC7BE1CE01019638
:108740000F940A0FCE0101960E94D8D8CE0101964F
:108750000F94DA0C8FE1781671F062EC7BE1CE01B8
:1087600001960F940A0FCE0101960E94D8D8CE012F
:1087700001960F94DA0C0E94B7D90F5F1F4F003299
:10878000110509F00ACF60EC7BE1CE0101960F9450
:108790000A0FCE0101960E940BDACE0101960F94CA
:1087A000DA0C61E070E080E090E026960FB6F89475
:1087B000DEBF0FBECDBFDF91CF911F910F91FF9014
:1087C000EF90DF90CF90BF90AF909F908F907F9071
:1087D000089588EE90E30E9437BB682F70E080E038
:1087E00090E0089588EE90E30E9499BC61E070E00B
:1087F00080E090E00895CF92DF92EF92FF920F9386
:108800001F93CF93DF93CDB7DEB764970FB6F8947D
:10881000DEBF0FBECDBF8DE79BE20E94371D1982E0
:108820008E010F5F1F4F60E7E62E63E1F62EFC011D
:1088300024916C01FFEFCF1ADF0A2223C9F0D8017F
:108840000D900020E9F7822F992787FD90959F933F
:108850002F93FF92EF921197BF93AF930F94721FD4
:10886000C6010F900F900F900F900F900F90DFCFD9
:1088700040E050E0BA01C8010E945990BC0188272D
:1088800077FD8095982F64960FB6F894DEBF0FBEE3
:10889000CDBFDF91CF911F910F91FF90EF90DF90AF
:1088A000CF9008950F94001B882777FD8095982F0F
:1088B00008954F925F926F927F928F929F92AF92A4
:1088C000BF92CF92DF92EF92FF920F931F93CF93BD
:1088D000DF93CDB7DEB760970FB6F894DEBF0FBE5B
:1088E000CDBF8E01075F1F4F41E050E064E670E0AE
:1088F000C8010E9400BF0E948CBE7C010E94DABEAB
:10890000582E492E0E9467BE782E692E40E050E016
:10891000BA018BE391E10E945990982E892E40E094
:1089200050E0BA0181E899E10E945990B82EA92E31
:1089300040E050E0BA018FE790E10E945990D82EB4
:10894000C92E40E050E0BA0184E890E10E945990BD
:108950004F925F92FF92EF926F927F928F929F92CF
:10896000AF92BF92CF92DF929F938F9381E29FE06D
:108970009F938F931F930F930E9426BFA80161E1DD
:108980007CE2CE0101960E948232CE0101960E94C5
:108990000BDACE0101960F94DA0CC8010F94DA0CB1
:1089A000B701882777FD8095982F0FB6F894DEBF22
:1089B0000FBECDBF60960FB6F894DEBF0FBECDBF21
:1089C000DF91CF911F910F91FF90EF90DF90CF90AB
:1089D000BF90AF909F908F907F906F905F904F90DF
:1089E00008959F92AF92BF92CF92DF92EF92FF9243
:1089F0000F931F93CF93DF93B82E6B018A017901F8
:108A000083E190E00F942F19EC018EE0FE011192AA
:108A10008A95E9F7BB2011F083E001C082E18987E4
:108A2000DE82CD828DE29DE5988B8F8782E08F83F9
:108A30008887F80101900020E9F7CF010197801B9A
:108A4000910BF70101900020E9F73197EE19FF092A
:108A50008E0F9F1F02960F942F195C019D878C87A4
:108A6000F80101900020E9F79E2E901A9E86B80129
:108A70000F94591EB701C501890D911D0F94591E00
:108A8000CE010E941CF280914F2D8823E1F166E710
:108A900076E183E496E40F94360B4AE050E0B601A9
:108AA00083E496E40F944F0C63E776E183E496E465
:108AB0000F94360B4AE050E06E8583E496E40F9401
:108AC0008E0C60E776E183E496E40F94360B6C85B8
:108AD0007D8583E496E40F949A0B6AE676E183E45D
:108AE00096E40F94360BB70183E496E4DF91CF91BF
:108AF0001F910F91FF90EF90DF90CF90BF90AF90BC
:108B00009F900D949A0BDF91CF911F910F91FF9041
:108B1000EF90DF90CF90BF90AF909F900895AF926D
:108B2000BF92CF92DF92EF92FF920F931F93CF935A
:108B3000DF9300D000D0CDB7DEB764EE71E1CE0197
:108B400001960F940A0FCE0101960E94D8D8CE014B
:108B500001960F94DA0C0E94B7D90E9442F46C017E
:108B60008C01E12CF12CF80181819281019609F4AC
:108B700098C06CED71E1CE0101960F940A0FCE0101
:108B800001960E94D8D8CE0101960F94DA0CF80114
:108B9000808181700E9424D96EEC71E1CE01019632
:108BA0000F940A0FCE0101960E94D8D8CE010196EB
:108BB0000F94DA0CF8018081869581700E9424D987
:108BC00060EC71E1CE0101960F940A0FCE0101967F
:108BD0000E94D8D8CE0101960F94DA0CF80180815A
:108BE00082958F700E9424D962EB71E1CE010196CB
:108BF0000F940A0FCE0101960E94D8D8CE0101969B
:108C00000F94DA0CF801818192810E945ED964EAA6
:108C100071E1CE0101960F940A0FCE0101960E94D8
:108C2000D8D8CE0101960F94DA0CF8018381948193
:108C30000E945ED967E971E1CE0101960F940A0F97
:108C4000CE0101960E94D8D8CE0101960F94DA0C7D
:108C50005601AE0CBF1CF50185810E9424D96BE83A
:108C600071E1CE0101960F940A0FCE0101960E9488
:108C7000D8D8CE0101960F94DA0CF50186810E94B6
:108C800024D964E871E1CE0101960F940A0FCE0158
:108C900001960E94D8D8CE0101960F94DA0C0E945A
:108CA000B7D9F7E0EF0EF11C095F1F4F2CE8E21671
:108CB000F10409F058CF61E070E080E090E0269682
:108CC0000FB6F894DEBF0FBECDBFDF91CF911F91DD
:108CD0000F91FF90EF90DF90CF90BF90AF900895ED
:108CE0008DE79BE20E949E1FBC0180E090E008950A
:108CF0002F923F924F925F926F927F928F929F92AC
:108D0000AF92BF92CF92DF92EF92FF920F931F9399
:108D1000CF93DF93CDB7DEB72F970FB6F894DEBFB2
:108D20000FBECDBF7C0141E050E064E670E09E01E3
:108D30002F5F3F4F6901C9010E9400BF0E9442F4AA
:108D400020E030E000E010E0FC01E20FF31F418181
:108D500052814F3F5F4F11F00F5F1F4F295F3F4F11
:108D60002C38310589F78DE79BE20E94A61F282F3A
:108D70008DE79BE22F870E94A21F382E292E8DE7B8
:108D80009BE20E949E1F582E492E40E050E0BA01FF
:108D90008FE394E10E945990782E692E40E050E0D4
:108DA000BA0181E594E10E945990982E892E40E005
:108DB00050E0BA018FE294E10E945990B82EA92E9A
:108DC00040E050E0BA018BE890E10E945990898719
:108DD0009A8740E050E0BA0182E990E10E94599000
:108DE0008B879C8740E050E0BA018AE990E10E94BD
:108DF0005990382F9D8740E050E0BA0182EA90E117
:108E00003E870E9459901F922F852F931F930F9397
:108E10002F923F924F925F926F927F928F929F928A
:108E2000AF92BF922A852F9329852F932C852F935C
:108E30002B852F932D852F933E853F939F938F9363
:108E400087EA90E19F938F93DF92CF920E9426BF93
:108E50008DE79BE20E94C71F0FB6F894DEBF0FBEDE
:108E6000CDBFFC0164918C010F5F1F4F662329F079
:108E7000C6010F94560FC801F4CF6EEC70E1C60125
:108E80000F94460F8DE79BE20E94B71FFC0164918F
:108E90008C010F5F1F4F662329F0C6010F94560FF8
:108EA000C801F4CF69ED72E1C6010F94460FA60127
:108EB00061E17CE2C7010E948232C6010F94DA0CA4
:108EC000C7012F960FB6F894DEBF0FBECDBFDF915E
:108ED000CF911F910F91FF90EF90DF90CF90BF90B7
:108EE000AF909F908F907F906F905F904F903F904A
:108EF0002F900895CF93DF93CDB7DEB728970FB6A5
:108F0000F894DEBF0FBECDBFCE0101960E94784619
:108F1000CE0101960E940BDACE0101960F94DA0C75
:108F200061E070E080E090E028960FB6F894DEBF34
:108F30000FBECDBFDF91CF910895CF93DF93CDB713
:108F4000DEB761970FB6F894DEBF0FBECDBFBE018E
:108F50006F5F7F4F8DE79BE20E943F1F198ACE0112
:108F600001960E9407DA0F940605AB01BC01CE0101
:108F700001960E945990BC01882777FD8095982F13
:108F800061960FB6F894DEBF0FBECDBFDF91CF91D3
:108F900008958DE79BE20E94D22861E070E080E0B6
:108FA00090E008958DE79BE20E94BE2861E070E0AA
:108FB00080E090E008958DE79BE20E94FA20682F00
:108FC00070E080E090E00895CF92DF92EF92FF9200
:108FD0000F931F93CF93DF9300D000D0CDB7DEB7B0
:108FE00061E070E080E090E00E941EDF97FD0AC023
:108FF0000091892D10E020E030E0601771078207B2
:1090000093071CF064E97CE11CC042E1469F90019B
:10901000479F300D11248091872D9091882D60E01D
:1090200070E0820F931F0E94C3817C01009739F08A
:1090300000E010E06C018FEFC81AD80A24C06DE779
:109040007CE1CE0101960F940A0FCE0101960E9499
:109050000BDACE0101960F94DA0C60E070E0CB01E0
:109060001CC0601B710B6930710510F068E070E086
:1090700044E050E1C601800F911F0E9483400E948E
:10908000B7D9085F1F4FF701608170E00617170717
:1090900040F361E070E080E090E026960FB6F8942F
:1090A000DEBF0FBECDBFDF91CF911F910F91FF901B
:1090B000EF90DF90CF900895CF92DF92EF92FF92E2
:1090C00060E070E0CB010E941EDF62307105810517
:1090D0009105C9F462E070E080E090E00E941EDF3C
:1090E0006B017C0161E070E080E090E00E941EDF97
:1090F00041E0CD28CE28CF2809F440E088EE90E367
:109100000E94FABD15C060E070E0CB010E941EDF36
:10911000613071058105910539F461E070E080E00E
:1091200090E00E941EDFE9CF88EE90E30E9427BD09
:1091300061E070E080E090E0FF90EF90DF90CF90F2
:109140000895CF92DF92EF92FF9260E070E0CB0142
:109150000E941EDF6230710581059105C9F462E04D
:1091600070E080E090E00E941EDF6B017C0161E016
:1091700070E080E090E00E941EDF41E0CD28CE2824
:10918000CF2809F440E088EE90E30E94E9BD15C0C5
:1091900060E070E0CB010E941EDF61307105810547
:1091A000910539F461E070E080E090E00E941EDFFC
:1091B000E9CF88EE90E30E941FBD61E070E080E09F
:1091C00090E0FF90EF90DF90CF900895CF92DF92E4
:1091D000EF92FF9260E070E0CB010E941EDF6230F0
:1091E000710581059105C9F462E070E080E090E0CE
:1091F0000E941EDF6B017C0161E070E080E090E086
:109200000E941EDF41E0CD28CE28CF2809F440E09F
:1092100088EE90E30E94D8BD15C060E070E0CB01FD
:109220000E941EDF613071058105910539F461E00E
:1092300070E080E090E00E941EDFE9CF88EE90E3CE
:109240000E9417BD61E070E080E090E0FF90EF9039
:10925000DF90CF900895CF92DF92EF92FF9260E07F
:1092600070E0CB010E941EDF62307105810591051F
:10927000C9F462E070E080E090E00E941EDF6B01C4
:109280007C0161E070E080E090E00E941EDF41E040
:10929000CD28CE28CF2809F440E088EE90E30E9444
:1092A000C7BD15C060E070E0CB010E941EDF6130D9
:1092B00071058105910539F461E070E080E090E08E
:1092C0000E941EDFE9CF88EE90E30E940FBD61E0AF
:1092D00070E080E090E0FF90EF90DF90CF900895F5
:1092E000CF92DF92EF92FF9260E070E0CB010E949C
:1092F0001EDF6230710581059105C9F462E070E0FE
:1093000080E090E00E941EDF6B017C0161E070E074
:1093100080E090E00E941EDF41E0CD28CE28CF28DB
:1093200009F440E088EE90E30E94B6BD15C060E00D
:1093300070E0CB010E941EDF61307105810591054F
:1093400039F461E070E080E090E00E941EDFE9CF38
:1093500088EE90E30E9407BD61E070E080E090E05D
:10936000FF90EF90DF90CF900895CF92DF92EF9231
:10937000FF9260E070E0CB010E941EDF6230710559
:1093800081059105C9F462E070E080E090E00E9400
:109390001EDF6B017C0161E070E080E090E00E94E4
:1093A0001EDF41E0CD28CE28CF2809F440E088EE2A
:1093B00090E30E94A5BD15C060E070E0CB010E9463
:1093C0001EDF613071058105910539F461E070E0BF
:1093D00080E090E00E941EDFE9CF88EE90E30E94DB
:1093E000FFBC61E070E080E090E0FF90EF90DF90E4
:1093F000CF900895CF92DF92EF92FF9260E070E0FD
:10940000CB010E941EDF6230710581059105C9F410
:1094100062E070E080E090E00E941EDF6B017C0162
:1094200061E070E080E090E00E941EDF41E0CD2826
:10943000CE28CF2809F440E088EE90E30E9494BD46
:1094400015C060E070E0CB010E941EDF6130710545
:109450008105910539F461E070E080E090E00E94C0
:109460001EDFE9CF88EE90E30E94F7BC61E070E078
:1094700080E090E0FF90EF90DF90CF900895CF9242
:10948000DF92EF92FF9260E070E0CB010E941EDF5E
:109490006230710581059105C9F462E070E080E0F9
:1094A00090E00E941EDF6B017C0161E070E080E0D3
:1094B00090E00E941EDF41E0CD28CE28CF2809F49D
:1094C00040E088EE90E30E9483BD15C060E070E04C
:1094D000CB010E941EDF613071058105910539F4D1
:1094E00061E070E080E090E00E941EDFE9CF88EE4E
:1094F00090E30E94EFBC61E070E080E090E0FF90BC
:10950000EF90DF90CF900895CF92DF92EF92FF928D
:1095100060E070E0CB010E941EDF623071058105C2
:109520009105C9F462E070E080E090E00E941EDFE7
:109530006B017C0161E070E080E090E00E941EDF42
:1095400041E0CD28CE28CF2809F440E088EE90E312
:109550000E9472BD15C060E070E0CB010E941EDF6A
:10956000613071058105910539F461E070E080E0BA
:1095700090E00E941EDFE9CF88EE90E30E94E7BCF6
:1095800061E070E080E090E0FF90EF90DF90CF909E
:109590000895CF92DF92EF92FF9260E070E0CB01EE
:1095A0000E941EDF6230710581059105C9F462E0F9
:1095B00070E080E090E00E941EDF6B017C0161E0C2
:1095C00070E080E090E00E941EDF41E0CD28CE28D0
:1095D000CF2809F440E088EE90E30E9461BD15C0F9
:1095E00060E070E0CB010E941EDF613071058105F3
:1095F000910539F461E070E080E090E00E941EDFA8
:10960000E9CF88EE90E30E94DFBC61E070E080E08B
:1096100090E0FF90EF90DF90CF900895CF92DF928F
:10962000EF92FF9260E070E0CB010E941EDF62309B
:10963000710581059105C9F462E070E080E090E079
:109640000E941EDF6B017C0161E070E080E090E031
:109650000E941EDF41E0CD28CE28CF2809F440E04B
:1096600088EE90E30E940BBE15C060E070E0CB0175
:109670000E941EDF613071058105910539F461E0BA
:1096800070E080E090E00E941EDFE9CF88EE90E37A
:109690000E9450BE61E070E080E090E0FF90EF90AB
:1096A000DF90CF90089560E070E0CB010E941EDF54
:1096B000672B682B692B31F461E081E19CE20E9409
:1096C00031330AC061E070E080E090E00E941EDF6C
:1096D00087E19CE20F94460F61E070E080E090E04B
:1096E0000895CF93DF93CDB7DEB728970FB6F894E0
:1096F000DEBF0FBECDBF8091042C811108C0CE010A
:1097000001960E94FD37CE0101960F94DA0C28963F
:109710000FB6F894DEBF0FBECDBFDF91CF91089595
:1097200061E070E080E090E00E94D1D7672B682B69
:10973000692B51F061E070E080E090E00E9473DFFF
:109740008DE79BE20C94782361E070E080E090E08C
:109750000E941EDF97FD13C061E070E080E090E0A2
:109760000E941EDF603271058105910544F461E0BD
:1097700070E080E090E00E941EDF862F08958FEF5A
:1097800008950F931F93CF93DF9300D000D0CDB7F0
:10979000DEB7082F0E94904B182F8F3F19F46DE70A
:1097A0007BE123C0682F8DE79BE20E94B0238823D2
:1097B00019F06AE57BE119C0033051F4612F8DE7A0
:1097C0009BE20E942423811103C067E37BE10DC06B
:1097D000602F8DE79BE20E94A123892B21F083E07B
:1097E000800F823090F466E27BE1CE0101960F9407
:1097F0000A0FCE0101960E940BDACE0101960F945A
:10980000DA0C60E070E0CB010FC0402F612F8DE7D4
:109810009BE20E945925811103C06CE07BE1E5CFFA
:1098200061E070E080E090E026960FB6F894DEBF2D
:109830000FBECDBFDF91CF911F910F910895DC0135
:10984000ED91FC910190F081E02D1994CF92DF927F
:10985000EF92FF920F931F93CF93DF9300D000D02E
:10986000CDB7DEB77C016B01FB0101900020E9F769
:109870008F0101501109061B170B67EA79E10F945C
:10988000480D4AE060E070E0CE0101960F94360E7C
:10989000CE0101960F94DA0CF701D182C0821583B4
:1098A000048326960FB6F894DEBF0FBECDBFDF91BE
:1098B000CF911F910F91FF90EF90DF90CF9008957F
:1098C000242FFB0142815381608171810C94DCBFA4
:1098D000CF93DF93CDB7DEB727970FB6F894DEBFEF
:1098E0000FBECDBF0E94AE2D6D837E838F838D8191
:1098F0009E81AF81BC018A2F90E027960FB6F89425
:10990000DEBF0FBECDBFDF91CF910895CF93DF9320
:10991000CDB7DEB727970FB6F894DEBF0FBECDBF29
:109920000E94AE2D29833A834B835C8369817A81BF
:109930008B819C8127960FB6F894DEBF0FBECDBFFA
:10994000DF91CF9108952F923F924F925F926F9245
:109950007F928F929F92AF92BF92CF92DF92EF92BF
:10996000FF920F931F93CF93DF93CDB7DEB7AF97DF
:109970000FB6F894DEBF0FBECDBF6C018E010B5E3B
:109980001F4F41E050E064E670E0C8010E9400BF54
:109990000E948CBE8DE79BE20E94371D44E150E09F
:1099A000BC01CE0101967C010F94FA1D1C8A0F9414
:1099B000001B962E872EE2E6FDE2908198A721817A
:1099C00029A742814AA783818BA70E94AE2DB42E7E
:1099D000A52E2D8F3E8F4F8F58A369A37AA38BA3FB
:1099E00040E050E0BA018BE696E12EA73FA70E9427
:1099F00059908CA79DA740E050E0BA0182ED90E11C
:109A00000E945990382E292E40E050E0BA018AED8C
:109A10009CE10E945990582E492E40E050E0BA0136
:109A200089ED90E10E945990782E692E40E050E037
:109A3000BA018FED90E10E9459908F929F924BA5B1
:109A40004F934AA54F9349A54F9348A54F93AF9283
:109A5000BF923FA53F932EA52F932DA52F932CA505
:109A60002F932F923F924F925F926F927F929F938C
:109A70008F9386EE90E19F938F931F930F930E9495
:109A800026BFFDA2ECA2F70101900020E9F7319773
:109A9000EE19FF09FFA3EEA341E0BE016C5D7F4F0D
:109AA000C8010E94604C6AED72E1C8010F94460F34
:109AB000A80161E17CE2C6010E948232C8010F94D4
:109AC000DA0C0FB6F894DEBF0FBECDBFC601AF965D
:109AD0000FB6F894DEBF0FBECDBFDF91CF911F91BF
:109AE0000F91FF90EF90DF90CF90BF90AF909F903D
:109AF0008F907F906F905F904F903F902F90089540
:109B0000CF93DF93CDB7DEB728970FB6F894DEBFBB
:109B10000FBECDBFCE0101960E94A34CCE0101968F
:109B20000E940BDACE0101960F94DA0C61E070E02E
:109B300080E090E028960FB6F894DEBF0FBECDBF50
:109B4000DF91CF9108956F927F928F92CF92DF92A3
:109B5000EF92CF93DF93CDB7DEB72E970FB6F89481
:109B6000DEBF0FBECDBF0E94AE2D288739874A8742
:109B70005B876C877D878E876090662D7090672DE0
:109B80008090682D88859985AA85BB85CC84DD84E5
:109B9000EE844091622D5091632D6091642D7091FF
:109BA000652D841B950BA60BB70BC614D704E804D0
:109BB00048F420ECC21A2DEBD20A20EFE20A0197FA
:109BC000A109B10989839A83AB83BC83C618D708DE
:109BD000E808CD82DE82EF82282F3A814B815C81BA
:109BE0006C2D7E818F8190E02E960FB6F894DEBFAB
:109BF0000FBECDBFDF91CF91EF90DF90CF908F90D0
:109C00007F906F900895CF93DF93CDB7DEB72797FE
:109C10000FB6F894DEBF0FBECDBF0E94A34D2983BF
:109C20003A834B835C8369817A818B819C812796FF
:109C30000FB6F894DEBF0FBECDBFDF91CF91089570
:109C4000CF93DF93CDB7DEB727970FB6F894DEBF7B
:109C50000FBECDBF0E94A34D6D837E838F838D8108
:109C60009E81AF81BC018A2F90E027960FB6F894B1
:109C7000DEBF0FBECDBFDF91CF9108950F931F932D
:109C8000CF93DF93CDB7DEB766970FB6F894DEBFFC
:109C90000FBECDBF41E050E064E670E0CE0101961A
:109CA0000E9400BF68EC78E1CE0101960F94E80EA7
:109CB0000E94AE2D89019A01AB01682FCE01019659
:109CC0000E947E3789819A810E9407DA60EC78E1F0
:109CD000CE0101960F94E80E0E94A34D89019A01CE
:109CE000AB01682FCE0101960E947E3789819A814F
:109CF0000E9407DA67EB78E1CE0101960F94E80E37
:109D00000091622D1091632D2091642D3091652D6D
:109D10004091662D5091672D6091682DCE0101967E
:109D20000E947E3789819A810E9407DACE010196CE
:109D30000F94DA0C61E070E080E090E066960FB678
:109D4000F894DEBF0FBECDBFDF91CF911F910F9171
:109D50000895CF92DF92EF92FF920F931F93CF93CC
:109D6000DF9300D000D0CDB7DEB7F82E8B0160E0D6
:109D700070E0CB010E941EDFCF2CD12CE12CF12C06
:109D80006C157D058E059F0579F0B801CE01019611
:109D90000F940A0FCE0101960E940BDACE010196B4
:109DA0000F94DA0C80E001C081E026960FB6F8949B
:109DB000DEBF0FBECDBFDF91CF911F910F91FF90FE
:109DC000EF90DF90CF90089568EF70E281E00E94FD
:109DD000A94E882399F061E070E080E090E00E9455
:109DE0001EDFCB010E94AA90009741F00F94131D33
:109DF000BC01882777FD8095982F089560E070E07A
:109E0000CB01089562EE70E281E00E94A94E8823A2
:109E100091F061E070E080E090E00E941EDFCB01F5
:109E20000E94AA90009739F00E9407DA61E070E082
:109E300080E090E0089560E070E0CB0108956DEC63
:109E400070E281E00E94A94E882371F061E070E029
:109E500080E090E00E941EDFCB010E94B89061E09C
:109E600070E080E090E0089560E070E0CB0108953C
:109E700060E170E281E00E94A94E882379F061E000
:109E800070E080E090E00E9473DF8DE79BE20E942B
:109E9000691D61E070E080E090E0089560E070E0AE
:109EA000CB010895CF93DF9300D000D0CDB7DEB7BC
:109EB00062EF7FE181E00E94A94E882321F161E0F9
:109EC00070E080E090E00E9473DFCB010E94099275
:109ED000892BE9F469ED7FE1CE0101960F940A0F19
:109EE000CE0101960E94D8D8CE0101960F94DA0CCB
:109EF00061E070E080E090E00E9473DFCB010E949F
:109F0000CCD80E94B7D960E070E0CB0104C061E01A
:109F100070E080E090E026960FB6F894DEBF0FBEAA
:109F2000CDBFDF91CF91089562E17CE181E00E9495
:109F3000A94E882349F00E94904B682F772767FD30
:109F40007095872F972F089560E070E0CB010895FA
:109F5000CF92DF92EF92FF921F93CF93DF9300D0C7
:109F600000D0CDB7DEB766EE7AE182E00E94A94E5E
:109F7000882309F442C00E94904B182F62E070E0E1
:109F800080E090E00E941EDF6B017C011F3F19F40E
:109F900063ED7AE126C0612F8DE79BE20E944023AA
:109FA000811103C067EA7AE11CC0612F8DE79BE253
:109FB0000E941923833041F48FEFC816D10421F099
:109FC00018F065E97AE10DC0612F8DE79BE20E94F0
:109FD00019238330B1F082E0C816D10490F063E811
:109FE0007AE1CE0101960F940A0FCE0101960E94EC
:109FF0000BDACE0101960F94DA0C60E070E0CB0131
:10A000000AC04C2D612F8DE79BE20E94C52561E0BF
:10A0100070E080E090E026960FB6F894DEBF0FBEA9
:10A02000CDBFDF91CF911F91FF90EF90DF90CF9048
:10A030000895CF93DF9300D000D0CDB7DEB768E6A8
:10A040007AE181E00E94A94E8823E1F00E94904BC2
:10A050008F3F79F465E57AE1CE0101960F940A0FFE
:10A06000CE0101960E940BDACE0101960F94DA0C14
:10A0700009C0682F8DE79BE20E944E23BC0180E05F
:10A0800090E003C060E070E0CB0126960FB6F89434
:10A09000DEBF0FBECDBFDF91CF9108956EE27AE1B2
:10A0A00082E00E94A94E882349F062E070E080E0DF
:10A0B00090E00E941EDF862F0C94C14B60E070E0A0
:10A0C000CB01089560E17AE181E00E94A94E8823E6
:10A0D00019F08FEF0C94C14B60E070E0CB01089554
:10A0E00069EE79E181E00E94A94E882319F083E0AE
:10A0F0000C94C14B60E070E0CB0108956BEC79E10A
:10A1000081E00E94A94E882319F083E00C94C14B92
:10A1100060E070E0CB0108956AEA79E181E00E9495
:10A12000A94E882319F081E00C94C14B60E070E0E7
:10A13000CB010895CF92DF92EF92FF92CF93DF93FE
:10A1400000D01F92CDB7DEB76BE479E183E00E94C7
:10A15000A94E882331F163E070E080E090E00E9436
:10A160001EDF9B01AC0162E070E080E090E029839B
:10A170003A834B835C830E941EDF6B017C0161E0AC
:10A1800070E080E090E00E941EDF29813A81A60104
:10A1900088EE90E30E94C2BB61E070E080E090E056
:10A1A00003C060E070E0CB010F900F900F900F9014
:10A1B000DF91CF91FF90EF90DF90CF900895CF92F5
:10A1C000DF92EF92FF92CF93DF9300D01F92CDB733
:10A1D000DEB767E279E183E00E94A94E882331F17E
:10A1E00063E070E080E090E00E941EDF9B01AC0124
:10A1F00062E070E080E090E029833A834B835C83E7
:10A200000E941EDF6B017C0161E070E080E090E065
:10A210000E941EDF29813A81A60188EE90E30E9408
:10A220004CBC61E070E080E090E003C060E070E072
:10A23000CB010F900F900F900F90DF91CF91FF9077
:10A24000EF90DF90CF9008951F93CF93DF931F92ED
:10A25000CDB7DEB76FE778E181E00E94A94E882391
:10A26000E1F061E070E080E090E00E941EDF8DE7A9
:10A270009BE269830E942521182F8DE79BE20E94B3
:10A28000581D6981680F611B8DE79BE20E945B1D71
:10A2900061E070E080E090E003C060E070E0CB013E
:10A2A0000F90DF91CF911F9108956BE578E181E0E8
:10A2B0000E94A94E882379F061E070E080E090E090
:10A2C0000E941EDF8DE79BE20E945B1D61E070E053
:10A2D00080E090E0089560E070E0CB0108956AE6C8
:10A2E00071E181E00E94A94E882399F061E070E05D
:10A2F00080E090E00E941EDF21E0672B682B692B35
:10A3000009F420E020934D2D61E070E080E090E0C2
:10A31000089560E070E0CB0108956DE471E181E0A3
:10A320000E94A94E882379F061E070E080E090E01F
:10A330000E941EDF8DE79BE20E949B1F682F70E04A
:10A3400080E090E0089560E070E0CB0108956DE258
:10A3500071E181E00E94A94E882379F061E070E00C
:10A3600080E090E00E941EDF8DE79BE20E948B1F41
:10A3700061E070E080E090E0089560E070E0CB0183
:10A3800008956EE071E181E00E94A94E882379F082
:10A3900061E070E080E090E00E941EDF8DE79BE2CC
:10A3A0000E947B1F61E070E080E090E0089560E033
:10A3B00070E0CB0108950F931F93CF93DF93CDB738
:10A3C000DEB760970FB6F894DEBF0FBECDBF64EF67
:10A3D00070E181E00E94A94E882399F161E070E06C
:10A3E00080E090E00E9473DFFB0101900020E9F71C
:10A3F0008F0101501109061B170B40E150E06FEF70
:10A4000070E0CE0101960F943E1E61E070E080E0A6
:10A4100090E00E9473DFA8010131110514F040E1C2
:10A4200050E0CE0101960F94231EBE016F5F7F4F57
:10A430008DE79BE20E944C1E61E070E080E090E0BE
:10A4400003C060E070E0CB0160960FB6F894DEBF09
:10A450000FBECDBFDF91CF911F910F91089562ED97
:10A4600070E181E00E94A94E882379F061E070E0FC
:10A4700080E090E00E941EDF8DE79BE20E94EC1DD1
:10A4800061E070E080E090E0089560E070E0CB0172
:10A49000089561EB70E181E00E94A94E882379F074
:10A4A00061E070E080E090E00E941EDF8DE79BE2BB
:10A4B0000E94D41D61E070E080E090E0089560E0CB
:10A4C00070E0CB01089561E970E181E00E94A94E3E
:10A4D000882379F061E070E080E090E00E941EDF68
:10A4E0008DE79BE20E94BC1D61E070E080E090E09F
:10A4F000089560E070E0CB010895AF92BF92CF92D3
:10A50000DF92EF92FF920F931F93CF93DF9300D0D0
:10A5100000D0CDB7DEB7A82EB62E8A0160E070E07D
:10A52000CB010E941EDFCA2CD12CE12CF12C6C1522
:10A530007D058E059F0584F060E070E0CB010E94F0
:10A540001EDFCB2CD12CE12CF12CC616D706E80649
:10A55000F90614F081E00EC0B801CE0101960F9407
:10A560000A0FCE0101960E940BDACE0101960F94DC
:10A57000DA0C80E026960FB6F894DEBF0FBECDBF92
:10A58000DF91CF911F910F91FF90EF90DF90CF90CF
:10A59000BF90AF900895CF92DF92EF92FF924AEA78
:10A5A00050E262E081E00E947D52882309F45EC09F
:10A5B00060E070E0CB010E941EDF62307105810512
:10A5C00091054CF062E070E080E090E00E941EDFB8
:10A5D0006B017C0103C0C12CD12C760161E070E0DD
:10A5E00080E090E00E94D1D7672B682B692B91F017
:10A5F00061E070E080E090E00E9473DFDC01CB015D
:10A60000B701A6010E945990BC01882777FD80956B
:10A61000982F2FC061E070E080E090E00E941EDF84
:10A620009F938F937F936F9385E091E19F938F9397
:10A630001F9288E08F9381E09DE29F938F930F9408
:10A64000351FB701A60181E09DE20E945990BC012F
:10A65000882777FD8095982F2DB73EB7265F3F4F0F
:10A660000FB6F8943EBF0FBE2DBF03C060E070E090
:10A67000CB01FF90EF90DF90CF9008954FE25CE127
:10A6800060E080E00E947D52882321F08DE79BE20C
:10A690000E94A82560E070E0CB01089542E759E1EF
:10A6A00062E081E00E947D528823C9F060E070E0A2
:10A6B000CB010E941EDF623071058105910569F4AE
:10A6C00062E070E080E090E00E941EDF672B682B64
:10A6D000692B19F480E00C94C14B82E0FCCF60E060
:10A6E00070E0CB0108954F925F926F927F928F92AC
:10A6F0009F92AF92BF92CF92DF92EF92FF920F9311
:10A700001F93CF93DF9300D01F92CDB7DEB740EDFC
:10A7100058E165E083E00E947D52882309F498C0E7
:10A7200060E070E0CB010E941EDF6530710581059D
:10A730009105B1F565E070E080E090E00E941EDFD9
:10A740006B017C0164E070E080E090E00E941EDF1D
:10A750004B015C0163E070E080E090E00E941EDF4E
:10A760009B01AC0162E070E080E090E029833A83D5
:10A770004B835C830E941EDF2B013C0161E070E093
:10A7800080E090E00E941EDFE1E029813A81CD283F
:10A79000CE28CF2809F4E0E0EE2E8401A20131C0DA
:10A7A00060E070E0CB010E941EDF6430710581051E
:10A7B000910581F564E070E080E090E00E941EDF8A
:10A7C0002B013C0163E070E080E090E00E941EDF1E
:10A7D0009B01AC0162E070E080E090E029833A8365
:10A7E0004B835C830E941EDF4B015C0161E070E0E3
:10A7F00080E090E00E941EDFE12C820129813A81F5
:10A80000A40188EE90E30E942FBD61E070E080E03B
:10A8100090E021C063E070E080E090E00E941EDFE5
:10A820009B01AC0162E070E080E090E029833A8314
:10A830004B835C830E941EDF4B015C0161E070E092
:10A8400080E090E00E941EDFE12C04EF11E0D6CF03
:10A8500060E070E0CB010F900F900F900F90DF91B0
:10A86000CF911F910F91FF90EF90DF90CF90BF900D
:10A87000AF909F908F907F906F905F904F900895D2
:10A880000F931F93CF93DF9300D000D0CDB7DEB7E7
:10A890004BE250E162E081E00E947D52882309F49E
:10A8A00051C00E94904B182F60E070E0CB010E94D5
:10A8B0001EDF623071058105910569F462E070E088
:10A8C00080E090E00E941EDF01E0672B682B692B7F
:10A8D00019F400E001C001E01F3F19F468E170E1E4
:10A8E0001BC0812F0E940679811103C066EF7FE0B3
:10A8F00013C0612F8DE79BE20E94B023882319F0DB
:10A900006FEC7FE009C0612F8DE79BE20E9433234B
:10A9100081110FC06FEA7FE0CE0101960F940A0FFC
:10A92000CE0101960E940BDACE0101960F94DA0C4B
:10A9300009C0602F812F0E94C07861E070E080E044
:10A9400090E003C060E070E0CB0126960FB6F8946B
:10A95000DEBF0FBECDBFDF91CF911F910F91089544
:10A96000CF92DF92EF92FF92CF93DF9300D000D08F
:10A97000CDB7DEB749E750E262E081E00E947D5248
:10A980008823A9F160E070E0CB010E941EDF6230F5
:10A99000710581059105A1F462E070E080E090E02E
:10A9A0000E941EDF6B017C0161E070E080E090E0BE
:10A9B0000E9473DFCE0101960E94264CA6010CC0B6
:10A9C00061E070E080E090E00E9473DFCE010196CC
:10A9D0000E94264C40E050E060E0CE0101960E94CB
:10A9E00035901A821982CE0101960F94DA0C60E03C
:10A9F00070E0CB0126960FB6F894DEBF0FBECDBF38
:10AA0000DF91CF91FF90EF90DF90CF9008952F923C
:10AA10003F924F925F926F927F928F929F92AF92EE
:10AA2000BF92CF92DF92EF92FF920F931F93CF933B
:10AA3000DF9300D01F92CDB7DEB74B015C018A01D6
:10AA400020E030E0A9010F94A21387FD05C060E06B
:10AA500070E080E09FE304C060E070E080E09FEB86
:10AA6000E12CF12CE016F10654F420E030E040E255
:10AA700051E40F94A6132FEFE21AF20AF3CF9B01D1
:10AA8000AC01C501B4010F943E136B017C0120E0C1
:10AA900030E0A901C501B4010F94A21387FF04C0DF
:10AAA000F7FAF094F7F8F0941C821B828DEC782E64
:10AAB0009CEC692E2CEC522E3DE3432E20E030E03E
:10AAC00040E251E4672D762D852D942D0F94A3152A
:10AAD0001B0189839A83A70196010F94A21318166C
:10AAE00054F08B819C8101969C838B83722C632C08
:10AAF00059804A80E3CF20E030E0A901C501B401CC
:10AB00000F94A21387FF03C08DE20E9408D9EB8146
:10AB1000FC81EF2B19F480E30E9408D9212C312C01
:10AB20008B819C8128163906B4F5272D362D452DAD
:10AB3000542DC701B6010F94A6130F940E144B01A8
:10AB40005C01CB010E9441D9B401882777FD809533
:10AB5000982F0F944514272D362D452D542D0F94E5
:10AB6000A3159B01AC01C701B6010F943D136B0106
:10AB70007C0120E030E040E251E4672D762D852D08
:10AB8000942D0F94A613762E672E582E492EFFEF84
:10AB90002F1A3F0AC5CF101611065CF58EE20E94EF
:10ABA00008D9612C712C20E030E040E251E4C7016B
:10ABB000B6010F94A3156B017C010F940E144B0189
:10ABC0005C01CB010E9441D9B401882777FD8095B3
:10ABD000982F0F9445149B01AC01C701B6010F9447
:10ABE0003D136B017C019FEF691A790A60167106AB
:10ABF000D1F60F900F900F900F90DF91CF911F9192
:10AC00000F91FF90EF90DF90CF90BF90AF909F900B
:10AC10008F907F906F905F904F903F902F9008950E
:10AC2000CF92DF92EF92FF928DE79BE20E94EF209E
:10AC3000BC01882777FD8095982F0F94451420E05C
:10AC400030E048EC52E40F94A6136B017C0142E023
:10AC500050E00E9407550E94B7D9C701B6010F9472
:10AC60000E14882777FD8095982FFF90EF90DF9046
:10AC7000CF9008950E9407550C94B7D94F925F92D8
:10AC80006F927F928F929F92AF92BF92CF92DF92FC
:10AC9000EF92FF920F931F93CF93DF93CDB7DEB761
:10ACA00028970FB6F894DEBF0FBECDBF4C018B01C5
:10ACB00041E050E064E670E00E9400BF60E070E0B8
:10ACC000CB010E941EDF5B0189E0A816B1041CF0D5
:10ACD00048E0A42EB12C6BE77AE2C4010F94D80DA2
:10ACE00017FF02C092E013C01F930F9381E091E120
:10ACF0009F938F939F928F920E9426BF0F900F90E9
:10AD00000F900F900F900F90012B61F791E080E072
:10AD1000092F182FC12CD12C7601C801AA2797FD25
:10AD2000A095BA2F8D839E83AF83B887A016B106F6
:10AD30000CF446C04D805E806F8078844C0C5D1CA6
:10AD40006E1C7F1CC301B2010E94D1D7672B682BF8
:10AD5000692B69F0C301B2010E9473DFDC01CB01F2
:10AD600041E050E060E070E00E94599005C0C301EE
:10AD7000B2010E941EDFCB010E94AA909A838983B0
:10AD8000DC010D900020E9F71197A81BB90BBC83DB
:10AD9000AB8341E0BE016F5F7F4FC4010E94604CF6
:10ADA0000A151B052CF463E071E1C4010F94460FF2
:10ADB0000F5F1F4F9FEFC91AD90AE90AF90AB6CFE8
:10ADC00060E07FE1C4010F94460FC40128960FB6DE
:10ADD000F894DEBF0FBECDBFDF91CF911F910F91D1
:10ADE000FF90EF90DF90CF90BF90AF909F908F90AB
:10ADF0007F906F905F904F900895AF92BF92CF92E7
:10AE0000DF92EF92FF920F931F93CF93DF93CDB713
:10AE1000DEB728970FB6F894DEBF0FBECDBF44E46F
:10AE200050E26FEF82E00E947D52882309F4A0C0B7
:10AE300061E070E080E090E00E94D1D7672B682B42
:10AE4000692B41F061E070E080E090E00E941EDF3D
:10AE50008B010AC061E070E080E090E00E941EDF9C
:10AE6000CB010E94AA908C010115110521F0F80177
:10AE70008081811103C089E091E127C06FEF7FEFEE
:10AE8000CE0101960E943E5689819A810F94091E37
:10AE90007C01CE0101960F94DA0CD7010D900020B1
:10AEA000E9F71197AE19BF09F80101900020E9F701
:10AEB0003197E01BF10BEA0FFB1FE135F10540F084
:10AEC000C7010F94C71980E391E10E9407DA50C0CF
:10AED00067EA79E181E39DE20F94D80D40E050E00C
:10AEE000BA0181E491E10E945990B82EA92E40E068
:10AEF00050E0BA0188E491E10E945990D82EC92E01
:10AF000040E050E0BA0181E491E10E945990FF9243
:10AF1000EF921F930F93AF92BF92CF92DF929F93C6
:10AF20008F932DE431E13F932F9321E33DE23F9353
:10AF30002F930E9426BFC7010F94C71941E35DE21A
:10AF400061E17CE2CE0101960E948232CE0101963F
:10AF50000E940BDACE0101960F94DA0C0FB6F8942A
:10AF6000DEBF0FBECDBF61E070E080E090E003C0C7
:10AF700060E070E0CB0128960FB6F894DEBF0FBEFC
:10AF8000CDBFDF91CF911F910F91FF90EF90DF9098
:10AF9000CF90BF90AF900895CF93DF93CDB7DEB73A
:10AFA00028970FB6F894DEBF0FBECDBF6BE270E2FC
:10AFB00081E00E94A94E8823C1F060E070E0CE01DC
:10AFC00001960E943E56AE014F5F5F4F60E070E019
:10AFD00081E19CE20E94EF30CE0101960F94DA0CE1
:10AFE00061E070E080E090E003C060E070E0CB01E1
:10AFF00028960FB6F894DEBF0FBECDBFDF91CF917C
:10B000000895CF93DF93CDB7DEB728970FB6F894A6
:10B01000DEBF0FBECDBF42E358E163E681E00E9490
:10B020007D528823E1F061E070E0CE0101960E943C
:10B030003E5661E070E080E090E00E941EDFAE01CD
:10B040004F5F5F4F81E19CE20E94EF30CE0101969D
:10B050000F94DA0C61E070E080E090E003C060E003
:10B0600070E0CB0128960FB6F894DEBF0FBECDBFBF
:10B07000DF91CF910895CF92DF92EF92FF921F93CD
:10B08000CF93DF93CDB7DEB728970FB6F894DEBF26
:10B090000FBECDBF49E058E163E681E00E947D52DA
:10B0A000882309F45DC061E070E0CE0101960E9442
:10B0B0003E5661E070E080E090E00E941EDF6B0190
:10B0C0007C018091392D811142C0D092402DC092D7
:10B0D0003F2D11E01093412D1093422D83E080937A
:10B0E000432D89819A810F94091E9093472D809357
:10B0F000462D8D818F5F8093482D85E09AE6909351
:10B100004A2D8093492D8AE39DE20E941CF2109300
:10B11000392D80914D2D8823D1F062EF77E183E4C2
:10B1200096E40F94360B4AE050E0B60183E496E4CF
:10B130000F944F0C6FEE77E183E496E40F94360B97
:10B14000BE016F5F7F4F83E496E40F94880BCE01BE
:10B1500001960F94DA0C61E070E080E090E003C0AB
:10B1600060E070E0CB0128960FB6F894DEBF0FBE0A
:10B17000CDBFDF91CF911F91FF90EF90DF90CF90E7
:10B180000895CB01BA010C94BFDFBF92CF92DF923A
:10B19000EF92FF920F931F93CF93DF93CDB7DEB75C
:10B1A00064970FB6F894DEBF0FBECDBF41E050E00C
:10B1B00060E070E08E010F5F1F4FC8010E9400BF6A
:10B1C00067EA79E189E29DE20F94D80D64E671E1C6
:10B1D000CE0109960F94480D1A8A198A8DEA9EE0CD
:10B1E000988B8F871C8B0B8BAE01475F5F4FBE0127
:10B1F000615F7F4F8EE49DE20E94E71FCE010996BA
:10B200000F94DA0C6AE0C8010F9405117C0197FDD8
:10B2100049C069ED7CE0CE0109960F94480DBE014E
:10B22000675F7F4FC8010F947D10882371F049E05C
:10B2300050E060E2C8010F94E9106C0181E0CE1487
:10B24000DF040CF080E0B82E01C0B12CCE010996CD
:10B250000F94DA0CBB20A9F096012F5F3F4F49E015
:10B2600050E0B801CE0109960F947311BE01675FDB
:10B270007F4F89E29DE20F943F0FCE0109960F9414
:10B28000DA0C2D813E81A7014F5F5F4FB801CE01DF
:10B2900009960F947311BE01675F7F4FC8010F9429
:10B2A000CC0DACCF80914F2D882361F06AE87FE010
:10B2B00083E496E40F94360B69E27DE283E496E43E
:10B2C0000F94880BC8010F94DA0C64960FB6F894AB
:10B2D000DEBF0FBECDBFDF91CF911F910F91FF90C9
:10B2E000EF90DF90CF90BF9008952F923F924F92B2
:10B2F0005F926F927F928F929F92AF92BF92CF9206
:10B30000DF92EF92FF920F931F93CF93DF93CDB70E
:10B31000DEB76A970FB6F894DEBF0FBECDBF8C01C3
:10B320004B0141E050E060E070E0CE0101965C012D
:10B330000E9400BF60E070E0CB010E941EDF7E8BA8
:10B340006D8BB401882777FD8095982F0E9473DF5D
:10B35000C8010F94D80D68E2C8010F94560F9FEFF3
:10B36000891A990A212C312C2101C401AA2797FDA1
:10B37000A095BA2F8F8B988FA98FBA8FED89FE89F0
:10B38000E815F9050CF48DC0CF88D88CE98CFA8CBF
:10B39000C20CD31CE41CF51CC701B6010E94D1D716
:10B3A000672B682B692B09F461C0C701B6010E94A5
:10B3B00073DF6B017C01DB01FB0101900020E9F7E9
:10B3C0003197E61BF70BE330F105ECF18C918036F9
:10B3D000D1F53F0191E0691A71086C0C7D1CF301F5
:10B3E0008081803681F567EA79E1C5010F94D80D37
:10B3F000D3011C92B6016F5F7F4FCE0109960F9467
:10B40000480D1A8A198AEDEAFEE0F88BEF87BC8AAC
:10B41000AB8AAE01475F5F4FBE01615F7F4F8EE435
:10B420009DE20E94E71FCE0109960F94DA0CC50138
:10B430000F94DD1289819A819A8789878D819E81F7
:10B440009C878B870BC0DA86C986FD01019000209E
:10B45000E9F73197EC19FD09FC87EB8741E0BE0164
:10B46000675F7F4FC8010E94604C09C0C701B601E9
:10B470000E941EDFAB01BC01C8010F94F80F8D893B
:10B480009E898816990624F46CE2C8010F94560F21
:10B490009FEF891A990AAFEF2A1A3A0A4A0A5A0AFA
:10B4A0006DCF69E2C8010F94560F80914F2D88230C
:10B4B00059F067E671E183E496E40F94690BB801F3
:10B4C00083E496E40F94880BC5010F94DA0C6A9616
:10B4D0000FB6F894DEBF0FBECDBFDF91CF911F91A5
:10B4E0000F91FF90EF90DF90CF90BF90AF909F9023
:10B4F0008F907F906F905F904F903F902F90089526
:10B50000CF92DF92EF92FF92CF93DF93CDB7DEB76A
:10B510002E970FB6F894DEBF0FBECDBF4FEB56E1AE
:10B5200063E682E00E947D528823E1F062E070E0F1
:10B5300080E090E00E94D1D7672B682B692B91F0B7
:10B540008091392D882391F067EA76E1CE0101964A
:10B550000F940A0FCE0101960E940BDACE010196DC
:10B560000F94DA0CC12CD12C76013BC041E050E0A5
:10B5700060E070E0CE0101960E9400BF62E070E0E2
:10B58000CE0101960E9475598D819E818536910567
:10B5900090F06DE876E1CE0109960F940A0FCE0186
:10B5A00009960E940BDACE0109960F94DA0CC12C91
:10B5B000D12C760112C0E980FA8061E070E080E071
:10B5C00090E00E941EDF27EA39E1A70180E00E9497
:10B5D000F144C12CD12C7601C394CE0101960F9475
:10B5E000DA0CC701B6012E960FB6F894DEBF0FBE77
:10B5F000CDBFDF91CF91FF90EF90DF90CF90089576
:10B60000CF92DF92EF92FF92CF93DF93CDB7DEB769
:10B610002E970FB6F894DEBF0FBECDBF4BE655E1B7
:10B6200063E681E00E947D528823E1F061E070E0F2
:10B6300080E090E00E94D1D7672B682B692B91F0B6
:10B640008091392D882391F063E575E1CE01019653
:10B650000F940A0FCE0101960E940BDACE010196DB
:10B660000F94DA0CC12CD12C760136C041E050E0A9
:10B6700060E070E0CE0101960E9400BF61E070E0E2
:10B68000CE0101960E9475598D819E818536910566
:10B6900090F069E375E1CE0109960F940A0FCE018F
:10B6A00009960E940BDACE0109960F94DA0CC12C90
:10B6B000D12C76010DC049815A8127EA39E161E038
:10B6C00070E080E00E94F144C12CD12C7601C3943B
:10B6D000CE0101960F94DA0CC701B6012E960FB673
:10B6E000F894DEBF0FBECDBFDF91CF91FF90EF90FA
:10B6F000DF90CF900895CF92DF92EF92FF92CF9399
:10B70000DF93CDB7DEB762970FB6F894DEBF0FBEFA
:10B71000CDBF46E954E163E683E00E947D52882371
:10B7200009F471C061E070E080E090E00E94D1D740
:10B73000672B682B692B09F466C063E070E080E03A
:10B7400090E00E94D1D7672B682B692B09F45BC06E
:10B750008091392D882379F06EE774E1CE0101964E
:10B760000F940A0FCE0101960E940BDACE010196CA
:10B770000F94DA0C48C041E050E060E070E0CE0188
:10B7800001960E9400BF63E070E0CE0101960E9426
:10B7900075598D819E818536910590F064E674E13E
:10B7A000CE0109960F940A0FCE0109960E940BDA7A
:10B7B000CE0109960F94DA0CC12CD12C76011EC053
:10B7C00061E070E080E090E00E941EDF9B01AC0130
:10B7D000E980FA8062E070E080E090E02F87388BAB
:10B7E000498B5A8B0E941EDF2F853889A70181E083
:10B7F0000E94F144C12CD12C7601C394CE01019654
:10B800000F94DA0C03C0C12CD12C7601C701B6010C
:10B8100062960FB6F894DEBF0FBECDBFDF91CF9119
:10B82000FF90EF90DF90CF900895CF92DF92EF924C
:10B83000FF92CF93DF93CDB7DEB72E970FB6F89474
:10B84000DEBF0FBECDBF4EE254E163E682E00E9450
:10B850007D528823E1F062E070E080E090E00E9499
:10B86000D1D7672B682B692B91F08091392D8823D4
:10B8700091F066E174E1CE0101960F940A0FCE01BA
:10B8800001960E940BDACE0101960F94DA0CC12CBE
:10B89000D12C76013BC041E050E060E070E0CE0189
:10B8A00001960E9400BF62E070E0CE0101960E9406
:10B8B00075598D819E818536910590F06CEF73E10D
:10B8C000CE0109960F940A0FCE0109960E940BDA59
:10B8D000CE0109960F94DA0CC12CD12C760112C03E
:10B8E000E980FA8061E070E080E090E00E941EDF75
:10B8F00027EA39E1A70181E00E94F144C12CD12C53
:10B900007601C394CE0101960F94DA0CC701B601FB
:10B910002E960FB6F894DEBF0FBECDBFDF91CF914C
:10B92000FF90EF90DF90CF900895BF92CF92DF927B
:10B93000EF92FF920F931F93CF93DF93CDB7DEB7B4
:10B940002E970FB6F894DEBF0FBECDBF60EE73E149
:10B9500081E00E94A94E882309F46CC00E9442F441
:10B960008C01E12CF12CF80181819281019609F47E
:10B9700052C061E070E080E090E00E9473DFCE0191
:10B9800009960F94480D41E050E060E870E0CE0168
:10B9900001960E9400BFBE01675F7F4FCE010196F6
:10B9A0000F943F0F68E2CE0101960F94560FF801F5
:10B9B000C380D480B68061817281CE0101960F94DC
:10B9C000C70F6CE2CE0101960F94560F6B2DCE017E
:10B9D00001960F946A0F6CE2CE0101960F94560FF8
:10B9E000B601CE0101960F94C70F69E2CE01019610
:10B9F0000F94560FAE014F5F5F4F60E070E08EE432
:10BA00009DE20E94E71FCE0101960F94DA0CCE0151
:10BA100009960F94DA0CFFEFEF1AFF0A095F1F4F28
:10BA200024E1E216F10409F09ECF61E070E080E0CD
:10BA300090E003C060E070E0CB012E960FB6F89462
:10BA4000DEBF0FBECDBFDF91CF911F910F91FF9051
:10BA5000EF90DF90CF90BF900895EF92FF920F93F9
:10BA60001F93CF93DF93CDB7DEB72E970FB6F89421
:10BA7000DEBF0FBECDBF8C0180914F2D882309F40E
:10BA80006BC0F801818981112CC063E476E183E405
:10BA900096E40F94360BF801658176814AE050E018
:10BAA00083E496E40F94AC0CF80182898823A1F01A
:10BAB00063E276E183E496E40F94360B4AE050E0CB
:10BAC000F801628983E496E40F948E0C61E276E1DA
:10BAD00083E496E40F94360B83E496E40F94720BA0
:10BAE0003BC069E176E183E496E40F94360BF801FC
:10BAF0008189813189F028F4823041F0803149F028
:10BB000011C0803261F0813221F00CC069E076E131
:10BB10000BC06BEE75E108C061ED75E105C06FEA21
:10BB200075E102C06DE975E183E496E40F94360B8C
:10BB30006BE975E183E496E40F94360B40E150E045
:10BB4000F801618983E496E40F948E0C69E975E14C
:10BB500083E496E40F94760BF801828990E0909349
:10BB6000522D8093512D868564857585680F711DD2
:10BB7000FB018081882309F442C0CE0109960F940D
:10BB8000480D41E050E060E870E0CE0101960E946F
:10BB900000BFBE01675F7F4FCE0101960F943F0F3C
:10BBA00068E2CE0101960F94560FE090512DF0906F
:10BBB000522DF8016189CE0101960F946A0F6CE253
:10BBC000CE0101960F94560FB701CE0101960F9446
:10BBD000960F69E2CE0101960F94560FAE014F5FAA
:10BBE0005F4F60E070E08EE49DE20E94E71FCE01AF
:10BBF00001960F94DA0CCE0109960F94DA0CF80135
:10BC0000848595850F94C719C8012E960FB6F894B0
:10BC1000DEBF0FBECDBFDF91CF911F910F91FF907F
:10BC2000EF900D94C719EF92FF920F931F93CF934C
:10BC3000DF9300D000D0CDB7DEB78B016115710561
:10BC400009F43FC080914F2D882359F065E77FE0CC
:10BC500083E496E40F94360BB80183E496E40F94E2
:10BC60009A0BC8010E94B2D681112DC0E12CF12C93
:10BC7000B801CE0101960F94480DA701BE016F5F78
:10BC80007F4F89E29DE20F9409117C01CE0101965C
:10BC90000F94DA0CF7FC15C0F80101900020E9F7C9
:10BCA000BF0161507109601B710B6E0D7F1D89E230
:10BCB0009DE20F94BD10803231F0FFEFEF1AFF0AC2
:10BCC000D7CF80E001C081E026960FB6F894DEBFA2
:10BCD0000FBECDBFDF91CF911F910F91FF90EF90DD
:10BCE0000895CF93DF9360E070E0CB010E941EDFE8
:10BCF000672B682B692B09F444C060E070E0CB012E
:10BD00000E941EDF6330710581059105D4F560E066
:10BD100070E0CB010E941EDF623071058105910544
:10BD20006CF162E070E080E090E00E94D1D7672B78
:10BD3000682B692B41F062E070E080E090E00E94A7
:10BD400073DFEB010AC062E070E080E090E00E94E7
:10BD50001EDFCB010E94AA90EC012097D1F0BE011A
:10BD60008EE49DE20E94135E811113C086EA91E188
:10BD70000E94CCD8CE010E94CCD807C0C0E0D0E051
:10BD800008C081E891E10E9407DA60E070E0CB0131
:10BD900011C061E070E080E090E00E941EDFAB0126
:10BDA000BC019E018DE79BE20E940C2661E070E0E1
:10BDB00080E090E0DF91CF910895CF93DF93CDB7EE
:10BDC000DEB728970FB6F894DEBF0FBECDBFCE0109
:10BDD00001960E94483FCE0101960F94DA0CCE01E5
:10BDE00001960E94A34CCE0101960F94DA0CCE016D
:10BDF00001960E943F3ACE0101960F94DA0CCE01D3
:10BE000001960E94C938CE0101960F94DA0CCE013A
:10BE100001960E94673CCE0101960F94DA0CCE0188
:10BE200001960E94203BCE0101960F94DA0CCE01C0
:10BE300001960E947846CE0101960F94DA0CCE014D
:10BE400001960E945C39CE0101960F94DA0CCE0166
:10BE500001960E94FD37CE0101960F94DA0C2896C8
:10BE60000FB6F894DEBF0FBECDBFDF91CF9108951E
:10BE7000CF93DF9300D000D0CDB7DEB763EA78E18F
:10BE8000CE0101960F940A0FCE0101960E940BDAA3
:10BE9000CE0101960F94DA0C8EE49DE20E94DD5EE5
:10BEA00061E070E080E090E026960FB6F894DEBF87
:10BEB0000FBECDBFDF91CF91089590ED980F9A30CE
:10BEC00088F09FE9980F9A3110F4875508959FEBF9
:10BED000980F9A3110F4875308958EE00E94BADBD0
:10BEE00080E00895892F08957F928F929F92AF925C
:10BEF000BF92CF92DF92EF92FF920F931F93CF9357
:10BF0000DF936C018B014A0160FF03C08EE00E9449
:10BF1000BADBC0E0D0E0C017D107D0F47E01F694C0
:10BF2000E794E80CF91C5601AC0EBD1EF5018081AA
:10BF30000E945D5F782EF50181810E945D5FF0E1D6
:10BF40007F9E90011124822BF70180832296E3CFFC
:10BF5000F601E00FF11F8081882381F08EE0DF91F0
:10BF6000CF911F910F91FF90EF90DF90CF90BF90F6
:10BF7000AF909F908F907F900C94BADBDF91CF9120
:10BF80001F910F91FF90EF90DF90CF90BF90AF90F7
:10BF90009F908F907F9008952F923F924F925F9243
:10BFA0006F927F928F929F92AF92BF92CF92DF92C9
:10BFB000EF92FF920F931F93CF93DF9300D000D0A7
:10BFC000CDB7DEB70DB71EB761E070E080E090E05E
:10BFD0000E941EDF6B017C0197FD0AC08091892DB4
:10BFE00090E0A0E0B0E0C816D906EA06FB061CF017
:10BFF0006BED7CE171C060E070E0CB010E941EDF60
:10C00000623071058105910559F462E070E080E0CD
:10C0100090E00E9473DFCB01212C312C21010FC055
:10C0200062E070E080E090E00E941EDF1B012C01C6
:10C0300063E070E080E090E00E9473DFCB01FC01E0
:10C0400001900020E9F7BF0161507109681B790B6D
:10C050003B01769467942DB73EB7261937090FB682
:10C06000F8943EBF0FBE2DBFEDB7FEB731964F011E
:10C07000AF010E94745F22E12C9DC0012D9D900DA7
:10C080001124A090872DB090882DA80EB91E60E0D5
:10C0900070E0C5010E94C381C5010E940F82C501E5
:10C0A0000E941B82262DA401B101F5018085918596
:10C0B0000E94C87C009719F463EC7CE10DC0F50187
:10C0C00091878087AC016C2D8BE79DE20E94EF7B0E
:10C0D000811112C06CEA7CE1CE0101960F940A0F27
:10C0E000CE0101960E940BDACE0101960F94DA0C74
:10C0F00060E070E0CB0104C061E070E080E090E0BF
:10C100000FB6F8941EBF0FBE0DBF26960FB6F8945B
:10C11000DEBF0FBECDBFDF91CF911F910F91FF907A
:10C12000EF90DF90CF90BF90AF909F908F907F90D7
:10C130006F905F904F903F902F900895CF93DF9333
:10C1400000D0CDB7DEB769E079E181E00E94A94E69
:10C15000882389F161E070E080E090E00E94D1D70F
:10C16000672B682B692B41F061E070E080E090E084
:10C170000E941EDFCB0109C061E070E080E090E02A
:10C180000E941EDFCB010E94AA90AE014F5F5F4F5D
:10C1900066E070E00E94745F2B8130E04A8150E0DD
:10C1A000698170E088EE90E30E944CBC61E070E031
:10C1B00080E090E003C060E070E0CB010F900F9052
:10C1C0000F90DF91CF91089562E77FE083E496E4DA
:10C1D0000F94360B6091212D7091222D83E496E40B
:10C1E0000F94690B60E070E081E29DE20D94D80D40
:10C1F000FC018081882321F081E29DE20D94460FAD
:10C2000083E496E40D94690BAF92BF92CF92DF92D4
:10C21000EF92FF920F931F93CF93DF936A017B01FD
:10C220005901F90101900020E9F78F01015011092E
:10C23000021B130BC8010F960F942F19EC018EE00F
:10C24000FE0111928A95E9F7A8014F5F5F4FB50192
:10C25000CE010E960F94231E1B861A8685E99BE657
:10C260009D878C87CE82DF82E886F986CE01DF91BA
:10C27000CF911F910F91FF90EF90DF90CF90BF90E3
:10C28000AF900D94BE004F925F926F927F928F920B
:10C290009F92AF92BF92CF92DF92EF92FF92CF9395
:10C2A000DF9360E070E0CB010E941EDFEB0120977E
:10C2B00061F061707727672B41F4C12CD12C760196
:10C2C000C394812C912C540130C085EC91E10E94E3
:10C2D00007DA60E070E0CB0139C0260137018FEF4B
:10C2E000481A580A680A780AC301B2010E94D1D7D5
:10C2F000672B682B692BE9F0C301B2010E941EDF96
:10C300003B01C701B6010E941EDF860E971EA81EC4
:10C31000B91E9301B501A4018EE49DE20E9404615F
:10C3200082E0C80ED11CE11CF11CCC16DD06ACF27B
:10C3300009C0C301B2010E941EDFCB010E94AA9076
:10C340003C01DFCF61E070E080E090E0DF91CF91D1
:10C35000FF90EF90DF90CF90BF90AF909F908F9025
:10C360007F906F905F904F900895AF92BF92CF9261
:10C37000DF92EF92FF920F931F93CF93DF935C01B5
:10C380006A017B018901C9010F94F11D01960F9487
:10C390002F19EC01B8010F94CB1D9E01B701A60126
:10C3A000C5010E940461CE01DF91CF911F910F91D1
:10C3B000FF90EF90DF90CF90BF90AF900D94C71992
:10C3C000CF92DF92EF92FF92CF93DF93CDB7DEB79C
:10C3D0002E970FB6F894DEBF0FBECDBF4EE055E1ED
:10C3E00063E681E00E947D528823E1F061E070E025
:10C3F00080E090E00E94D1D7672B682B692B91F0E9
:10C400008091392D882391F066EF74E1CE01019679
:10C410000F940A0FCE0101960E940BDACE0101960D
:10C420000F94DA0CC12CD12C760140C041E050E0D1
:10C4300060E070E0CE0101960E9400BF61E070E014
:10C44000CE0101960E9475598D819E818536910598
:10C4500090F06CED74E1CE0109960F940A0FCE01B5
:10C4600009960E940BDACE0109960F94DA0CC12CC2
:10C47000D12C760117C049815A8127EA39E161E060
:10C4800070E080E00E94F14429813A8144E650E066
:10C4900060E070E08EE49DE20E940461C12CD12C2A
:10C4A0007601C394CE0101960F94DA0CC701B60150
:10C4B0002E960FB6F894DEBF0FBECDBFDF91CF91A1
:10C4C000FF90EF90DF90CF900895CF93DF93CDB79B
:10C4D000DEB74885598560E070E08E819F810E94BB
:10C4E000E71FDF91CF9108954F925F926F927F92F5
:10C4F0008F929F92AF92BF92CF92DF92EF92FF9274
:10C500000F931F93CF93DF93CDB7DEB7CA55D109F1
:10C510000FB6F894DEBF0FBECDBF8C01FC01E780E3
:10C52000F08480914D2D8823F1F169E272E283E479
:10C5300096E40F94360BB70183E496E40F94690BED
:10C5400062E272E283E496E40F94360BF8016081B4
:10C5500071814AE050E083E496E40F94AC0C6CE106
:10C5600072E283E496E40F94360B4AE050E0F8015F
:10C57000628583E496E40F948E0C65E172E283E4B5
:10C5800096E40F94360BF8016385772767FD709565
:10C5900077FF03C07195619571094AE050E083E42B
:10C5A00096E40F94570CF8012385332727FD309527
:10C5B00037FF03C03195219531092093512D3093D8
:10C5C000522DF801828590E09093542D8093532D45
:10C5D000808191819093562D8093552D822F0E94BA
:10C5E0006FF8F70101900020E9F73197EE19FF0984
:10C5F000339708F4BFC0F70180818B3509F0BAC0CA
:10C600000F9406059B01AC01BE016F5B7F4FC70114
:10C610000E9406910F9406056B017C016BEE71E19F
:10C62000CE0101965C010F94591EB5018EE49DE286
:10C630000E94135E882309F47EC0F80181818F93E4
:10C6400080818F938CEF91E19F938F931F9280E471
:10C650008F93BF92AF920F94351F01E410E00C0F3F
:10C660001D1F0C5F1F4F0FB6F894DEBF0FBECDBF6E
:10C6700092E0492E512C25E2822E2AE2922E30E4BD
:10C68000632E712C23968EAD9FAD2397841595054F
:10C6900024F1F801808191810E5F1F4FF501019017
:10C6A0000020E9F73197EA19FB099F938F939F9236
:10C6B0008F92C3018E1B9F0B9F938F93EA0DFB1DDF
:10C6C000FF93EF930F94351FFFEF4F1A5F0A0FB6DA
:10C6D000F894DEBF0FBECDBFD5CFF501019000208D
:10C6E000E9F73197EA19FB0989EE91E19F938F935E
:10C6F00080E490E08E1B9F0B9F938F93EA0DFB1DB0
:10C70000FF93EF930F94351F8E010B5A1F4FB50106
:10C71000C8010F94480D1F930F938EE49DE29F93E1
:10C720008F930E946562C8010F94DA0C0FB6F894DB
:10C73000DEBF0FBECDBF1091032C1123E9F060EFD7
:10C7400071E283E496E40F94360B0F940605AB0177
:10C75000BC014C195D096E097F092AE030E083E4D1
:10C7600096E40F94810C6DEE71E283E496E40F94ED
:10C77000760B03C010E001C011E0812FC65ADF4FD5
:10C780000FB6F894DEBF0FBECDBFDF91CF911F91E2
:10C790000F91FF90EF90DF90CF90BF90AF909F9060
:10C7A0008F907F906F905F904F900895AF92BF925F
:10C7B000CF92DF92EF92FF920F931F93CF93DF936D
:10C7C000CDB7DEB7A2970FB6F894DEBF0FBECDBFD0
:10C7D000B82EA62E8091042C811166C00F940605F8
:10C7E0006B017C018E010F5F1F4FC8010E945C39F5
:10C7F000C8010F94DA0C60E172E18EE49DE20E94C0
:10C80000135E882399F12A2D332727FD30953F9316
:10C81000AF922B2D332727FD30953F93BF9280E1B8
:10C8200092E19F938F938FE192E19F938F931F9259
:10C830008CE18F931F930F930F94351F5E018DE151
:10C84000A80EB11CB801C5010F94480DBF92AF925C
:10C850008EE49DE29F938F930E946562C5010F94C1
:10C86000DA0C0FB6F894DEBF0FBECDBF8091032C5B
:10C870008823D1F06AEC71E283E496E40F94360BDE
:10C880000F940605AB01BC014C195D096E097F09C7
:10C890002AE030E083E496E40F94810C67EC71E2C7
:10C8A00083E496E40F94760BA2960FB6F894DEBF5D
:10C8B0000FBECDBFDF91CF911F910F91FF90EF90F1
:10C8C000DF90CF90BF90AF900895AF92BF92CF927C
:10C8D000DF92EF92FF920F931F93CF93DF93CDB729
:10C8E000DEB7A2970FB6F894DEBF0FBECDBFB82E4D
:10C8F0008091042C81115CC00F9406056B017C01B2
:10C900008E010F5F1F4FC8010E943F3AC8010F946C
:10C91000DA0C6AE272E18EE49DE20E94135E8823E3
:10C9200049F11F92BF928AE292E19F938F938EE327
:10C9300092E19F938F931F928CE18F931F930F939C
:10C940000F94351F5E018DE1A80EB11CB801C50121
:10C950000F94480DBF92AF928EE49DE29F938F9308
:10C960000E946562C5010F94DA0C0FB6F894DEBF21
:10C970000FBECDBF8091032C8823D1F06FE971E207
:10C9800083E496E40F94360B0F940605AB01BC01CB
:10C990004C195D096E097F092AE030E083E496E4D2
:10C9A0000F94810C6CE971E283E496E40F94760BAA
:10C9B000A2960FB6F894DEBF0FBECDBFDF91CF9128
:10C9C0001F910F91FF90EF90DF90CF90BF90AF90AD
:10C9D0000895AF92BF92CF92DF92EF92FF920F93A2
:10C9E0001F93CF93DF93CDB7DEB76E970FB6F89452
:10C9F000DEBF0FBECDBFB82E8091042C81115CC06C
:10CA00000F9406056B017C018E010F5F1F4FC8015B
:10CA10000E943F3AC8010F94DA0C65E472E18EE49B
:10CA20009DE20E94135E882349F11F92BF9285E424
:10CA300092E19F938F938EE392E19F938F931F9246
:10CA400088E18F931F930F930F94351F5E0189E147
:10CA5000A80EB11CB801C5010F94480DBF92AF924A
:10CA60008EE49DE29F938F930E946562C5010F94AF
:10CA7000DA0C0FB6F894DEBF0FBECDBF8091032C49
:10CA80008823D1F067E771E283E496E40F94360BD4
:10CA90000F940605AB01BC014C195D096E097F09B5
:10CAA0002AE030E083E496E40F94810C64E771E2BD
:10CAB00083E496E40F94760B6E960FB6F894DEBF7F
:10CAC0000FBECDBFDF91CF911F910F91FF90EF90DF
:10CAD000DF90CF90BF90AF9008958F929F92AF92CA
:10CAE000BF92CF92DF92EF92FF920F931F93CF935B
:10CAF000DF93CDB7DEB767970FB6F894DEBF0FBEF2
:10CB0000CDBFB82E962E872E8091042C811173C034
:10CB10004F8B0F9406056B017C018E010F5F1F4F39
:10CB2000C8010E94203BC8010F94DA0C1F92BF92EB
:10CB300026E532E13F932F931F9240E1A42EAF925E
:10CB40001F930F930F94351FB8018EE49DE20E944E
:10CB5000135E0FB6F894DEBF0FBECDBF4F8988239A
:10CB600061F1242F332727FD30953F934F938F9208
:10CB70009F921F92BF928DE592E19F938F931F9298
:10CB8000AF921F930F930F94351F5E0131E1A30EF7
:10CB9000B11CB801C5010F94480DBF92AF928EE44D
:10CBA0009DE29F938F930E946562C5010F94DA0CFA
:10CBB0000FB6F894DEBF0FBECDBF8091032C882343
:10CBC000D1F064E571E283E496E40F94360B0F94A0
:10CBD0000605AB01BC014C195D096E097F092AE00D
:10CBE00030E083E496E40F94810C61E571E283E424
:10CBF00096E40F94760B67960FB6F894DEBF0FBEDF
:10CC0000CDBFDF91CF911F910F91FF90EF90DF90FB
:10CC1000CF90BF90AF909F908F9008956F927F922A
:10CC20008F929F92AF92BF92CF92DF92EF92FF923C
:10CC30000F931F93CF93DF93CDB7DEB766970FB6F1
:10CC4000F894DEBF0FBECDBF782E4B01642E8091CD
:10CC5000042C8111ABC00F9406056B017C018E0181
:10CC60000F5F1F4FC8010E94673CC8010F94DA0C88
:10CC70001F927F928CE692E19F938F931F9250E1D7
:10CC8000B52EBF921F930F930F94351FB8018EE4FA
:10CC90009DE20E94135E0FB6F894DEBF0FBECDBFBB
:10CCA000882361F1862D992787FD90959F936F9238
:10CCB0009F928F921F927F9223E732E13F932F93AF
:10CCC0001F92BF921F930F930F94351F5E0131E1A6
:10CCD000A30EB11CB801C5010F94480DBF92AF92CD
:10CCE0002EE43DE23F932F930E946562C5010F94AD
:10CCF000DA0C0FB6F894DEBF0FBECDBF862D8D7F48
:10CD0000B9F5892829F41F927F9281E892E104C045
:10CD10001F927F928CE892E19F938F931F9280E104
:10CD20008F931F930F930F94351F0FB6F894DEBFA8
:10CD30000FBECDBFB8018EE49DE20E94135E882332
:10CD4000B9F05E0191E1A90EB11CB801C5010F94C3
:10CD5000480DBF92AF928EE49DE29F938F930E9405
:10CD60006562C5010F94DA0C0F900F900F900F9031
:10CD70008091032C8823D1F060E371E283E496E490
:10CD80000F94360B0F940605AB01BC014C195D09DD
:10CD90006E097F092AE030E083E496E40F94810C69
:10CDA0006DE271E283E496E40F94760B66960FB61B
:10CDB000F894DEBF0FBECDBFDF91CF911F910F91D1
:10CDC000FF90EF90DF90CF90BF90AF909F908F90AB
:10CDD0007F906F900895EF92FF920F931F93CF93E0
:10CDE000DF93CDB7DEB7E0970FB6F894DEBF0FBE86
:10CDF000CDBF6FE071E282E00E94A94E882351F01E
:10CE000061E070E080E090E00E94D1D7672B682B52
:10CE1000692B21F460E070E0CB0140C061E070E07C
:10CE200080E090E00E9473DF162F072F62E070E031
:10CE300080E090E00E941EDFCB010E94AA909F93A9
:10CE40008F930F931F930F931F9388E992E19F9302
:10CE50008F931F928AE28F93CE0101967C01FF92FD
:10CE60008F930F94351F8E01055D1F4FB701C801C9
:10CE70000F94480D1F930F938EE49DE29F938F9321
:10CE80000E946562C8010F94DA0C0FB6F894DEBFF9
:10CE90000FBECDBF61E070E080E090E0E0960FB69D
:10CEA000F894DEBF0FBECDBFDF91CF911F910F91E0
:10CEB000FF90EF900895CF92DF92EF92FF920F9341
:10CEC0001F93CF93DF93CDB7DEB72E970FB6F894AD
:10CED000DEBF0FBECDBF60E070E0CB010E941EDF61
:10CEE000613071058105910509F04DC061E070E088
:10CEF00080E090E00E941EDF672B682B692B09F40D
:10CF000042C0C090122CD090132CE090142CF090C2
:10CF1000152C0E94AE2D288739874A875B87888524
:10CF20009985AA85BB858093122C9093132CA0938E
:10CF3000142CB093152C61E070E080E090E00E942A
:10CF40001EDF623071058105910509F450C0C114DE
:10CF5000D104E104F10409F44AC08091122C9091AB
:10CF6000132CA091142CB091152C8C199D09AE098D
:10CF7000BF09CD97A105B105D0F567EA79E181E355
:10CF80009DE20F94D80D8091122C9091132CA091BA
:10CF9000142CB091152C892B8A2B8B2B19F10E9404
:10CFA000AE2D29833A834B835C8349815A816B81FF
:10CFB0007C818091122C9091132CA091142CB09113
:10CFC000152C481B590B6A0B7B0B31E020E080E0ED
:10CFD00090E04C3351056105710508F030E0632F96
:10CFE000722F38C060E070E080E090E033C08EE4E3
:10CFF0009DE20E94DD5E69EB72E18EE49DE20E949B
:10D00000135E8823B9F06DE970E28E010F5F1F4F48
:10D01000C8010F940A0F1F930F938EE49DE29F9314
:10D020008F930E946562C8010F94DA0C0F900F90E5
:10D030000F900F908091352D9091362D892B09F40A
:10D040009CCF41E35DE26FEE7EEB81E19CE20E94CA
:10D05000EF3093CF2E960FB6F894DEBF0FBECDBF44
:10D06000DF91CF911F910F91FF90EF90DF90CF90C4
:10D070000895CF92DF92EF92FF920F931F93CF9379
:10D08000DF93CDB7DEB760970FB6F894DEBF0FBE63
:10D09000CDBF8DE79BE20E948C228E010F5F1F4F58
:10D0A00081110FC063E87FE1C8010F940A0FC80126
:10D0B0000E940BDAC8010F94DA0C60E070E0CB013B
:10D0C000C0C064E67FE1C8010F940A0FC8010E9446
:10D0D0000BDAC8010F94DA0C7E0129E0E20EF11C94
:10D0E00041E050E064E670E0C7010E9400BF40E00C
:10D0F00050E0BA0186EC92E10E945990D82EC92ED8
:10D1000040E050E0BA0188EB98E10E945990CF923C
:10D11000DF929F938F938BEC92E19F938F93FF927B
:10D12000EF920E9426BFA70161E17CE2C8010E9444
:10D130008232C8010F94DA0C80919D2D90919E2D22
:10D140000FB6F894DEBF0FBECDBF009709F041C007
:10D150008DE79BE20E94561F24E140E050E060E032
:10D1600070E08DE79BE20E94FA1D8DE79BE20E9432
:10D17000971D20E030E04FEF50E060E070E088EE77
:10D1800090E30E94C2BB6DED72E1C8010F94480D9F
:10D190001F930F936EE4C62E6DE2D62EDF92CF92D0
:10D1A0000E946562C8010F94DA0C62EE72E1C80158
:10D1B0000F94480D1F930F93DF92CF920E946562E8
:10D1C000C8010F94DA0C0FB6F894DEBF0FBECDBFC6
:10D1D00031C04DEE52E163E476E40E94D1888111C2
:10D1E0000DC061E47FE1C8010F940A0FC8010E94DD
:10D1F000D8D8C8010F94DA0CD12C02C0DD24D39406
:10D2000042EF52E163E476E480919D2D90919E2D52
:10D210000E94D18881110CC06EE17FE1C8010F949A
:10D220000A0FC8010E94D8D8C8010F94DA0C02C0B6
:10D23000D1108ECFC7010F94DA0C61E070E080E06E
:10D2400090E060960FB6F894DEBF0FBECDBFDF91C1
:10D25000CF911F910F91FF90EF90DF90CF900895A5
:10D260000F931F93CF93DF93CDB7DEB72E970FB6F3
:10D27000F894DEBF0FBECDBF40E95BE163E082E022
:10D280000E947D52882309F482C00E94904B182F7F
:10D2900062E070E080E090E00E941EDF062F862FA3
:10D2A0000E94C14B672B682B692B09F470C041E0C9
:10D2B00050E060E870E0CE0101960E9400BF68EF88
:10D2C00072E1CE0101960F94460F612F8DE79BE22C
:10D2D0000E949523BC01CE0101960F942A106AE0AA
:10D2E00073E1CE0101960F94460F612F8DE79BE20B
:10D2F0000E949523BC01CE0101960F942A106BE188
:10D3000073E1CE0101960F94460F602F8DE79BE2EB
:10D310000E94A123BC01CE0101960F942A106FE157
:10D3200073E1CE0101960F94460F60E070E0CB01EF
:10D330000E941EDF633071058105910511F40130F3
:10D3400051F162E273E1CE0101960F94460F6981BB
:10D350007A818E01075F1F4FC8010F94480D1F93FC
:10D360000F938EE49DE29F938F930E946562C801A4
:10D370000F94DA0CCE0101960F94DA0C0F900F90F7
:10D380000F900F9061E070E080E090E033C060E0CB
:10D3900070E0CB012FC063E070E080E090E00E947D
:10D3A0001EDF062F462F612F8DE79BE20E94C525C9
:10D3B00065E273E1CE0101960F94460F612F8DE770
:10D3C0009BE20E949523BC01CE0101960F942A1086
:10D3D0006BE173E1CE0101960F94460F602FCE01F1
:10D3E00001960F946A0F6FE173E1CE0101960F94DD
:10D3F000460FA7CF2E960FB6F894DEBF0FBECDBF57
:10D40000DF91CF911F910F910895AF92BF92CF926C
:10D41000DF92EF92FF920F931F93CF93DF93CDB7DD
:10D42000DEB7A6970FB6F894DEBF0FBECDBF8C0156
:10D430001092392DFC01848595850F94C719809130
:10D440004D2D882309F46BC0F801818981112CC00E
:10D4500068EC77E183E496E40F94360BF80165817C
:10D4600076814AE050E083E496E40F94AC0CF80136
:10D4700082898823A1F068EA77E183E496E40F9437
:10D48000360B4AE050E0F801628983E496E40F9499
:10D490008E0C66EA77E183E496E40F94360B83E41E
:10D4A00096E40F94720B3BC06EE977E183E496E457
:10D4B0000F94360BF8018189813189F028F482308C
:10D4C00041F0803149F011C0803261F0813221F0A9
:10D4D0000CC06EE877E10BC060E777E108C066E555
:10D4E00077E105C064E377E102C062E277E183E4BB
:10D4F00096E40F94360B60E277E183E496E40F94B0
:10D50000360B40E150E0F801618983E496E40F9422
:10D510008E0C6EE177E183E496E40F94760BF801CC
:10D52000828990E09093522D8093512D0F9406059F
:10D530006B017C0164E373E1CE0101965C010F9401
:10D54000591EB5018EE49DE20E94135E882391F17D
:10D55000F8018189811103C0828990E002C080E0D6
:10D5600090E09F938F93F80186818F9385818F93AD
:10D5700086E493E19F938F931F9280E28F93BF92F3
:10D58000AF920F94351F8E010F5D1F4FB501C8017B
:10D590000F94480D1F930F938EE49DE29F938F93FA
:10D5A0000E946562C8010F94DA0C0FB6F894DEBFD2
:10D5B0000FBECDBF8091032C8823D1F068EF76E1B8
:10D5C00083E496E40F94360B0F940605AB01BC017F
:10D5D0004C195D096E097F092AE030E083E496E486
:10D5E0000F94810C65EF76E183E496E40F94760B5B
:10D5F000A6960FB6F894DEBF0FBECDBFDF91CF91D8
:10D600001F910F91FF90EF90DF90CF90BF90AF9060
:10D610000895EF92FF920F931F93CF93DF9300D063
:10D6200000D0CDB7DEB761EC73E181E00E94A94E76
:10D63000882309F46AC060E973E18E010F5F1F4F10
:10D64000C8010F940A0F1F930F937EE4E72E7DE22B
:10D65000F72EFF92EF920E946562C8010F94DA0CD8
:10D660006AE173E1C8010F940A0F1F930F93FF92B1
:10D67000EF920E946562C8010F94DA0C68EC72E1C7
:10D68000C8010F940A0F1F930F93FF92EF920E940D
:10D690006562C8010F94DA0C64E972E1C8010F9465
:10D6A0000A0F1F930F93FF92EF920E946562C801C9
:10D6B0000F94DA0C6FE772E1C8010F940A0F1F9301
:10D6C0000F93FF92EF920E946562C8010F94DA0CEB
:10D6D00061E070E080E090E00E941EDF9B01AC0101
:10D6E000A8EEB3E00F94CF17AB01BC0128E432E100
:10D6F000C7010E94B5610FB6F894DEBF0FBECDBF63
:10D7000061E070E080E090E003C060E070E0CB0199
:10D7100026960FB6F894DEBF0FBECDBFDF91CF9136
:10D720001F910F91FF90EF900895EF92FF920F934A
:10D730001F93CF93DF9300D000D0CDB7DEB77C012D
:10D7400080914F2D8701025F1F4F882359F06DECA8
:10D750007EE083E496E40F94360BB80183E496E40C
:10D760000F949A0BB8018E010F5F1F4FC8010F94E1
:10D77000480D1F930F938EE49DE29F938F930E9419
:10D780006562C8010F94DA0C0F900F900F900F9004
:10D79000C70126960FB6F894DEBF0FBECDBFDF914E
:10D7A000CF911F910F91FF90EF900D94C7197F9229
:10D7B0008F929F92AF92BF92CF92DF92EF92FF92A1
:10D7C0000F931F93CF93DF93CDB7DEB7A6970FB616
:10D7D000F894DEBF0FBECDBF6C0181E0F6018187FA
:10D7E0000E94AEE20E941EE08EE49DE20E94C558B7
:10D7F0006DE57FE08E010F5F1F4FC8010F940A0F88
:10D80000C8010E940BDAC8010F94DA0C6CE27FE0C9
:10D81000C8010F940A0FC8010E940BDAC8010F94C7
:10D82000DA0C6AE27FE0C8010F940A0FC8010E9477
:10D83000D8D8C8010F94DA0C8DE79BE20E94A91F8B
:10D840000E94CCD86CE17FE0C8010F940A0FC80198
:10D850000E94D8D8C8010F94DA0C8DE79BE20E9491
:10D86000AD1F0E94CCD86AE17FE0C8010F940A0F77
:10D87000C8010E940BDAC8010F94DA0C68E17FE05E
:10D88000C8010F940A0FC8010E94D8D8C8010F948C
:10D89000DA0C0E949BD60E947BD96CE07FE0C80125
:10D8A0000F940A0FC8010E940BDAC8010F94DA0C1A
:10D8B0008DE79BE20E948022882319F06AEF7EE0C8
:10D8C00002C067EE7EE0C8010F940A0FC8010E94F3
:10D8D0000BDAC8010F94DA0C1F921F9280E693E1D5
:10D8E0009F938F931F9280E28F931F930F930F94B8
:10D8F000351FB8018EE49DE20E94135E0FB6F894C6
:10D90000DEBF0FBECDBF8823B9F07E0131E2E30E4A
:10D91000F11CB801C7010F94480DFF92EF928EE4FD
:10D920009DE29F938F930E946562C7010F94DA0C6A
:10D930000F900F900F900F90E1E6EE2EF12CF8E68D
:10D940008F2EF3E19F2EA0E27A2E5E0181E2A80ED7
:10D95000B11CFF92EF929F928F921F927F921F9322
:10D960000F930F94351FB8018EE49DE20E94135E61
:10D970000FB6F894DEBF0FBECDBF882399F0B80173
:10D98000C5010F94480DBF92AF928EE49DE29F9324
:10D990008F930E946562C5010F94DA0C0F900F906F
:10D9A0000F900F90FFEFEF1AFF0A2AE7E216F1043B
:10D9B00081F6B12C7E0131E2E30EF11C40E250E031
:10D9C00061E073E1C8010F94601E6B2D8DE79BE24F
:10D9D0000E94952340E250E0BC01C8010F94D21D83
:10D9E000B8018EE49DE20E94135E882399F0B8018D
:10D9F000C7010F94480DFF92EF928EE49DE29F9332
:10DA00008F930E946562C7010F94DA0C0F900F90FC
:10DA10000F900F90B39480E2B812D0CFC6010E944D
:10DA2000E460A6960FB6F894DEBF0FBECDBFDF91BF
:10DA3000CF911F910F91FF90EF90DF90CF90BF900B
:10DA4000AF909F908F907F900895CF93DF93EC01DC
:10DA50000E94949162E27AE383E793E10E94BFDF40
:10DA60006BED77E484E893E10E94BFDF65E37AE33E
:10DA700085E993E10E94BFDF6BE27AE383EA93E1F9
:10DA80000E94BFDF60E176E581EB93E10E94BFDF9A
:10DA900062ED77E48DEB93E10E94BFDF69EC77E400
:10DAA0008DEC93E10E94BFDF69E17AE38EED93E1B3
:10DAB0000E94BFDF61E77EE581EF93E10E94BFDF57
:10DAC0006DEF7AE38DEF93E10E94BFDF60E474E5D0
:10DAD0008AE094E10E94BFDF69ED73E78BE194E196
:10DAE0000E94BFDF63E672E587E294E10E94BFDF38
:10DAF00069E472E587E394E10E94BFDF6FE272E5BB
:10DB000085E494E10E94BFDF6BED71E586E594E169
:10DB10000E94BFDF6DE977E482E694E10E94BFDFF7
:10DB200066E37FE38EE694E10E94BFDF61EC71E57E
:10DB30008CE794E10E94BFDF67EA71E58BE894E12E
:10DB40000E94BFDF6DE871E58BE994E10E94BFDFC1
:10DB50006FE671E588EA94E10E94BFDF6AE777E447
:10DB600085EB94E10E94BFDF6FE875E481EC94E1FE
:10DB70000E94BFDF61EF76E38EEC94E10E94BFDF8D
:10DB80006DEF76E38AED94E10E94BFDF66E077E314
:10DB900084EE94E10E94BFDF60E776E48EEE94E1CC
:10DBA0000E94BFDF69E07BE686EF94E10E94BFDF61
:10DBB00065E97CE585E095E10E94BFDF65E17CE5F4
:10DBC0008FE095E10E94BFDF6BE77BE58DE195E19A
:10DBD0000E94BFDF60EE71E68FE295E10E94BFDF39
:10DBE00060E07BE58BE395E10E94BFDF60E87AE5CA
:10DBF0008AE495E10E94BFDF6BE378E58EEE91E168
:10DC00000E94BFDF61E078E584ED9DE00E94BFDF08
:10DC100061E579E388E595E10E94BFDF66E479E399
:10DC200086E695E10E94BFDF66EF79E384E795E140
:10DC30000E94BFDF65E571E587E895E10E94BFDFDF
:10DC400064E271E58DE995E10E94BFDF62E574E46D
:10DC500083EB95E10E94BFDF69E574E480EC95E118
:10DC60000E94BFDF68E37FE58AE497E10E94BFDF9F
:10DC70006DE57EE38DEA94E10E94BFDF6EE577E318
:10DC80008EEC95E10E94BFDF60E27EE48AED95E1D3
:10DC90000E94BFDF63E07EE48EEE95E10E94BFDF6D
:10DCA0006EED76E383E096E10E94BFDF68EE76E3F7
:10DCB0008AE196E10E94BFDF66E87CE482E396E1B8
:10DCC0000E94BFDF68E67CE481E496E10E94BFDF4A
:10DCD00060E87DE48FE496E10E94BFDF6BEF73E4C0
:10DCE0008DE596E10E94BFDF6EE37EE481E796E179
:10DCF0000E94BFDF6EE37EE48FED90E10E94BFDF04
:10DD00006EE07BE48FE796E10E94BFDF62EF73E491
:10DD100086E896E10E94BFDF69EC7AE48EE896E13E
:10DD20000E94BFDF64E87AE486E996E10E94BFDFE3
:10DD30006FE37AE480EA96E10E94BFDF6AEF79E45C
:10DD400089EA96E10E94BFDF65EB79E482EB96E118
:10DD50000E94BFDF60E779E48DEB96E10E94BFDFB0
:10DD60006BE279E48DEC96E10E94BFDF66EE78E429
:10DD700089ED96E10E94BFDF61EA78E484EE96E1E6
:10DD80000E94BFDF6CE578E48FEE96E10E94BFDF72
:10DD90006EE07BE489EF96E10E94BFDF63E773E505
:10DDA00083E097E10E94BFDF6EE970E68DE097E1C6
:10DDB0000E94BFDF66E97DE388E197E10E94BFDF53
:10DDC0006FED70E583E297E10E94BFDF69EE73E4D7
:10DDD0008EE297E10E94BFDF6AE970E588E397E190
:10DDE0000E94BFDF66EA78E386E497E10E94BFDF26
:10DDF0006FE077E383E992E10E94BFDF64E177E3BC
:10DE000088E892E10E94BFDF68E177E388E997E163
:10DE10000E94BFDF6DE177E381E597E10E94BFDFFC
:10DE200061E277E38FE697E10E94BFDF65E277E387
:10DE30008DE797E10E94BFDF6AE277E38AE597E129
:10DE40000E94BFDF6FE277E38CE894E20E94BFDFBD
:10DE50006EE473E587E697E10E94BFDF6CE870E54A
:10DE600085E797E10E94BFDF6EE770E584E897E100
:10DE70000E94BFDF60E770E580E997E10E94BFDFA5
:10DE800062E670E585EA97E10E94BFDF6EE470E527
:10DE900081EB97E10E94BFDF69E170E58DEB97E1CF
:10DEA0000E94BFDF68EA7FE486EC97E10E94BFDF53
:10DEB00060E379E680ED97E10E94BFDF68EA72E4F3
:10DEC00089ED97E10E94BFDF64E97FE484EE97E18A
:10DED0000E94BFDF6EE373E58FEE97E10E94BFDF24
:10DEE00063E77DE386E098E10E94BFDF64E47CE3C2
:10DEF00089E198E10E94BFDF63E279E38BE298E178
:10DF00000E94BFDF68EB70E48BE398E10E94BFDF03
:10DF100064EE77E489E498E10E94BFDF6CEC7FE572
:10DF200089E598E10E94BFDF69E471E480E798E148
:10DF30000E94BFDF63EB70E780E898E10E94BFDFDB
:10DF400060E670E483E998E10E94BFDF6FE37FE35E
:10DF500080EA98E10E94BFDF63E471E68BEE9CE00B
:10DF60000E94BFDF69E378E682EB98E10E94BFDFA1
:10DF700061E37FE382EE92E10E94BFDF68E27FE32C
:10DF80008EEB98E10E94BFDF67E477E38CEC98E1C9
:10DF90000E94BFDF69EC7EE38BED98E10E94BFDF5A
:10DFA00062E57FE489EE98E10E94BFDF68E37FE4E9
:10DFB00087EF98E10E94BFDF6DE97EE383E099E19E
:10DFC0000E94BFDF67E47EE38FE099E10E94BFDF3C
:10DFD0006CEC77E58AE199E10E94BFDF6DEF76E5B1
:10DFE00083E299E10E94BFDF63E57BE48DE299E182
:10DFF0000E94BFDF60EB74E587E399E10E94BFDF19
:10E000006BE577E68CEB92E10E94BFDF64E37EE391
:10E0100085E499E10E94BFDF60E27EE382E599E159
:10E020000E94BFDF69EE7DE38EE599E10E94BFDFCC
:10E0300064E377E38EE699E10E94BFDF6BEC72E563
:10E040008AE694E10E94BFDF6FE17FE48DE799E10A
:10E050000E94BFDF62E07FE486E899E10E94BFDFB3
:10E0600064EE7EE480E999E10E94BFDF6BEE76E624
:10E070008BE999E10E94BFDF8EE096E69093902BAA
:10E0800080938F2B8DE695E69093922B8093912B26
:10E0900089EE94E69093942B8093932B85E694E6F7
:10E0A0009093962B8093952B86ED93E690939A2BE5
:10E0B0008093992B81E79BE49093E9308093E8303B
:10E0C0008985882319F0CE010E94D76B44E752E678
:10E0D00061E08DE79BE20E94771F8EE49DE2DF9175
:10E0E000CF910C94DD5E20E02F77FC018081382FEA
:10E0F00032953F7099F08F7090E0A0E0F3E1880FC7
:10E10000991FAA1FFA95D9F7582F492F3D578A2FE3
:10E1100030FB87F936952078232B21C0811104C06C
:10E1200050E040E020781BC033E8482F4870880F4B
:10E130009FEF930F411102C0392FF7CF932F969580
:10E140002078292B90E0A0E043E1880F991FAA1FB7
:10E150004A95D9F7582F492F8A2F30FB87F9652F19
:10E16000742F922F0895AF92BF92CF92DF92EF92C9
:10E17000FF920F931F93CF93DF9300D000D0CDB7C2
:10E18000DEB761E070E080E090E00E941EDF97FD66
:10E190000AC00091892D10E020E030E0601771077F
:10E1A000820793071CF066E07FE117C042E1469FBB
:10E1B0009001479F300D11248091872D9091882DDB
:10E1C000820F931F0E9448828C01009721F0C12C7E
:10E1D000B6E0DB2E3BC068ED7EE1CE0101960F94E8
:10E1E0000A0FCE0101960E940BDACE0101960F9420
:10E1F000DA0C60E070E0CB014CC2580128E0C29E0E
:10E20000A00CB11C1124C50101965C01DC0114961F
:10E21000ED91FC911597309741F0868197810E948E
:10E22000CCD888E093E10E94CCD8F501808191811F
:10E230008430910509F440C174F08630910509F4E9
:10E24000F2C10CF4D0C00797E1F1C394D8018C91CE
:10E25000C81698F21AC28230910509F449C1039791
:10E26000A1F7A680B780F50183810E9424D966EECC
:10E270007DE1CE0101960F940A0FCE0101960E9416
:10E28000D8D8CE0101960F94DA0CD5018C910E945A
:10E2900024D969ED7DE1CE0101960F940A0FCE01DC
:10E2A00001960E94D8D8CE0101960F94DA0CF501A0
:10E2B000608170E040E050E0818192810E94834063
:10E2C000E1C1A680B780C50102960E94CCD86BEC54
:10E2D0007EE1CE0101960F940A0FCE0101960E94B5
:10E2E000D8D8CE0101960F94DA0CF5016081D69E44
:10E2F000B001112467597C4DCE0101960F940A0F8D
:10E30000CE0101960E94D8D8CE0101960F94DA0C66
:10E310006CEB7EE1CE0101960F940A0FCE010196BF
:10E320000E94D8D8CE0101960F94DA0CD50111962F
:10E330008C91882309F448C0E894F7F8282F229597
:10E340002F70A9F08F7090E0A0E0B3E1880F991FC3
:10E35000AA1FBA95D9F7582F492F2758EA2E20FB24
:10E36000E7F82695EF2DE078FE2EF22A21C099E7F6
:10E37000382F3870880F2FEF290F311102C0922FDC
:10E38000F7CF90FBE7F89695FF2DF078FF2EF92A4E
:10E3900090E0A0E023E1880F991FAA1F2A95D9F7E2
:10E3A000582F492F8A2F8F773E2D3078E32EE82A79
:10E3B000FA0144E650E06F2F7E2F8E2D9F2D0E9494
:10E3C000075568EB7EE102C060EB7EE1CE0101966D
:10E3D0000F940A0FCE0101960E94D8D8CE01019663
:10E3E0000F94DA0C4FC1A680B780C50106960E9433
:10E3F000CCD862EA7EE1CE0101960F940A0FCE01DD
:10E4000001960E94D8D8CE0101960F94DA0CF5013E
:10E410006081D69EB001112467597C4DCE010196D2
:10E420000F940A0FCE0101960E94D8D8CE01019612
:10E430000F94DA0C6AE97EE1CE0101960F940A0F7F
:10E44000CE0101960E94D8D8CE0101960F94DA0C25
:10E45000D50111966C91D69EB001112467597C4D5F
:10E46000CE0101960F940A0FCE0101960E94D8D8D2
:10E47000CE0101960F94DA0C6FE87EE1CE01019691
:10E480000F940A0FCE0101960E94D8D8CE010196B2
:10E490000F94DA0CF5016281738184819581611595
:10E4A00071058105910529F00E9499D96BE87EE1FB
:10E4B0008DCF63E87EE18ACFA680B780C501019643
:10E4C0000E94CCD864E77EE1CE0101960F940A0F3A
:10E4D000CE0101960E94D8D8CE0101960F94DA0C95
:10E4E000F5016081D69EB001112467597C4D6ECF35
:10E4F000A680B78066E67EE1CE0101960F940A0FF2
:10E50000CE0101960E94D8D8CE0101960F94DA0C64
:10E51000F5016081D69EB001112467597C4DCE0172
:10E5200001960F940A0FCE0101960E94D8D8CE0111
:10E5300001960F94DA0C69E57EE1CE0101960F9405
:10E540000A0FCE0101960E94D8D8CE0101960F94F1
:10E55000DA0CD50111968C91882359F0C5010196EA
:10E560000E94737044E650E00E94075566E57EE124
:10E5700002C06EE47EE1CE0101960F940A0FCE0137
:10E5800001960E94D8D8CE0101960F94DA0C61E46E
:10E590007EE1CE0101960F940A0FCE0101960E94F2
:10E5A000D8D8CE0101960F94DA0CF5018281882328
:10E5B00059F0C50102960E94737044E650E00E9433
:10E5C00007556EE37EE102C066E37EE1CE0101966F
:10E5D0000F940A0FCE0101960E94D8D8CE01019661
:10E5E0000F94DA0C69E27EE1CE0101960F940A0FD6
:10E5F000CE0101960E94D8D8CE0101960F94DA0C74
:10E60000D50113968C91882359F0C50103960E9479
:10E61000737044E650E00E94075566E27EE1D6CE74
:10E620006EE17EE1D3CEF501A680B780C5010396E9
:10E630000E94CCD86CE07EE1CE0101960F940A0FC7
:10E64000CE0101960E94D8D8CE0101960F94DA0C23
:10E65000D5018C910E9424D96DEF7DE1CE01019608
:10E660000F940A0FCE0101960E94D8D8CE010196D0
:10E670000F94DA0CF501818192810E945ED968EFD6
:10E680007DE1A4CE0E94B7D9E0CD61E070E080E0EA
:10E6900090E026960FB6F894DEBF0FBECDBFDF9197
:10E6A000CF911F910F91FF90EF90DF90CF90BF908F
:10E6B000AF900895CF92DF92EF92FF92CF93DF93C6
:10E6C000CDB7DEB76A970FB6F894DEBF0FBECDBFE9
:10E6D00041E050E060E870E0CE0101960E9400BF8A
:10E6E00068A579A5CE0101960F943F0F68E2CE018F
:10E6F00001960F94560FEAA5FBA560817181CE01AA
:10E7000045960F94480D68EE7CE0CE0109960F9473
:10E71000480D69E173E1CE010F960F94480DAE01EB
:10E72000475F5F4FBE01615F7F4FCE0145960F94FB
:10E73000B811CE010F960F94DA0CCE0109960F9402
:10E74000DA0C62E2CE0101960F94560FBE016B5EA9
:10E750007F4FCE0101960F943F0F62E2CE010196EA
:10E760000F94560FCE0145960F94DA0C69E2CE0154
:10E7700001960F94560FAE014F5F5F4F6EA17FA1C0
:10E780008CA19DA10E94E71F6B017C01CE01019627
:10E790000F94DA0CC701B6016A960FB6F894DEBF83
:10E7A0000FBECDBFDF91CF91FF90EF90DF90CF9064
:10E7B0000895CF92DF92EF92FF920F931F93CF9322
:10E7C000DF93CDB7DEB729970FB6F894DEBF0FBE43
:10E7D000CDBF48E550E164E082E00E947D5288238D
:10E7E00009F459C060E070E0CB010E941EDF633085
:10E7F00071058105910544F063E070E080E090E0F0
:10E800000E941EDF262F01C024E162E070E080E05C
:10E8100090E029870E941EDF6B017C0161E070E0BF
:10E8200080E090E00E941EDF2985A6018DE79BE233
:10E830000E94FA1D60E070E0CB010E941EDF643090
:10E840007105810591055CF164E070E080E090E085
:10E850000E9473DF78876F8366E574E18E010F5F36
:10E860001F4FC8010F94480DCE0107969F938F93B9
:10E870001F930F931F921F928EE49DE29F938F939D
:10E880000E945A73C8010F94DA0C0FB6F894DEBFD9
:10E890000FBECDBF04C060E070E0CB0104C061E0FA
:10E8A00070E080E090E029960FB6F894DEBF0FBECE
:10E8B000CDBFDF91CF911F910F91FF90EF90DF902F
:10E8C000CF9008950F9300E020E040E060E088E5FD
:10E8D0009DE20F94C30A81E08093572D41E050E000
:10E8E00060E070E081E39DE20E9400BF41E050E003
:10E8F00060E070E089E29DE20E9400BF41E050E0EC
:10E9000060E070E081E29DE20E9400BF41E050E0E3
:10E9100060E070E089E19DE20E9400BF67EA79E172
:10E9200083E19DE20F94480D41E050E060E070E02B
:10E9300089E09DE20F910C9400BF89E09DE20F9465
:10E94000DA0C83E19DE20F94DA0C89E19DE20F94E9
:10E95000DA0C81E29DE20F94DA0C89E29DE20F94D9
:10E96000DA0C81E39DE20D94DA0C8F929F92AF92C4
:10E97000BF92CF92DF92EF92FF920F931F93CF93AC
:10E98000DF93CDB7DEB72C970FB6F894DEBF0FBE7E
:10E99000CDBF8C01FC018185882309F4EDC08DEA8F
:10E9A000C82E8EE0D82E99E0A92E9DE2B92E99248A
:10E9B000939483E496E40F94CF07892B09F4DAC08B
:10E9C00083E496E40F94E807882EFDE08F1719F092
:10E9D0008AE0881247C083E496E40F94720B80911A
:10E9E0001D2D90911E2D892BC9F16091192D7091CB
:10E9F0001A2DCE0101960F94480D1A861986D886D5
:10EA0000CF82BC86AB86AE014F5F5F4FBE01695FB0
:10EA10007F4F8EE49DE20E94E71FCE0101960F9486
:10EA2000DA0C6091092D70910A2D83E496E40F941D
:10EA3000690B69E17DE283E19DE20F94B50D60E031
:10EA400070E089E09DE20F94D80DBC0189E19DE260
:10EA50000F94B50D8EE49DE20E94C558C8010E9436
:10EA6000E4607BC0E8E08E1226C080911D2D90915D
:10EA70001E2D892BC9F0E0914346F0914446028057
:10EA8000F381E02D43E050E064EA79E183E496E429
:10EA9000199560911D2D70911E2D6150710989E1AC
:10EAA0009DE20F94D91259C067E070E083E496E4C8
:10EAB0000E941F4C52C0FBE18F1203C09092112D97
:10EAC0004CC08091112D8823D9F18091122D8B316A
:10EAD00009F443C08B3589F581E488122EC06DE0BE
:10EAE00070E083E496E40E941F4CE12CF12C8091AD
:10EAF0001D2D90911E2DE816F90650F460E270E08D
:10EB000083E496E40E941F4CEFEFEE1AFE0AEFCF6B
:10EB10006DE070E083E496E40E941F4CC8010E94FF
:10EB2000E46063E17DE289E19DE20F94B50D69E166
:10EB30007DE283E496E40F945B0B1092112D0DC0DF
:10EB4000682D772767FD709583E496E40E941F4C3B
:10EB5000682D89E19DE20F94560F8092122D21E0DD
:10EB600080911D2D90911E2D892B09F420E0F80134
:10EB700020831FCF0E9485F00F9406050E94D49039
:10EB80002C960FB6F894DEBF0FBECDBFDF91CF91AC
:10EB90001F910F91FF90EF90DF90CF90BF90AF90BB
:10EBA0009F908F9008951F920F920FB60F9211248D
:10EBB0008F9381E08093702D8F910F900FBE0F90F7
:10EBC0001F9018951F920F920FB60F921124CF929B
:10EBD000DF92EF922F933F934F935F938F939F9387
:10EBE000AF93BF938091692D90916A2DA0916B2D69
:10EBF000B0916C2DC0906D2DD0906E2DE0906F2D4A
:10EC00004E2D9601205C394B484F203452E4350795
:10EC10005FE0450728F48159934FAE4FBF4F08C0BE
:10EC20004E2D96013C5F47408059934FAE4FBF4FEA
:10EC30008093692D90936A2DA0936B2DB0936C2DCA
:10EC400020936D2D30936E2D40936F2DBF91AF911A
:10EC50009F918F915F914F913F912F91EF90DF9016
:10EC6000CF900F900FBE0F901F9018951895209180
:10EC7000E1003091E2006091E300862F90E0A0E097
:10EC8000B0E077276627732B622B2091E400922B4C
:10EC900008952091ED003091EE006091EF00862FF5
:10ECA00090E0A0E0B0E077276627732B622B2091DD
:10ECB000F000922B08950F931F93092F11272227FD
:10ECC00033270093F0008C01222733270093EF00B5
:10ECD000072F182F292F33270093EE006093ED00A4
:10ECE0001F910F910895E6EBF0E0808180628083B0
:10ECF000E1EBF0E08081887F81608083ECEDF0E0E3
:10ED0000808180638083EFEDF0E080818860808384
:10ED1000E8E6F0E0808181608083089578948895AA
:10ED2000F8949091702D911104C0882311F080E027
:10ED300008959091702D911104C09091E00092FF80
:10ED4000EDCF84E08093E00081E08093702D089502
:10ED5000CF92DF92EF92FF92CF939B01AC01A8EE8E
:10ED6000B3E00F94CF176B017C01C4E0F694E794F5
:10ED7000D794C794CA95D1F782E0C816D104E104AC
:10ED8000F10428F4B2E0CB2ED12CE12CF12CCFB73A
:10ED9000F8940E9437766C0D7D1D8E1D9F1D0E947C
:10EDA0005B7684E08093E0001092702DCFBFCF910E
:10EDB000FF90EF90DF90CF900895CF92DF92EF9287
:10EDC000FF920E9449766B017C010E943776209168
:10EDD000E00022FD04C02091702D222321F060E08C
:10EDE00070E0CB0108C0A7019601261B370B480B2A
:10EDF000590BCA01B901FF90EF90DF90CF900895B1
:10EE00002F923F924F925F926F927F928F929F923A
:10EE1000AF92BF92CF92DF92EF92FF920F931F9328
:10EE2000CF93DF93CDB7DEB72D970FB6F894DEBF43
:10EE30000FBECDBF182F20B72B8380E880BF8091F5
:10EE40007A008C8380917A008F7780937A009091FA
:10EE5000C1009D838091C10083FF06C080E00F94B4
:10EE60007807892B09F46DC183B7817F866083BFE2
:10EE700083B7816083BFF894A091B100AE831092F4
:10EE8000B100EDB3EF83F0916B00F887D89A8091D1
:10EE90005E2D90915F2DA091602DB091612D91FF1D
:10EEA00005C080916B00816080936B0080915E2D26
:10EEB00090915F2DA091602DB091612D94FF05C0C0
:10EEC00080916B00826080936B0080915E2D9091A9
:10EED0005F2DA091602DB091612D92FF05C08091B2
:10EEE0006B00846080936B0080915E2D90915F2D0C
:10EEF000A091602DB091612D93FF05C080916B00B2
:10EF0000886080936B0080915E2D82FF05C08091A8
:10EF10006B00806880936B0080915E2D90915F2DD7
:10EF2000A091602DB091612D97FF07C041E050E0A6
:10EF300060E070E082E00F94C30280915E2D9091BA
:10EF40005F2DA091602DB091612DA0FF07C041E021
:10EF500050E060E070E083E00F94C30280915E2D8A
:10EF600090915F2DA091602DB091612D95FF07C00C
:10EF700041E050E060E070E084E00F94C3028091D3
:10EF80005E2D90915F2DA091602DB091612D96FF27
:10EF900007C041E050E060E070E085E00F94C302FC
:10EFA00080915E2D84FF07C040E050E060E070E09B
:10EFB00080E00F94C30280915E2D85FF07C040E082
:10EFC00050E060E070E081E00F94C30280915E2D1C
:10EFD00087FF07C040E050E060E070E086E00F94FB
:10EFE000C30240915E2D50915F2D6091602D709114
:10EFF000612D62FF07C040E050E060E070E087E014
:10F000000F94C3028091E00082FD82C08091DF00F6
:10F0100084608093DF000E9437766B017C01812F32
:10F020000E948E760E9437766C197D098E099F09A1
:10F0300020E130E040E050E00F94421829833A8309
:10F040001A014B018D879C874090622D5090632D53
:10F050006090642D7090652D8091662D9091672D44
:10F06000A091682D89879A87AB8710E4A12E02E4CE
:10F07000B02E8FE0C82ED12CE12CF12C00E010E056
:10F08000A101B4018D859C850F946F1859016A0107
:10F090004A0C5B1C6C1C7D1C90E4A92E22E4B22E51
:10F0A0003FE0C32ED12CE12CF12C00E010E02981AF
:10F0B0003A81A101B4018D859C850F946D18490199
:10F0C0005A0189859A85AB85880D991DAA1D8034C2
:10F0D000E2E49E07EFE0AE0740F080549244AF4078
:10F0E000FFEF4F1A5F0A6F0A7F0A4092622D50921B
:10F0F000632D6092642D7092652D8093662D9093A0
:10F10000672DA093682D8091DF008B7F8093DF00B7
:10F1100083B78E7F83BF288520936B008F818DBB43
:10F1200078949E819093B100AD81A093C100EB8152
:10F13000E0BFFC81F0937A0080917B0087FFFCCFD9
:10F1400006C08091C100877F8093C1008DCE2D962F
:10F150000FB6F894DEBF0FBECDBFDF91CF911F91E8
:10F160000F91FF90EF90DF90CF90BF90AF909F9066
:10F170008F907F906F905F904F903F902F90089569
:10F180000F931F9300915E2D10915F2D2091602DA4
:10F190003091612D6623B1F08F3F61F041E050E086
:10F1A00060E070E004C0440F551F661F771F8A950A
:10F1B000D2F703C040E050E0BA01402B512B622B44
:10F1C000732B19C08F3F61F041E050E060E070E0C8
:10F1D00004C0440F551F661F771F8A95D2F703C0DE
:10F1E00040E050E0BA0140955095609570954023FD
:10F1F00051236223732340935E2D50935F2D6093C0
:10F20000602D7093612D1F910F9108958F3F61F0D4
:10F2100041E050E060E070E004C0440F551F661FFD
:10F22000771F8A95D2F703C040E050E0BA01447BD3
:10F230005E7F6570772781E0452B462B472B09F4CD
:10F2400080E00895FC01408150E09B012D5F3F4F1D
:10F2500042175307B0F042505109461B570BFB01B0
:10F260003196E80FF91F21E030E0819187FD07C05A
:10F27000C90101964217530720F09C01F6CFC9013E
:10F28000089580E090E00895CF93DF93EB0100971D
:10F29000C9F0FC0120812330A8F0318138834CE093
:10F2A0004983313079F430E0225031092D30310575
:10F2B00048F06CE070E00E942279982F8A8381E008
:10F2C000911101C080E0DF91CF910895CF93DF933A
:10F2D000FA01E20FF31F1082F9013197DA01AE0F44
:10F2E000BF1F680F791FEB01C20FD31F88818F7773
:10F2F0008C939F012150310948F0FB01E20FF31F6D
:10F300008181FA01E20FF31F8083F4CFDF91CF9167
:10F310000895CF92DF92EF92FF920F931F93CF93B6
:10F32000DF9300D0CDB7DEB77C01BE016F5F7F4FAA
:10F330000E944479882331F1CB80D12CC6010696F6
:10F340000F942F198C018981F8018083F701828144
:10F35000F8018183F7018381F8018283F7018485B5
:10F36000F8018383A8014B5F5F4F6A8170E09601CB
:10F37000C7010E9466798B819A81890FF801848385
:10F38000C80102C080E090E00F900F900F90DF91D5
:10F39000CF911F910F91FF90EF90DF90CF90089544
:10F3A0000F931F93CF93DF93EA01FC01208130E09C
:10F3B000AB014D5F5F4F2417350708F451C0FC01C6
:10F3C000E60FF71F1181412F50E059834883EFEF7B
:10F3D000E10FE83008F044C022503109261B370BFA
:10F3E000ABE0A49FF001A59FF00D1124E05FFC4D60
:10F3F00004910A83A49FF001A59FF00D1124EF5EF4
:10F40000FC4DE491402F50E02417350748F1DB0113
:10F410001196A80FB91F153099F018F4133021F088
:10F4200013C0183050F010C011964C911197400F36
:10F430004A8350E02417350798F011962C9102C0AA
:10F4400013962C9127FF0EC0EE2361F02A81620FE4
:10F45000711D0E942279982F8B8381E0911104C045
:10F4600080E002C01B8281E0DF91CF911F910F915C
:10F4700008958F929F92AF92BF92CF92DF92EF92B8
:10F48000FF920F931F93CF93DF9300D01F92CDB7BE
:10F49000DEB78C016115710519F0FB01B4800AC05B
:10F4A000BE016F5F7F4F0E9444798823D9F1BB80F2
:10F4B0008A81B80EFB2CD12C6F2D70E0F801808171
:10F4C00090E0029768177907B4F4F801E60FF71F88
:10F4D00081818F3F11F4F394EFCFAE014F5F5F4F07
:10F4E000C8010E94D0798823E9F0D3948C819B8154
:10F4F000890FF80EE1CFF8E0DF9EC00111240196DC
:10F500000F942F197C01FC01D082912C812CA12C0D
:10F5100012C0AE014F5F5F4FB601C8010E94D079A3
:10F52000811113C090E030C0F801EC0DFD1D818108
:10F530008F3F79F7B394CB2CD12CF801808190E0E8
:10F540000297C816D90684F31EC0F70128E0A29ED0
:10F55000E00DF11D1124319689819A819183808378
:10F56000D382C28217821682019729F415821482EF
:10F570009E2E8F2E02C094828582A3948C819B81C3
:10F58000890FB80ED8CFC7010F900F900F900F9032
:10F59000DF91CF911F910F91FF90EF90DF90CF906F
:10F5A000BF90AF909F908F9008953F924F925F923F
:10F5B0006F927F928F929F92AF92BF92CF92DF9283
:10F5C000EF92FF920F931F93CF93DF9300D01F9280
:10F5D000CDB7DEB75C016B01FB0162817381AE01C7
:10F5E0004F5F5F4F0E94D079582E882309F4E0C006
:10F5F000E980FA808BE08E9D40018F9D900C112454
:10F60000C401805F9C4D4C01F601028113810F5FA4
:10F610001F4F0A0D1B1DFC01329634903197E49167
:10F6200044244394E11101C0412CF3E0EF16F104AE
:10F6300021F4F8016180630C01C0632C442059F06F
:10F640008C81811104C0C40103960F94F11D860DB5
:10F6500066246394680E712CC3010F942F19DC018A
:10F66000F60197838683009739F46CEA72E283E4AB
:10F6700096E40F94760B9BC0F4E0EF16F10409F4C6
:10F680004EC0ECF492E0E916F10409F44DC0E3E059
:10F69000EE16F10409F06AC0F80141814C9350E084
:10F6A000C301841B950B8A0F9B1F12969C938E930C
:10F6B0001197B8016E5F7F4F0F94231E57C0F6E07D
:10F6C000EF16F10409F440C06CF097E0E916F1047C
:10F6D00009F04CC0F80181818F738C93828111965F
:10F6E0008C9344C0F80181818F738C9382818F73D6
:10F6F0008C9393819F709B3008F053C084E0989F57
:10F70000F0011124E452FD4D45915591659174919C
:10F7100012964D935D936D937C93159727C0F801D6
:10F7200081818F738C9322C0F80181818F738C93B8
:10F73000828111968C931197838112968C931297E4
:10F74000848113968C9312C0F80181818F778C93FA
:10F7500082818370E82FF0E0EE0FFF1FE85FFC4D21
:10F760008591949112969C938E931197F6018681C0
:10F7700097814420E9F0830D911D2C81222359F0BB
:10F7800030E04B8162817381640F711DAC01C50152
:10F790000E9466790DC0B4016D5F7F4F0F94CB1D41
:10F7A00007C0CD010F94C719F60117821682512C9C
:10F7B000852D0F900F900F900F90DF91CF911F919B
:10F7C0000F91FF90EF90DF90CF90BF90AF909F9000
:10F7D0008F907F906F905F904F903F9008950F9320
:10F7E0001F93CF93DF93EC019A012F5F3F4FFA01F4
:10F7F000008140E00E94E17F182F81110BC068EA70
:10F8000079E183E496E40F949A0B63E476E4CE0105
:10F810000E942E81812FDF91CF911F910F9108952A
:10F82000CF93FC01680F791F80E090E0A1E0E6171C
:10F83000F707C9F0B19128E030E040E8592F551F93
:10F840005527551FC42FCB2309F05A27880F991F1E
:10F85000552321F053ED852757EA952746952150EA
:10F86000310961F7E4CFCF9108958F929F92AF92C3
:10F87000BF92CF92DF92EF92FF920F931F93CF939D
:10F88000DF9300D0CDB7DEB75C01162F03E09E01F9
:10F890002F5F3F4F40E00E94838081110CC06EEBD0
:10F8A00079E183E496E40F949A0B63E476E4C5016E
:10F8B0000E942E8159C08981813071F063ED79E118
:10F8C00083E496E40F94690B4AE050E0698183E495
:10F8D00096E40F948E0C48C00B81802E912CC401AD
:10F8E00001960F942F197C01009739F460EF79E1AC
:10F8F00083E496E40F949A0B37C0F70101936F01EC
:10F900009F0140E0612FC5010E94838081110CC0DE
:10F910006EEB79E183E496E40F949A0B63E476E46A
:10F92000C5010E942E811DC05401F2E0AF1AB1083A
:10F93000B501C6010E94107CF701EA0DFB1D218173
:10F9400030E0322F2227F701E80DF91D4081242BEA
:10F950002817390761F064E17AE183E496E40F94B3
:10F960009A0BC7010F94C71980E090E001C0C7014E
:10F970000F900F900F90DF91CF911F910F91FF90FB
:10F98000EF90DF90CF90BF90AF909F908F900895B1
:10F99000AF92BF92CF92DF92EF92FF920F931F939D
:10F9A000CF93DF9300D01F921F92CDB7DEB78C01AB
:10F9B0007B016A01009731F461157105D1F067E7A9
:10F9C00072E208C0FC01408150E04617570748F436
:10F9D0006EE372E283E496E40F94760B80E090E0AD
:10F9E00081C0822F90E00296860F971F4817590713
:10F9F000B0F4622F70E06D5F7F4F6E0D7F1DC80108
:10FA00002D830F940D1B8C012D81009719F46EE24C
:10FA10007AE129C082E0820F8E0DF8018083C70150
:10FA200030E0CE18DF08AC014E195F0942175307CA
:10FA300080F4AC01435051094830510540F0F601C3
:10FA4000E80FF91F4081F801E80FF91F4183019683
:10FA5000EACF60E070E0C8010E94397A6C0100973B
:10FA600039F46AE57AE183E496E40F949A0BB6CF11
:10FA7000FC01808198E0899FE00DF11D11243897E9
:10FA8000A380B480AE014F5F5F4FB501C8010E94F3
:10FA9000D0798B81EC80F12CE80EF11CEA0CFB1C78
:10FAA0005701E2E0AE0EB11CC6010F94C719F80170
:10FAB000A382808190E0A816B90649F0B7016D5F76
:10FAC0007F4FC8010F940D1B8C01FC01A082B70170
:10FAD000C80101960E94107CF801EE0DFF1D918374
:10FAE0008283C8010F900F900F900F900F90DF91BD
:10FAF000CF911F910F91FF90EF90DF90CF90BF902B
:10FB0000AF900895FC01118210820895262FFC0108
:10FB1000638360E0822F0D9409071F93CF93DF93D7
:10FB2000EC011FEF8B810F9478071150019741F082
:10FB30001111F8CF82E090E09983888380E001C0C2
:10FB400081E0DF91CF911F9108950F931F93CF9381
:10FB5000DF93EC010E948D7D182F882379F10F949B
:10FB600012056C837D838E839F8361E08B810F946C
:10FB7000090760E08B810F9442070F9412050C81F6
:10FB80001D812E813F81601B710B820B930B643CA6
:10FB900079408105910588F360E08B810F94090716
:10FBA000CE010E948D7D182F882341F082E390E0E2
:10FBB0000F945D051C821D821E821F82812FDF91A2
:10FBC000CF911F910F9108950F931F93CF93DF93C0
:10FBD000EC018C819D81AE81BF81892B8A2B8B2B7F
:10FBE00099F10F941205088519852A853B85601BBC
:10FBF000710B820B930B623371058105910588F3BC
:10FC00000F9412050C811D812E813F81601B710BA9
:10FC1000820B930B6C3B72408105910588F30F9426
:10FC200012050C811D812E813F81601B710B820B9F
:10FC3000930B6D3474408105910530F088E090E0BD
:10FC40009983888380E007C00F9412056C837D83BD
:10FC50008E839F8381E0DF91CF911F910F91089553
:10FC6000CF92DF92EF92FF920F931F93CF93DF9388
:10FC7000EC01062F0E94E47D8823C9F1CE010E9489
:10FC80008D7D182F882399F161E08B810F940907EE
:10FC90000F941205CC80DD80EE80FF806C197D0909
:10FCA0008E099F096D3771058105910588F3002341
:10FCB00021F060E08B810F9409070F941205CC802E
:10FCC000DD80EE80FF806C197D098E099F096A38FE
:10FCD00072408105910588F360E08B810F940907DC
:10FCE0000F941205688779878A879B8701C010E087
:10FCF000812FDF91CF911F910F91FF90EF90DF90B7
:10FD0000CF900895CF92DF92EF92FF920F931F93BF
:10FD1000CF93DF93EC018B010E94E47D882329F0CF
:10FD2000CE010E948D7D811102C010E04AC061E0C9
:10FD30008B810F9409070F941205CC80DD80EE8033
:10FD4000FF806C197D098E099F096D37710581054A
:10FD5000910588F360E08B810F9409070F941205D9
:10FD6000CC80DD80EE80FF806C197D098E099F09B3
:10FD70006E3571408105910588F38B810F9478076A
:10FD800021E0892B09F420E0F80120830F9412056B
:10FD90000C811D812E813F81601B710B820B930BA7
:10FDA0006A3872408105910588F3CE010E948D7DED
:10FDB000182F882331F00F941205688779878A8776
:10FDC0009B87812FDF91CF911F910F91FF90EF9033
:10FDD000DF90CF900895EF92FF920F931F93CF93F0
:10FDE000DF931F92CDB7DEB77C0105E110E0015033
:10FDF000110961F0BE016F5F7F4FC7010E94827ED3
:10FE0000882351F09981992391F306C081E090E015
:10FE1000F7019183808380E00F90DF91CF911F9154
:10FE20000F91FF90EF9008950F931F93CF93DF935F
:10FE30001F921F92CDB7DEB78C01BE016E5F7F4F60
:10FE40000E94827E882399F0BE016F5F7F4FC801B8
:10FE50000E94827E882359F09A812981911109C0DC
:10FE6000211107C086E090E0F8019183808380E053
:10FE700015C021110EC0B8016E5F7F4FC8010E94EE
:10FE80000880882319F083E090E0EECF84E090E0D2
:10FE9000EBCF992319F085E090E0E6CF0F900F901B
:10FEA000DF91CF911F910F910895CF92DF92EF9242
:10FEB000FF920F931F93CF93DF93EC01D62E08E0B0
:10FEC00010E080E8E82EF12CCC24C3949E2D9D21D7
:10FED00009F0FC2461E0911101C060E0CE010E94B4
:10FEE000307E8823D9F0E6940150110979F761E05A
:10FEF0006F25CE010E94307E882381F0CE010E94C2
:10FF0000EB7E882359F0CE01DF91CF911F910F91A5
:10FF1000FF90EF90DF90CF900C94147F80E0DF9102
:10FF2000CF911F910F91FF90EF90DF90CF900895A8
:10FF3000EF92FF920F931F93CF93DF931F92CDB752
:10FF4000DEB78C017B01460F4E1559F0F701619128
:10FF50007F01C80149830E94557F49818111F4CFF7
:10FF600001C081E00F90DF91CF911F910F91FF9021
:10FF7000EF900895EF92FF921F93CF93DF931F921C
:10FF8000CDB7DEB77C01142F69830E94A57D6981FE
:10FF9000882379F0C7010E94557F882351F0612F93
:10FFA000C7010F90DF91CF911F91FF90EF900C94BC
:10FFB000557F80E00F90DF91CF911F91FF90EF90E0
:10FFC0000895EF92FF920F931F93CF93DF93EC016D
:10FFD000142F790142E00E94BA7F882389F0612FB3
:10FFE000CE010E94557F882359F0402FB701CE01E2
:10FFF000DF91CF911F910F91FF90EF900C94987F1C
:020000021000EC
:1000000080E0DF91CF911F910F91FF90EF900895C5
:100010009F92AF92BF92CF92DF92EF92FF920F9397
:100020001F93CF93DF931F92CDB7DEB78C017B0177
:10003000FB01108298E0C92ED12C20E8A22EB12C11
:1000400099249394BE016F5F7F4FC8010E94827E06
:10005000882339F18981882329F0F70180818A2951
:100060008083B924A694F1E0CF1AD10859F7BE01D4
:100070006F5F7F4FC8010E94827E882391F0898143
:100080008B1106C087E090E0F8019183808309C05E
:10009000C8010E94EB7E882321F0C8010E94147FD2
:1000A00001C080E00F90DF91CF911F910F91FF90E1
:1000B000EF90DF90CF90BF90AF909F900895EF9218
:1000C000FF920F931F93CF93DF931F92CDB7DEB7AD
:1000D0007C019B01460F421769F089010F5F1F4F9A
:1000E000B901C70149830E9408804981882319F01A
:1000F0009801F1CF81E00F90DF91CF911F910F9187
:10010000FF90EF900895EF92FF920F931F93CF937C
:10011000DF93EC01142F790141E00E94BA7F88231C
:1001200089F0612FCE010E94557F882359F0402F1E
:10013000B701CE01DF91CF911F910F91FF90EF900A
:100140000C945F8080E0DF91CF911F910F91FF9021
:10015000EF9008957F928F929F92AF92BF92CF922D
:10016000DF92EF92FF920F931F93CF93DF93CDB760
:10017000DEB728970FB6F894DEBF0FBECDBF8C0157
:100180006B010E94A57D882309F44CC06EEFC80165
:100190000E94557F882309F445C03FE7932E8824A9
:1001A00083944FE2742ECE0101967C01A12CB12CD8
:1001B000B701C8010E940880811103C0A1103AC094
:1001C00031C0F70141917F0188E090E020E83B2DAC
:1001D000331F3327331F522F542309F03825BB0C0C
:1001E0003111B7242695019791F7A394F8E0AF1247
:1001F000DFCFBB2019F089E090E010C0CE0101965E
:10020000F60119959A9479F6BE016F5F7F4FC80188
:100210000E940880882331F08AE090E0F801918301
:10022000808307C081E0F8012081318125303105CC
:1002300009F080E028960FB6F894DEBF0FBECDBF60
:10024000DF91CF911F910F91FF90EF90DF90CF90B2
:10025000BF90AF909F908F907F9008950F931F93C2
:10026000CF93DF938C01EB01FC01608171816B30D6
:10027000710558F4FB01EE0FFF1FE25FFD4F608137
:100280007181CE010F94690B05C04AE050E0CE01A8
:100290000F944F0CF80180819181039781F469E7F5
:1002A0007AE1CE010F94690B40E150E0F8016281E0
:1002B000CE01DF91CF911F910F910D948E0CDF91A4
:1002C000CF911F910F9108950F9300E020E040E03F
:1002D00060E081E79DE20F94C30A0F910895CF93E8
:1002E000DF93EC012091892D30E02F5F3F4F82E1B9
:1002F000829FB001839F700D11248091872D909172
:10030000882D0F940D1BDC019093882D8093872DF1
:100310008091892D91E0980F9093892D92E1899F8A
:10032000A00DB11D112419961C921E9218971B96B0
:100330001C921E921A971D961C921E921C974FEFAC
:100340005FEFBA011E964D935D936D937C93519729
:1003500088E0FE0101900D928A95E1F7DF91CF913F
:1003600008950895BC0183E496E40F94690B63E457
:1003700076E48BE79DE20E942E8183E496E40F945D
:10038000720B80E00895CF93DF93EC018885998507
:100390000097C9F48091872D9091882D9E01281B8C
:1003A000390BC9019595879529E33EE8829FB001F5
:1003B000839F700D929F700D11248BE79DE20E9428
:1003C000357C99878887DF91CF910895CF93DF930C
:1003D000EC01888599850F94C71919861886DF91D5
:1003E000CF9108950F931F93CF93DF93EC010A856C
:1003F0001B850115110569F460E070E00E94C3815E
:10040000892B39F0888599850E9489798C019B8791
:100410008A87C801DF91CF911F910F910895CF93E3
:10042000DF93EC018A859B850F94C7191B861A867A
:10043000DF91CF910895FF920F931F93CF93DF9396
:100440008C01FC0184859585892BE1F0F12CF80164
:1004500084859585FC012081F21678F4EC01F8E0A2
:10046000FF9EC00DD11D112421968E819F810F9476
:10047000C7191F821E82F394EACF0F94C719F8019F
:1004800015861486DF91CF911F910F91FF900895EB
:10049000FF920F931F93CF93DF93EC010C851D8583
:1004A0000115110559F560E070E00E94C381892BA8
:1004B00029F16A857B85888599850E94397A9D878F
:1004C0008C87892BD9F0F12CEC85FD858081F8167D
:1004D000A0F4BF0188E0F89E600D711D11246F5FCC
:1004E0007F4F888599850E94D57A811104C0CE01FD
:1004F0000E941B8203C0F394E7CF8F01C801DF91F4
:10050000CF911F910F91FF900895AF92BF92CF921C
:10051000DF92EF92FF920F931F93CF93DF93EC0143
:100520004E855F85688979894F3F8FEF5807680747
:10053000780709F08DC0CE010E944882A12C40E0CE
:1005400050E0BA01E6E0BE2E01E010E020E030E02D
:10055000DC01EC91AE1608F077C0FC01A8E0AA9E81
:10056000E00DF11D11243196A081B181A530B105B6
:10057000A1F034F4A230B10559F0149749F062C0EB
:10058000A630B10509F43DC0179709F43DC05AC023
:100590000680F781E02DC0801EC0A681B781CC9077
:1005A000BC9CF0011124E859FC4DE491EF3F51F05F
:1005B0006801790104C0CC0CDD1CEE1CFF1CEA951F
:1005C000D2F703C0C12CD12C76014C295D296E29AC
:1005D0007F291196CC90BC9CF0011124E859FC4D68
:1005E000E491EF3F51F06801790104C0CC0CDD1CAF
:1005F000EE1CFF1CEA95D2F721C0C12CD12C76014C
:100600001DC0506861601EC00680F781E02DC0806B
:10061000BC9CF0011124E859FC4DE491EF3F51F0EE
:100620006801790104C0CC0CDD1CEE1CFF1CEA95AE
:10063000D2F703C0C12CD12C76015C614C295D2915
:100640006E297F29A39484CF4E875F87688B798B2F
:10065000CB01642F752FDF91CF911F910F91FF90E8
:10066000EF90DF90CF90BF90AF9008950F931F93BE
:10067000CF93DF93082F10E08091892D1817F0F4A5
:1006800082E1189FE00111248091872D9091882D9F
:100690008C0F9D1F0E940F828091872D9091882D35
:1006A0008C0F9D1F0E94E6818091872D9091882D4F
:1006B0008C0F9D1F0E941B821F5FDECF0023A1F0C5
:1006C0008091872D9091882D0F94C7191092882DB5
:1006D0001092872D1092892D1092772D1092782DDF
:1006E0001092792D10927A2DDF91CF911F910F9159
:1006F000089540E02091892D421780F4E091872DE4
:10070000F091882D22E1429FE00DF11D11242281FC
:1007100031818217930721F04F5FECCF80E008957D
:1007200081E00895CF92DF92EF92FF92CF93C0E0E5
:10073000C12CD12C76018091892DC81788F4809125
:10074000872D9091882D22E1C29F800D911D11244B
:100750000E948582C62AD72AE82AF92ACF5FEBCFE2
:10076000C092772DD092782DE092792DF0927A2D4B
:10077000CF91FF90EF90DF90CF900895CF93DF93CC
:100780001F92CDB7DEB781E00E9436836FE671E835
:100790008BE79DE20E94AA80811107C084E09BE163
:1007A0000F90DF91CF910C94B28189830E94928344
:1007B00089810F90DF91CF910895882341F065E002
:1007C00070E080E090E00F9435050C94BE8381E0EA
:1007D0000C9436838091012C9091022C90932702E7
:1007E0008093260284E292E09093022C8093012C65
:1007F00065E070E080E090E00F94350563E18BE701
:100800009DE20E94867D0E94BE8381E090E00E946E
:100810007983882321F082E29BE10E94099280E0A3
:100820000C9436830F9300E020E040E060E08AE81B
:100830009DE20F94C30A8BE79DE20F910C94827D99
:1008400023EE3BE1FC01318320830895A091902D9C
:10085000B091912D109749F0ED91FC911197019075
:10086000F081E02D682FCD011994089523EE3BE12E
:10087000FC01318320830D94F60ACF93DF93EC01C2
:100880008FEE9BE199838883CE014A960E9440C2F5
:1008900083EE9BE199838883DF91CF910895CF9375
:1008A000DF93EC010E943D84CE01DF91CF910D9446
:1008B000F60A0F931F93CF93DF938B01EC01080F80
:1008C000191FC017D10721F089910E9480D8F9CF54
:1008D000DF91CF911F910F910C94B7D90F931F9374
:1008E000CF93DF93EC018B011C8A1B8A1A8A198A29
:1008F0001D8A1E8A1F8A188E0E94111A8CB58C7F41
:1009000081608CBD8DB58E7F8DBD80EE97E89F8F09
:100910008E8FDBA3CAA3FE01E150FD4F83E496E472
:1009200091838083329611821082F80183816A96C6
:1009300021E530E08131C9F445E067E0CE010E9455
:10094000EDCE882381F00091301D1091311D0115ED
:10095000110569F022E33DE140E067E27BE1CE0171
:100960000E947AD504C080E003C04FEFE6CF81E05B
:10097000DF91CF911F910F910895CF93DF93EC01F9
:100980008FEE9BE199838883CE014A961D821C825B
:1009900048EE53E060E070E04E835F8368877987BC
:1009A0009F878E872FEF288B24E43AE23B832A83AC
:1009B000198E0E9413C2CD5FDC4F1882DF91CF9158
:1009C00008959F92AF92BF92CF92DF92EF92FF92E3
:1009D0000F931F93CF93DF93B62EA72E8A01EC01BE
:1009E0006A961F921F928DE29BE19F938F93DF93F4
:1009F000CF930E942BCE982E0F900F900F900F90B8
:100A00000F900F9001151105B9F1F801808188232D
:100A100099F16801E12CF12CF60181916F01882395
:100A200079F0FBE1EF16F10489F0992787FD9095A5
:100A30000F948C1D892B51F0FFEFEF1AFF0AECCFBA
:100A4000E894E4F82AE0E216F104B1F1992009F4FF
:100A50005AC01F930F9384E49BE19F938F93DF937E
:100A6000CF930E942BCE0F900F900F900F900F906E
:100A70000F90811104C047C0992009F444C01F920F
:100A80001F9287EA99E19F938F93AF92BF921F9233
:100A90001F9281E59BE19F938F93DF93CF930E94F9
:100AA0002BCEEDB7FEB73C960FB6F894FEBF0FBE47
:100AB000EDBF811116C027C0992029F11F930F9314
:100AC00088E39BE19F938F93DF93CF930E942BCE7C
:100AD0000F900F900F900F900F900F90882399F028
:100AE000B8CF1F921F9288E69BE19F938F93DF936D
:100AF000CF930E942BCE0F900F900F900F900F90DE
:100B00000F90811102C080E011C01F921F928FE6EA
:100B10009BE19F938F93DF93CF930E942BCE0F90F7
:100B20000F900F900F900F900F9081E0DF91CF9179
:100B30001F910F91FF90EF90DF90CF90BF90AF90FB
:100B40009F900895CF93DF93AB01EC016A9661E02B
:100B5000CE010E9454D3882321F11F921F9288E670
:100B60009BE19F938F93DF93CF930E942BCE0F90A7
:100B70000F900F900F900F900F90882391F01F927D
:100B80001F928FE69BE19F938F93DF93CF930E94F9
:100B90002BCE0F900F900F900F900F900F9081E041
:100BA00001C080E0DF91CF910895AF92BF92CF92C4
:100BB000DF92EF92FF920F931F93CF93DF931F92D9
:100BC0001F92CDB7DEB77B016A014A965C0140E017
:100BD00050E060E029833A830E9454D329813A810E
:100BE000882389F1A601B701C5010E947ED388231D
:100BF00051F1B801C5010E9411D4882321F11F923F
:100C00001F9288E69BE19F938F93BF92AF920E94C1
:100C10002BCE0F900F900F900F900F900F90882376
:100C200091F01F921F928FE69BE19F938F93BF924B
:100C3000AF920E942BCE0F900F900F900F900F90BD
:100C40000F9081E001C080E00F900F90DF91CF9175
:100C50001F910F91FF90EF90DF90CF90BF90AF90DA
:100C600008950F931F93CF93DF93EC01FC01ED5F89
:100C7000FC4F80818823E9F00F94060568387341A2
:100C80008105910530F460EA7FE080E090E00F9408
:100C900035056A9600E010E020E041E060E0CE011A
:100CA0000E94C6D5CE01DF91CF911F910F910C9478
:100CB00031D3DF91CF911F910F9108950F931F931F
:100CC000CF93DF93EC010E943186FE01ED5FFC4F74
:100CD00081E08083898D882339F041E064E670E00B
:100CE00088EE90E30E9472BD6A961F921F921F9237
:100CF0008BE08F9386E79BE19F938F93DF93CF9356
:100D00000E942BCE00E010E020E041E061E0CE0147
:100D10000E94C6D52DB73EB7285F3F4F0FB6F89457
:100D20003EBF0FBE2DBFDF91CF911F910F91089550
:100D3000EF92FF920F931F93CF93DF93CDB7DEB760
:100D40002D970FB6F894DEBF0FBECDBF8C01CE013C
:100D500008960F94B90A6091A62D7091A72D40E0D6
:100D600050E0CE0108960E94A0C2811138C0409187
:100D7000A62D5091A72DB801665E7F4FCE0101963A
:100D80000E94DDD44B815C816D817E814A875B87C7
:100D90006C877D878091942D9091952DA091962DB3
:100DA000B091972D481759076A077B07C1F48091C6
:100DB000112C882309F490C066EE74E283E496E473
:100DC0000F94360B66EA7DE283E496E40F945B0BA6
:100DD0006DEC74E283E496E40F94760B49C0809145
:100DE000112C8823E1F068EB74E283E496E40F941D
:100DF000360B66EA7DE283E496E40F945B0B6FECBE
:100E00007DE083E496E40F94690B60912C0270916D
:100E10002D024AE050E083E496E40F94B20C409136
:100E20002C0250912D0280EA9AE29A8389838A8566
:100E30009B85AC85BD858B839C83AD83BE83780108
:100E400082E0E80EF11CBE016F5F7F4FC7010E9478
:100E500048D6892B79F48091112C882331F06BE8E6
:100E600074E283E496E40F94760BC8010E945E86D8
:100E700080E032C08091A52D882371F067E27BE18C
:100E8000C7010E940BD6811107C08091112C8823C5
:100E900061F366E574E2E5CFF801818D882321F0E6
:100EA00088EE90E30E9499BC0E94CC32F8018389BD
:100EB00094890196948B838B0E94AE2D29833A836B
:100EC0004B835C8389819A81AB81BC81F801858BDE
:100ED000968BA78BB08F81E02D960FB6F894DEBF6E
:100EE0000FBECDBFDF91CF911F910F91FF90EF907B
:100EF00008950F931F93CF93DF93CDB7DEB7279756
:100F00000FB6F894DEBF0FBECDBF8C014A960E948B
:100F100039D2F80185899689A789B08D892B8A2BCA
:100F20008B2B09F442C00280F381E02D0488F589FF
:100F3000E02DC80102961995811137C08091112CBE
:100F40008823F9F06EE274E283E496E40F94360BA2
:100F50000E94AE2D29833A834B835C8349815A8159
:100F60006B817C81F80185899689A789B08D481BA2
:100F7000590B6A0B7B0B2AE030E083E496E40F9474
:100F8000C80CD80155961D921D921D921C9258971F
:100F9000C80127960FB6F894DEBF0FBECDBFDF9114
:100FA000CF911F910F910C94988627960FB6F894C5
:100FB000DEBF0FBECDBFDF91CF911F910F9108957E
:100FC000CF92DF92EF92FF920F93CF93DF93CDB743
:100FD000DEB72C970FB6F894DEBF0FBECDBF7C01F5
:100FE000FC01818992890196928B818B148A138AE4
:100FF000818D882321F088EE90E30E94E7BC8091E8
:10100000A52D8823B1F16701FAE1CF0ED11C4BE881
:101010005BE1B601CE0101960E94DDD48B819C81FB
:10102000AD81BE814091942D5091952D6091962D6A
:101030007091972D84179507A607B70769F00AE006
:1010400020E831E541E050E0BE016F5F7F4FC6010F
:101050000E946DD481110DC08091112C882331F034
:1010600069EF74E283E496E40F94760BC7010E9463
:101070005E8668E97BE18EE49DE20E94135E882330
:1010800009F447C068E97BE1CE0107960F94480D4B
:1010900080914F2D882361F067E17BE083E496E443
:1010A0000F94360B6F81788583E496E40F949A0B46
:1010B0008091502D882341F01092912D1092902D07
:1010C00086E294E80E94C2D88F8198850E94EEF053
:1010D0008091502D81110E94C7D869ED7CE0CE012E
:1010E00001960F94480DBE016F5F7F4FCE010796AA
:1010F0000F947D10D82ECE0101960F94DA0CDD20CE
:1011000021F08EE49DE20E94C558CE0107960F940F
:10111000DA0CC7010E9498862C960FB6F894DEBFB1
:101120000FBECDBFDF91CF910F91FF90EF90DF9079
:10113000CF900895CF93DF93EC014A960E9410D28E
:10114000C350DD4F81E09881911101C080E0DF91B3
:10115000CF910895CF93DF93EC012296DC01129694
:10116000ED91FC9113970488F589E02DCE01199536
:10117000882369F08091A52D882359F0CE010E9423
:1011800012D691E0811101C090E0892F03C080E068
:1011900001C081E0DF91CF91089580E0089580E063
:1011A0000895CF93DF93EC016A965F934F938DE69A
:1011B00099E29F938F93DF93CF930E941BCE20E001
:1011C00030E040E050E069E574E8CE010E94C4CB15
:1011D00021E00F900F900F900F900F900F90892BA0
:1011E00009F020E0822FDF91CF9108950F931F9394
:1011F000CF93DF93EC018B010F94060568387341A0
:101200008105910530F460EA7FE080E090E00F9482
:1012100035054AEA5BE1B801CE01DF91CF911F911C
:101220000F910C94D18840EB5BE10C94D1880F9323
:101230001F93CF93DF93EC018B0145EB5BE10E94A1
:10124000D18840EC5BE1B801CE01DF91CF911F91D5
:101250000F910C94D18849EC5BE10C94D18880E02B
:10126000089580E0089542ED5BE10C94D188DC01A3
:10127000A150BD4FFC01EF5FFC4F83E496E48D93DA
:101280009C93662319F091838083089511821082C4
:1012900008950F9300E020E040E060E082E99DE2E5
:1012A0000F94C30A0F9108958AEF98E20895CF939F
:1012B000DF9300D000D0CDB7DEB780919D2D909107
:1012C0009E2D892B81F46BE578E2CE0101960F9477
:1012D0000A0FCE0101960E940BDACE0101960F94FF
:1012E000DA0C80E001C081E026960FB6F894DEBFEC
:1012F0000FBECDBFDF91CF910895CF93DF930E94B2
:101300005789882349F1C0919D2DD0919E2D60E091
:1013100070E0CB010E941EDF672B682B692B71F0F8
:1013200061E070E080E090E00E941EDF21E0672B2A
:10133000682B692B09F420E0822F01C081E0898F9E
:10134000882329F0CE010E949A88882349F0698D6C
:1013500070E080E090E00CC060E070E0CB0108C07D
:1013600041E064E670E088EE90E30E9472BDEFCF4A
:10137000DF91CF91089561E478E281E00E94A94E67
:101380008823C1F061E070E080E090E00E941EDF01
:1013900021E0672B682B692B09F420E0622F8091F4
:1013A0009D2D90919E2D0E94378961E070E080E034
:1013B00090E0089560E070E0CB010895CF93DF9353
:1013C00000D000D0CDB7DEB70E9457898823B9F08E
:1013D00080919D2D90919E2D0E943189811113C085
:1013E0006EE178E2CE0101960F940A0FCE010196CC
:1013F0000E940BDACE0101960F94DA0C04C060E073
:1014000070E0CB0104C061E070E080E090E02696DF
:101410000FB6F894DEBF0FBECDBFDF91CF91089518
:10142000CF93DF9300D000D0CDB7DEB70E945789AD
:101430008823B9F080919D2D90919E2D0E942F8937
:10144000811113C06CEF77E2CE0101960F940A0F61
:10145000CE0101960E940BDACE0101960F94DA0CB0
:1014600004C060E070E0CB0104C061E070E080E0A7
:1014700090E026960FB6F894DEBF0FBECDBFDF9189
:10148000CF910895CF93DF9300D000D0CDB7DEB7D2
:101490000E9457898823C9F063E476E480919D2DEA
:1014A00090919E2D0E943389811113C060ED77E2E7
:1014B000CE0101960F940A0FCE0101960E940BDA1D
:1014C000CE0101960F94DA0C04C060E070E0CB010D
:1014D00004C061E070E080E090E026960FB6F894DA
:1014E000DEBF0FBECDBFDF91CF910895CF93DF93C5
:1014F00000D000D0CDB7DEB76EEA77E281E00E947F
:10150000A94E811104C060E070E0CB0127C00E94A9
:1015100057898823C1F361E070E080E090E00E9489
:1015200073DFAB0163E476E480919D2D90919E2D55
:101530000E94CD8881110EC067E877E2CE01019646
:101540000F940A0FCE0101960E940BDACE0101968C
:101550000F94DA0C61E070E080E090E026960FB620
:10156000F894DEBF0FBECDBFDF91CF910895CF932A
:10157000DF9300D000D0CDB7DEB76AE677E281E036
:101580000E94A94E811104C060E070E0CB0127C029
:101590000E9457898823C1F361E070E080E090E009
:1015A0000E9473DFAB0163E476E480919D2D9091FE
:1015B0009E2D0E94CF8881110EC069E477E2CE0192
:1015C00001960F940A0FCE0101960E940BDACE010C
:1015D00001960F94DA0C61E070E080E090E02696CE
:1015E0000FB6F894DEBF0FBECDBFDF91CF91089547
:1015F000CF93DF9300D000D0CDB7DEB76AE277E2B9
:1016000081E00E94A94E811104C060E070E0CB012E
:1016100027C00E9457898823C1F361E070E080E011
:1016200090E00E9473DFAB0163E476E480919D2D2E
:1016300090919E2D0E94D18881110EC067E077E2C3
:10164000CE0101960F940A0FCE0101960E940BDA8B
:10165000CE0101960F94DA0C61E070E080E090E03A
:1016600026960FB6F894DEBF0FBECDBFDF91CF91A7
:1016700008950E945789882359F080919D2D90915B
:101680009E2D0E94318661E070E080E090E0089538
:1016900060E070E0CB0108950E945789882359F0DB
:1016A00080919D2D90919E2D0E945E86682F70E006
:1016B00080E090E0089560E070E0CB0108950F9322
:1016C0001F93CF93DF93CDB7DEB7E0970FB6F894B3
:1016D000DEBF0FBECDBF61ED76E284E00E94A94E71
:1016E000882309F4A5C00E945789882309F4A0C063
:1016F000CE018B960F94B90ACE0185960F94B90A44
:10170000CE014F960F94B90ACE0149960F94B90AAB
:1017100061E070E080E090E00E9473DF40E050E024
:10172000CE018B960E94A0C2811103C067EB76E2C6
:1017300073C062E070E080E090E00E9473DF40E000
:1017400050E0CE0185960E94A0C2811103C060EADC
:1017500076E262C063E070E080E090E00E9473DFB8
:1017600040E050E0CE014F960E94A0C2811103C01C
:1017700069E876E251C063E070E080E090E00E94AA
:1017800073DF40E050E0CE0149960E94A0C2811173
:1017900003C06FE676E240C020EA3AE23C8B2B8B36
:1017A0008B8D9C8DAD8DBE8D8D8B9E8BAF8BB88FB1
:1017B0003E872D8789A19AA1ABA1BCA18F87988B69
:1017C000A98BBA8B38872F838FA198A5A9A5BAA515
:1017D00089879A87AB87BC873A8329838DA59EA585
:1017E000AFA5B8A98B839C83AD83BE838E010D5EAC
:1017F0001F4F9E01235F3F4FAE01495F5F4FBE0108
:101800006F5F7F4F80919D2D90919E2D0E94D58579
:10181000811112C06CE276E2CE0101960F940A0F9C
:10182000CE0101960E940BDACE0101960F94DA0CDC
:1018300060E070E0CB0104C061E070E080E090E027
:10184000E0960FB6F894DEBF0FBECDBFDF91CF910B
:101850001F910F910895CF93DF9300D000D0CDB7A3
:10186000DEB70E945789882351F160E070E0CB0118
:101870000E941EDF16161706180619063CF461E0D2
:1018800070E080E090E00E9473DF02C060E070E0F2
:1018900080919D2D90919E2D0E94A285811113C053
:1018A00069EE75E2CE0101960F940A0FCE01019602
:1018B0000E940BDACE0101960F94DA0C04C060E0AE
:1018C00070E0CB0104C061E070E080E090E026961B
:1018D0000FB6F894DEBF0FBECDBFDF91CF91089554
:1018E000CF93DF93CDB7DEB7C654D1090FB6F894C6
:1018F000DEBF0FBECDBF46EB55E262E081E00E9445
:101900007D52811104C060E070E0CB0145C00E94AF
:1019100057898823C1F360E070E0CB010E941EDF8D
:10192000623071058105910549F462E070E080E064
:1019300090E00E9473DF40E450E004C040E450E0D7
:1019400067EA79E1CE0101960F94821E61E070E0B2
:1019500080E090E00E9473DFAE014F5F5F4F8091A7
:101960009D2D90919E2D0E94E184811111C063E70D
:1019700075E2CE018F5B9F4F0F940A0FCE018F5BF4
:101980009F4F0E940BDACE018F5B9F4F0F94DA0CB2
:1019900061E070E080E090E0CA5BDF4F0FB6F89442
:1019A000DEBF0FBECDBFDF91CF910895CF93DF9300
:1019B00000D000D0CDB7DEB70E9457898823C1F090
:1019C00063E476E480919D2D90919E2D0E94F6888F
:1019D000811112C060E675E2CE0101960F940A0FE4
:1019E000CE0101960E940BDACE0101960F94DA0C1B
:1019F00060E070E0CB0104C061E070E080E090E066
:101A000026960FB6F894DEBF0FBECDBFDF91CF9103
:101A100008950E9457898823F1F060E070E0CB01BF
:101A20000E941EDF1616170618061906C4F461E098
:101A300070E080E090E00E941EDF6130710581055A
:101A4000910569F463E476E480919D2D90919E2D3B
:101A50000E94138914C060E070E0CB01089563E434
:101A600076E480919D2D90919E2D0E942B8963E4B8
:101A700076E480919D2D90919E2D0E94178961E0C2
:101A800070E080E090E008950F931F93CF93DF9371
:101A9000CDB7DEB727970FB6F894DEBF0FBECDBF28
:101AA00060ED78E2CE0101960F940A0FCE01019607
:101AB0000E94D8D8CE0101960F94DA0CE0919D2DAA
:101AC000F0919E2D818992890E9417DA6BE978E264
:101AD000CE0101960F940A0FCE0101960E94D8D82C
:101AE000CE0101960F94DA0CE0919D2DF0919E2D80
:101AF000838994890E9417DA67E778E2CE0101961C
:101B00000F940A0FCE0101960E94D8D8CE010196FB
:101B10000F94DA0CE0919D2DF0919E2D8589968988
:101B2000A789B08D892B8A2B8B2BE1F00E94AE2DDB
:101B300029833A834B835C836D837E838F83E0911B
:101B40009D2DF0919E2D69817A818B819C810589E3
:101B500016892789308D601B710B820B930B0E94B5
:101B60001BDA04C080E090E00E9413DA27960FB6DB
:101B7000F894DEBF0FBECDBFDF91CF911F910F91C3
:101B800008952F923F924F925F926F927F928F9221
:101B90009F92AF92BF92CF92DF92EF92FF920F93FC
:101BA0001F93CF93DF93CDB7DEB76F970FB6F8943F
:101BB000DEBF0FBECDBF41E050E064E670E08E01B5
:101BC0000F5F1F4FC8010E9400BF0E9457898111FB
:101BD00009C041E050E060E070E0CE0109960E944B
:101BE00000BFB5C080909D2D90909E2DF4018589F9
:101BF0009689A789B08D892B8A2B8B2BB9F00E94EF
:101C0000AE2D298B3A8B4B8B5C8B6D8B7E8B8F8BA8
